:100000000C944F190C9480190C9480190C9480193D
:100010000C9480190C9480190C9480190C948019FC
:100020000C9480190C9480190C9480190C948019EC
:100030000C9480190C9480190C9480190C948019DC
:100040000C9480190C9423990C9480190C948019A9
:100050000C9480190C9480190C94A2C80C94B0CF05
:100060000C9480190C9431510C9480190C948019C3
:100070000C9480190C9480190C9480190C9480199C
:100080000C9480190C9480190C9480190C9480198C
:100090000C948AD30C94C0D30C9480190C948019BE
:1000A0000C9480190C9480190C9480190C9480196C
:1000B0000C9480190C9480190C9480190C9480195C
:1000C0000C9480190C9480190C9480190C9480194C
:1000D0000C9480190C9480190C9480190C9480193C
:1000E0000C948019364736474147414741474C47B2
:1000F0004C474C476147574757475747365D425D26
:100100004E5D5A5D665D015D0D5DDBC8EBC80AC9D9
:100110000FC912C917C91AC91FC922C927C92AC9B3
:100120002FC932C937C941C9F1D0F6D0FBD005D1AA
:100130000FD188D119D121D129D133D13DD147D186
:1001400056D160D188D16AD174D17ED1AAD1ADD136
:100150009CD1A0D1A6D1E4D1B1D1B5D1BBD1BFD171
:10016000C3D1C9D1CDD1D1D1E4D1D7D1DBD1DFD168
:10017000084AD73B3BCE016E84BCBFFDC12F3D6C0E
:1001800074319ABD56833DDA3D00C77F11BED9E474
:10019000BB4C3E916BAAAABE000000803F05A84C54
:1001A000CDB2D44EB93836A9020C50B99186880820
:1001B0003CA6AAAA2ABE000000803F0048617264E3
:1001C000636F6465642053442044656661756C7494
:1001D0002053657474696E6773204C6F6164656445
:1001E000006F6B2000496E666F3A20002020256961
:1001F000204B6D202569206D20256920636D202509
:1002000069206D6D0046696C616D656E7420707259
:10021000696E7465643A00496E666F3A2000496EF3
:10022000666F3A20002020256920646179732025BB
:100230006920686F757273202569206D696E757409
:10024000657300506F776572206F6E2074696D65FD
:100250003A00496E666F3A200046696C616D656EC2
:10026000742073657474696E67733A2044697361AE
:10027000626C656400436F6E6669673A20002020F7
:100280004D323030204400436F6E6669673A20007B
:1002900046696C616D656E742073657474696E6710
:1002A000733A00436F6E6669673A2000204400206D
:1002B000490020500020204D333031204800436F4A
:1002C0006E6669673A20005049442073657474690A
:1002D0006E67733A00436F6E6669673A20002028A4
:1002E0004D6174657269616C2047554D2900204647
:1002F0000020420020204D31343520533220480068
:10030000436F6E6669673A200020284D61746572FC
:1003100069616C20414253290020460020420020A0
:10032000204D313435205331204800436F6E6669CB
:10033000673A200020284D6174657269616C205015
:100340004C41290020460020420020204D31343508
:10035000205330204800436F6E6669673A20004D95
:100360006174657269616C20686561747570207074
:100370006172616D65746572733A00436F6E666990
:10038000673A2000205A0020590020580020204DB4
:10039000323138205400436F6E6669673A20004856
:1003A0006F74656E64206F666673657420286D6D6A
:1003B000293A00436F6E6669673A2000205A002090
:1003C000590020204D323036205800436F6E666948
:1003D000673A2000486F6D65206F6666736574200C
:1003E000286D6D293A00436F6E6669673A200020D8
:1003F0004500205A002058002042002056002020AE
:100400004D323035205300436F6E6669673A2000E5
:10041000416476616E636564207661726961626CC5
:1004200065733A20533D4D696E206665656472615F
:10043000746520286D6D2F73292C20563D4D696EF3
:100440002074726176656C2066656564726174659E
:1004500020286D6D2F73292C20423D6D696E696DCA
:10046000756D207365676D656E742074696D6520A8
:10047000286D73292C20583D6D6178696D756D204C
:100480005859206A65726B20286D6D2F73292C20B6
:10049000205A3D6D6178696D756D205A206A6572CC
:1004A0006B20286D6D2F73292C2020453D6D6178C0
:1004B000696D756D2045206A65726B20286D6D2F02
:1004C000732900436F6E6669673A2000205200204E
:1004D000204D323034205400436F6E6669673A20F5
:1004E0000020560020204D323034205000436F6EE3
:1004F0006669673A2000416363656C65726174697F
:100500006F6E733A20503D7072696E74696E672C1D
:1005100020563D74726176656C20616E6420542AA9
:1005200020523D7265747261637400436F6E666938
:10053000673A2000204500205A0020590020204D15
:10054000323031205800436F6E6669673A20004DA3
:100550006178696D756D20416363656C6572617466
:10056000696F6E20286D6D2F7332293A00436F6ECC
:100570006669673A2000204500205A002059002073
:10058000204D323033205800436F6E6669673A2041
:10059000004D6178696D756D206665656472617482
:1005A000657320286D6D2F73293A00436F6E66695D
:1005B000673A2000204500205A0020590020204D95
:1005C0003932205800436F6E6669673A20005374D1
:1005D0006570732070657220756E69743A00436FA0
:1005E0006E6669673A200048617264636F6465648F
:1005F0002044656661756C742053657474696E6718
:1006000073204C6F61646564004563686F3A200035
:1006100020496E76616C696420686F74656E640051
:100620004D004572726F723A200020496E76616CFF
:100630006964206578747275646572004D00457256
:10064000726F723A20005072696E74657220686130
:100650006C7465642E206B696C6C28292063616C56
:100660006C656421004572726F723A20004B494CF0
:100670004C45442E20006F6B20006F6B20005265AC
:1006800073656E643A200020496E76616C6964205F
:1006900065787472756465720054004563686F3ADA
:1006A00020004D3330302053363539205032303031
:1006B0000A4D333030205336393820503230300034
:1006C0004F6666736574206170706C6965642E0096
:1006D0004F6666736574206170706C6965642E0086
:1006E0004563686F3A20004D33303020533430205A
:1006F00050323030004572723A20546F6F2066617C
:10070000722100546F6F206661722066726F6D20D7
:100710007265666572656E636520706F696E7400E0
:100720004572726F723A2000496E76616C6964207E
:100730006578747275646572004572726F723A20E2
:100740000020643A0020693A0020703A00483A00DC
:100750006F6B20002C002C002000486F74656E64C5
:10076000206F6666736574733A004563686F3A205C
:100770000053657474696E672054726176656C20ED
:10078000416363656C65726174696F6E3A20004500
:1007900063686F3A200053657474696E6720526510
:1007A000747261637420416363656C65726174691E
:1007B0006F6E3A20004563686F3A20005365747489
:1007C000696E67205072696E7420416363656C6561
:1007D000726174696F6E3A20004563686F3A200059
:1007E00053657474696E67205072696E7420616E0F
:1007F000642054726176656C20416363656C657238
:100800006174696F6E3A20004563686F3A20005644
:100810006F6C756D65747269632044697361626C95
:10082000656400496E666F3A2000566F6C756D65A1
:100830007472696320456E61626C656400496E661E
:100840006F3A20007A5F6D696E3A2000795F6D69BA
:100850006E3A2000785F6D696E3A20005265706FC5
:100860007274696E6720656E6473746F7020737440
:1008700061747573004563686F3A20004649524DB4
:10088000574152455F4E414D453A4D4B5F342E32F4
:100890002E385F646576204649524D574152455F78
:1008A00055524C3A68747470733A2F2F67697468A4
:1008B00075622E636F6D2F4D61676F4B696D62724C
:1008C000612F4D61726C696E4B696D62726120506F
:1008D000524F544F434F4C5F56455253494F4E3A37
:1008E000322E30204D414348494E455F54595045C2
:1008F0003A43617274657369616E2045585452556C
:100900004445525F434F554E543A31205555494462
:100910003A30303030303030302D303030302D30D3
:100920003030302D303030302D30303030303030CD
:1009300030303030300A00205A3A0020593A002036
:10094000436F756E7420583A0020453A00205A3A99
:100950000020593A00583A004B494C4C45442E204F
:1009600000444542554720454E41424C45440045D0
:1009700063686F3A2000444542554720445259521B
:10098000554E20454E41424C4544004563686F3A00
:100990002000444542554720494E464F20454E4190
:1009A000424C4544004563686F3A20004445425537
:1009B00047204543484F20454E41424C4544004561
:1009C00063686F3A200048656174696E6720646FE0
:1009D0006E652E003F0020573A0048656174696ECD
:1009E000672E2E2E006F6B20004B3430204C61732D
:1009F0006572204F46462E004563686F3A200025F9
:100A000069206D696E2C2025692073656300456E31
:100A1000642066696C65206C69737400426567695F
:100A20006E2066696C65206C697374004E6F206D72
:100A30006F76652E005374617274205072696E7403
:100A4000696E67004563686F3A200053746F7020C9
:100A50005072696E74696E67004563686F3A200072
:100A60004B3430204C617365722072656164792E5D
:100A700000526573756D696E67207072696E7400DF
:100A80005761697420666F7220757365722E2E2E01
:100A9000003A0020002D3E00205300526573746F11
:100AA00072696E6720706F736974696F6E00456359
:100AB000686F3A2000496E76616C696420736C6FD0
:100AC000742C20746F74616C20736C6F74733A2093
:100AD000004572726F723A200020453A00205A3A5F
:100AE0000020593A003C2D583A00205300536176BB
:100AF000656420706F736974696F6E004563686F19
:100B00003A2000496E76616C696420736C6F742CB6
:100B100020746F74616C20736C6F74733A2000459D
:100B200072726F723A2000203E2028686F6D655FF8
:100B30006F66667365745B617869735D3D3D0073D4
:100B400065745F617869735F69735F61745F686F13
:100B50006D652000496E666F3A2000546865204834
:100B60006F6D696E672042756D70204665656472B1
:100B70006174652044697669736F722063616E6E7B
:100B80006F74206265206C657373207468616E20D9
:100B900031004572726F723A200029003C3C3C20C3
:100BA000686F6D65617869732800496E666F3A20D9
:100BB00000496E666F3A2000496E666F3A20002940
:100BC000003E3E3E20686F6D65617869732800497C
:100BD0006E666F3A2000496E666F3A20003C3C3CDE
:100BE0002067636F64655F47323800496E666F3A0D
:100BF0002000496E666F3A200047323800202D2DC4
:100C00004C4556454C20504C415445205343524985
:100C100050542D2D004563686F3A2000496E666F71
:100C20003A2000496E666F3A200067636F64655F23
:100C3000473238203E3E3E00496E666F3A200050F3
:100C40006F73697469766520526173746572204CA4
:100C5000696E6500496E666F3A20004E6567617483
:100C600069766520526173746572204C696E650007
:100C7000496E666F3A2000536C6565702E2E2E000B
:100C80004563686F3A2000556E6B6E6F776E206318
:100C90006F6D6D616E643A2022004572726F723A18
:100CA000200020403A00202F00543A0029002C2038
:100CB000002C20003A2028004563686F3A20002568
:100CC0006920686F757273202569206D696E75746F
:100CD000657300446F6E65207072696E74696E672B
:100CE0002066696C65004B494C4C45442E200053EE
:100CF000544F505045442E20005072696E746572F6
:100D00002073746F707065642064756520746F2043
:100D10006572726F72732E20466978207468652040
:100D20006572726F7220616E6420757365204D3933
:100D3000393920746F20726573746172742E2028A3
:100D400054656D7065726174757265206973207287
:100D5000657365742E205365742069742061667410
:100D600065722072657374617274696E67290045DB
:100D700072726F723A20004E6F204C696E65204E81
:100D8000756D626572207769746820636865636B4E
:100D900073756D2C204C617374204C696E653A201C
:100DA000004E6F20436865636B73756D20776974BF
:100DB00068206C696E65206E756D6265722C204CC2
:100DC000617374204C696E653A2000636865636BDB
:100DD00073756D206D69736D617463682C204C614F
:100DE0007374204C696E653A20004C696E65204E24
:100DF000756D626572206973206E6F74204C61732B
:100E000074204C696E65204E756D6265722B312CB5
:100E1000204C617374204C696E653A20004D31316D
:100E200030004572726F723A20006F6B20004D32B5
:100E3000390020506C616E6E65724275666665722F
:100E400042797465733A200046726565204D656D80
:100E50006F72793A2000436F6D70696C65643A2057
:100E60004170722031392032303136004C61737458
:100E700020557064617465643A2041707220313984
:100E800020323031362030323A33393A3039207C12
:100E900020417574686F723A2028446F776E756EC2
:100EA00064657233356D2C204B3430204C61736592
:100EB0007229004D4B5F342E322E385F6465760008
:100EC0007374617274002200656E71756575656971
:100ED0006E672022004563686F3A2000FFFFFF0025
:100EE00000A0400000A04000000040000000000002
:100EF000000000000000000080A8430000664300DE
:100F00000048430000000000000000000000000056
:100F100080A8430000664300004843536F6674771F
:100F2000617265205265736574005761746368640B
:100F30006F672052657365740042726F776E206F21
:100F400075742052657365740045787465726E61BE
:100F50006C20526573657400506F77657255700030
:100F60004C6173657220657874696E677569736822
:100F7000656400496E666F3A20004C6173657220AB
:100F8000666972656400496E666F3A2000534420BA
:100F900072656D6F76656400534420696E73657287
:100FA000746564004D343238002D2D2D2E2D2D000A
:100FB0002D2D2D002D2D2D002D2D2D00452D2D3AC3
:100FC0002D2D00532D2D3A2D2D00452D2D3A2D2D53
:100FD000002D2D2D250025004730205A2573204651
:100FE00031353000473238205A2046313530004301
:100FF0007573746F6D00437573746F6D00376D6D2D
:1010000000366D6D202D20312F34696E00356D6DE9
:1010100000346D6D00336D6D202D20312F38696ED9
:1010200000326D6D00316D6D004C6173657220464C
:10103000756E6374696F6E73004D3830005761725E
:101040006D2D7570204C617365722032736563007D
:1010500031353030203130306D7300313530302053
:101060002035306D730031303030203130306D73C9
:101070000031303030202035306D73002038303072
:10108000203130306D730020383030202035306D05
:1010900073004C617365722046756E6374696F6E80
:1010A000730054657374204669726500536574203B
:1010B000466F637573004D61696E00473238205882
:1010C0002059204200466978206178697320737442
:1010D00065707300466C6F7700466C6F77004661F1
:1010E0006E2073706565640046616E20737065657F
:1010F00064004E6F7A7A6C65004E6F7A7A6C650088
:101100004E6F7A7A6C65004E6F7A7A6C6500537018
:10111000656564005370656564004D61696E0047E4
:1011200032380020202020202020202020202020B5
:1011300020202020200020424544206C6576656CEC
:10114000656421202020202020200020507265731B
:10115000732074686520627574746F6E202020009F
:10116000202020204973206974206F6B3F202020AD
:101170002020202000205072657373207468652041
:10118000627574746F6E202020002041646A75734C
:101190007420666F7572746820706F696E740020B9
:1011A00050726573732074686520627574746F6E15
:1011B000202020002041646A75737420746869726D
:1011C0006420706F696E7420002050726573732004
:1011D00074686520627574746F6E20202000204151
:1011E000646A757374207365636F6E6420706F69D1
:1011F0006E74002050726573732074686520627588
:1012000074746F6E202020002041646A757374200E
:10121000666972737420706F696E7420002050725A
:101220006573732074686520627574746F6E202016
:101230002000204C6576656C696E67206265642EBF
:101240002E2E2020202000473238204D004D616E88
:1012500075616C20426564204C6576656C696E67CB
:10126000004D6F76652058004D6F76652059004D12
:101270006F7665205A004578747275646572004512
:1012800078747275646572004D6F7665205A004DF2
:101290006F76652059004D6F76652058004D6F764A
:1012A000652061786973004D6F766520302E316D51
:1012B0006D004D6F766520316D6D004D6F76652048
:1012C00031306D6D004D6F74696F6E00436F6F6CE0
:1012D000646F776E004D38340044697361626C65E9
:1012E000207374657070657273004D6F7665206150
:1012F000786973004D616E75616C20426564204CA5
:101300006576656C696E670053657420686F6D65FE
:10131000206F666673657473004732382058205911
:10132000204632303030004175746F20686F6D6533
:10133000004D61696E0045302073746570732F6DC8
:101340006D0045302073746570732F6D6D00412DF5
:1013500072657472616374453000412D72657472F8
:10136000616374453000416D617820453000416D06
:10137000617820453000566D617820453000566D0B
:1013800061782045300056652D6A65726B453000E6
:1013900056652D6A65726B4530005A20737465700E
:1013A000732F6D6D005A2073746570732F6D6D000F
:1013B000592073746570732F6D6D005920737465B7
:1013C00070732F6D6D00582073746570732F6D6D81
:1013D00000582073746570732F6D6D00412D747209
:1013E0006176656C00412D74726176656C00416DAB
:1013F0006178205A00416D6178205A00416D617812
:10140000205900416D6178205900416D6178205864
:1014100000416D61782058005654726176206D69E4
:101420006E005654726176206D696E00566D696E5D
:1014300000566D696E00566D6178205A00566D61D8
:1014400078205A00566D6178205900566D617820D9
:101450005900566D6178205800566D61782058000B
:10146000567A2D6A65726B00567A2D6A65726B002A
:101470005678792D6A65726B005678792D6A657297
:101480006B00416363656C00416363656C00436F8F
:101490006E74726F6C00526573746F726520666152
:1014A000696C73616665004D6F74696F6E004D61A4
:1014B000696E00463A2569204B6D202569206D2014
:1014C000256920636D202569206D6D004F6E2078A1
:1014D0003A20256964202569682025696D004D3210
:1014E00034004D323320257300022E2E004D6169E9
:1014F0006E004E6F205344005072696E7420667205
:101500006F6D2053440053746F70207072696E7455
:1015100000526573756D65207072696E740050615C
:10152000757365207072696E7400537461746973A9
:101530007469637300436F6E74726F6C00507265F0
:10154000706172650054756E65004C617365722040
:1015500046756E6374696F6E7300496E666F2073B3
:10156000637265656E0000060900FE0701920321A3
:1015700020FFFF08FF07FF0000000600000107072B
:101580000602008080808080008003020206010540
:10159000A0A00507070600005050F850F85050056D
:1015A00007070600002078A07028F020050707062E
:1015B0000000C0C81020409818050707060000600A
:1015C00090A040A89068020303060104C040800375
:1015D000070706010020408080804020030707069F
:1015E00001008040202020408005050506000120E4
:1015F000A870A8200505050600012020F82020027B
:1016000003030602FFC04080050101060003F80243
:101610000202060200C0C0050505060001081020F0
:101620004080050707060000708888888888700356
:10163000070706010040C040404040E0050707069C
:101640000000708808708080F8050707060000F821
:101650001020100808F00507070600001030509011
:10166000F81010050707060000F880F008088870D9
:10167000050707060000708080F08888700507075E
:10168000060000F8081020202020050707060000AB
:101690007088887088887005070706000070888841
:1016A00078080870020505060200C0C000C0C0022C
:1016B00006060602FFC0C000C040800407070600FF
:1016C0000010204080402010050303060002F800AF
:1016D000F80407070601008040201020408005071D
:1016E0000706000070880810200020050707060084
:1016F0000070880868A8A8700507070600007088B1
:1017000088F8888888050707060000F08888F08830
:1017100088F00507070600007088808080887005C3
:101720000707060000F08888888888F00507070604
:101730000000F88080F08080F8050707060000F8B8
:101740008080F0808080050707060000708880B8E0
:10175000888870050707060000888888F8888888C8
:1017600001070706020080808080808080050707CF
:1017700006000038101010109060050707060000E2
:101780008890A0C0A0908805070706000080808090
:10179000808080F805070706000088D8A888888818
:1017A000880507070600008888C8A8988888050764
:1017B000070600007088888888887005070706007B
:1017C00000F08888F0808080050707060000708898
:1017D0008888A89068050707060000F08888F0A0B0
:1017E0009088050707060000788080700808F005DB
:1017F0000707060000F82020202020200507070604
:101800000000888888888888700507070600008897
:1018100088888888502005070706000088888888FF
:1018200088A850050707060000888850205088883F
:101830000507070600008888885020202005070734
:10184000060000F80810204080F803070706010092
:10185000E08080808080E005050506000180402052
:101860001008030707060100E02020202020E005E3
:101870000303060004205088050101060000F80259
:101880000202060205804005050506000070087882
:1018900088780507070600008080B0C88888F005B2
:1018A00005050600007080808870050707060000A7
:1018B000080868988888780505050600007088F88B
:1018C00080700507070600003048E04040404005B2
:1018D00006060600FF70888878087005070706006E
:1018E000008080B0C8888888010707060200800051
:1018F00080808080800308080601FF2000202020CF
:1019000020A040040707060000808090A0C0A0909F
:10191000030707060100C04040404040E0050505C0
:10192000060000D0A8A8A8A8050505060000B0C8B4
:101930008888880505050600007088888870050677
:10194000060600FFF08888F080800506060600FF86
:10195000788888780808050505060000B0C88080EA
:101960008005050506000070807008F00407070672
:1019700000004040E040404030050505060000887A
:101980008888986805050506000088888850200525
:1019900005050600008888A8A85005050506000072
:1019A00088502050880506060600FF888888780839
:1019B00070050505060000F8102040F8030707062B
:1019C00001002040408040402001070706020080BF
:1019D00080808080808003070706010080404020CF
:1019E00040408005020206000268900000000600E8
:1019F00000000000060000000000060000000000DB
:101A000006000000000006000000000006000000C4
:101A100000000600000000000600000000000600B4
:101A200000000000060000000000060000000000AA
:101A30000600000000000600000000000600000094
:101A40000000060000000000060000000000060084
:101A5000000000000600000000000600000000007A
:101A60000600000000000600000000000600000064
:101A70000000060000000000060000000000060054
:101A8000000000000600000000000600000000004A
:101A90000600000000000600000000000600000034
:101AA0000000060000000000060000000000060024
:101AB0000000000006000001070706020080008009
:101AC000808080800507070600002070A8A0A8700D
:101AD00020050707060000304040E04050A80505FB
:101AE000050600008870507088050707060000880A
:101AF0005020F820F82001070706020080808000AF
:101B00008080800508080600003048205050209052
:101B100060030101060107A0050707060000F88819
:101B2000B8B8B888F8050707060001700878887803
:101B300000F80505050600012850A05028050303FC
:101B4000060001F8080802020206020640800507A6
:101B500007060000F888A88898A8F8050101060083
:101B600006F8040404060003609090600507070669
:101B700000002020F8202000F8040505060003607E
:101B8000902040F0030505060003E020E020E0027D
:101B9000020206020640800508080600FF888888C1
:101BA0008898E880800507070600007898987818DC
:101BB0001818020202060202C0C00202020602FF58
:101BC000408003050506000340C04040E0050707CC
:101BD000060001708888887000F805050506000178
:101BE000A0502850A00507070600008890A858B804
:101BF00008080507070600008890B84898203805AF
:101C00000808060000C040C048D838080805070783
:101C100006000020002040808870050808060000AB
:101C20004020007088F88888050808060000102009
:101C3000007088F8888805080806000020500070A9
:101C400088F888880508080600006890007088F801
:101C500088880508080600005000708888F8888881
:101C60000508080600002050207088F888880507BD
:101C7000070600003860A0B8E0A0B8050808060014
:101C8000FF7088808088702060050808060000408A
:101C90002000F880F080F805080806000008100011
:101CA000F880F080F8050808060000205000F88051
:101CB000F080F80507070600005000F880F080F873
:101CC000030808060100804000E0404040E00308AF
:101CD00008060100204000E0404040E003080806FC
:101CE000010040A000E0404040E00307070601007B
:101CF000A000E0404040E0050707060000704848AB
:101D0000E848487005080806000068900088C8A8E0
:101D10009888050808060000402070888888887028
:101D2000050808060000102070888888887005085B
:101D30000806000020500070888888700508080692
:101D40000000689000708888887005080806000008
:101D50005000708888888870050505060001885045
:101D60002050880508080600FF1070A8A8A8A870D1
:101D7000400508080600004020888888888870058B
:101D800008080600001020888888888870050808E0
:101D90000600002050008888888870050808060022
:101DA00000500088888888887005080806000010A0
:101DB000208850202020200509090600FFC040701F
:101DC0004848704040E00408080601FF609090A079
:101DD0009090E08005080806000040200070087818
:101DE00088780508080600001020007008788878B8
:101DF000050808060000205000700878887805085B
:101E000008060000689000700878887805070706C3
:101E10000000500070087888780508080600002047
:101E200050207008788878050606060000D02878CB
:101E3000A0A8500506060600FF7080887020600587
:101E400008080600004020007088F8807005080827
:101E50000600001020007088F88070050808060051
:101E6000002050007088F8807005070706000050B9
:101E7000007088F880700308080601008040004068
:101E8000C04040E003080806010020400040C04078
:101E900040E003080806010040A00040C04040E0C8
:101EA000030707060100A00040C04040E005070707
:101EB000060000A040A01078887005080806000001
:101EC000689000B0C888888805080806000040208F
:101ED00000708888887005080806000010200070CF
:101EE00088888870050808060000205000708888DF
:101EF000887005080806000068900070888888705F
:101F000005070706000050007088888870050505E1
:101F10000600012000F800200507070600FF1070EA
:101F2000A8A8A8704005080806000040200088887E
:101F3000889868050808060000102000888888989E
:101F40006805080806000020500088888898680501
:101F50000707060000500088888898680509090668
:101F600000FF102000888888F80870040707060121
:101F7000FFC04060506040E00508080600FF5000C8
:101F800088888878087000060900FE0000000000BC
:101F900001090008FE000005080806000040F0C81E
:101FA0008888987810050808060000C0F888888896
:101FB0008888F80505050600012030F8302005085E
:101FC000080600002070F820202020E005090906FE
:101FD00000FF2070A8A8B8888870200509090600AD
:101FE000FFE080C0B0A8283028280509090600FFB6
:101FF000F8A88888888888A8F8050A0A0600FE20BC
:102000005050505088A8A88870030303060003406E
:10201000A040FFF08F108F109F909F908010801035
:1020200080108010801080108010FFF0FFF08F1063
:102030008F109F909F90801086108610C630A650FB
:102040009690AF50FFF003FFFFFFFFFFFFFFFFFF82
:10205000FFFFFFC00FFFFFFFFFFFFFFFFFFFFFFFBF
:10206000FFF01E00000000000000000000000078EB
:10207000380000000000000000000000001C70009C
:1020800000000000000000000000000E60000000E2
:1020900000300000000001000006E01F7C0000335B
:1020A0000000000001800387C03FFE0000330000F5
:1020B000000001C00283C073CE00003000000000A9
:1020C00003C00383C0F3CE3C0F330F00000003C0F6
:1020D0000283C0E38E7E1FB31F8000001FE0000359
:1020E000C0E38EE739B339C00000FFFC0383C0E3CF
:1020F0008EC331B338C000003FFF0203C0E38EC37C
:10210000303338C0000007F00203C0E38EE3303301
:1021100038C0000107F00383C0E38EFBF03FF8C036
:10212000000383F00003C0638E7BF01FF8C000073C
:10213000C1F80003C00000000000000000039FFE83
:102140000003C0000000000000000000FFFF80430B
:10215000E00000000000000000007FFFF8C3F00076
:10216000000000000300000033FFFFC3F800003050
:10217000F0000300000019FFFF83FC000071E6007F
:10218000030000000C7FFF03FE000073C600030085
:102190000000067FFF03FF000077800003000000BF
:1021A000033FFE03FF80007F067FE3F0F0F0019F16
:1021B000FC03FFC0007E06FFF3F9F9F800CFF80337
:1021C000FFE0007C06E7339B9B9C0067F003FFF079
:1021D000007E06E31B1B1B0C0033C003FFF8007FCF
:1021E00006E31B1B030C00190003FFFC007386E3CE
:1021F0001B3B038C000C0003FFFE0071C6E31BF3C6
:1022000003EF00060007FFFF0030E66319E301EF6C
:1022100000020006FFFF8000000000000000000038
:10222000000EFFFFC0000000000000000000001CC6
:10223000FFFFE00000000000000000000078FFFF4A
:10224000FFFFFFFFFFFFFFFFFFFFFFF0FFFFFFFFAD
:10225000FFFFFFFFFFFFFFFFFFC04C6173657220B0
:10226000666972696E6720656E61626C65640049BB
:102270006E666F3A200053746570726174652074E5
:102280006F6F20686967683A20004C61736572203F
:10229000666972696E67206475726174696F6E2019
:1022A000656C61707365642C20696E20696E74655D
:1022B00072727570742066617374206C6F6F700039
:1022C000496E666F3A2000506978656C3A20004C80
:1022D0003A2000593A2000583A20004C6173657248
:1022E000207374617475732073657420746F206F2C
:1022F00066662C20696E20696E74657272757074E2
:102300002068616E646C657200496E666F3A2000E9
:102310004C6173657220666972696E6720647572BC
:102320006174696F6E20656C61707365642C2069DF
:102330006E20696E746572727570742068616E6467
:102340006C657200496E666F3A20004D3834205833
:102350002059205A204500656E6473746F70732095
:102360006869743A205A00205A3D00656E6473749F
:102370006F7073206869743A20590020593D0065D8
:102380006E6473746F7073206869743A205800200B
:10239000583D00656E6473746F7073206869743A99
:1023A00020004563686F3A200024F4D43050C38E77
:1023B00020C2A24017828B7011127A910D816CD9C4
:1023C0000AA861E108C7586607615143061E4B5DC4
:1023D00005C145A7041A411104093D98037139311B
:1023E000034036DB0265339102D4305402802E1D47
:1023F00002632CEE01752AC501B028A001102781C7
:10240000018F2564012B244B01E0223401AC211FF4
:10241000018D200D01801FFC00841EED00971DDF43
:1024200000B81CD200E61BC600201BBC00641AB218
:1024300000B219A8000A19A0006A189900D11791D2
:102440000040178B00B516840031167E00B3157955
:10245000003A157300C7146F0058146A00EE136633
:10246000008813630025135E00C7125B006C1257CF
:102470000015125400C111510070114F0021114B71
:1024800000D61049008D104700461044000210424B
:1024900000C00F4000800F3E00420F3C00060F3B83
:1024A00000CB0E3800930E37005C0E3500270E343B
:1024B00000F30D3200C10D3100900D3000600D2E83
:1024C00000320D2D00050D2C00D90C2B00AE0C296F
:1024D00000850C29005C0C2700350C27000E0C260B
:1024E00000E80B2400C40B2400A00B23007D0B2369
:1024F000005A0B2100390B2100180B2000F80A1F8D
:1025000000D90A1E00BB0A1E009D0A1D00800A1D7C
:1025100000630A1C00470A1B002C0A1B00110A1A40
:1025200000F7091A00DD091900C4091900AB0919DF
:1025300000920917007B091800630917004C09165F
:102540000036091600200916000A091500F50815BD
:1025500000E0081400CC081400B8081400A4081403
:1025600000900813007D0812006B08130058081231
:102570000046081200340811002308110012081147
:102580000001081100F0071000E0071000D007104C
:1025900000C0071000B0070F00A107100091070E40
:1025A0000083070F0074070F0065070E0057070E22
:1025B0000049070E003B070D002E070E0020070DF7
:1025C0000013070D0006070D00F9060C00ED060DBF
:1025D00000E0060C00D4060C00C8060C00BC060C7B
:1025E00000B0060C00A4060B0099060C008D060B2B
:1025F0000082060B0077060B006C060B0061060AD2
:102600000057060B004C060A0042060A0038060A6C
:10261000002E060A0024060A001A060A00100609FF
:102620000007060A00FD050900F4050900EB05098D
:1026300000E2050900D9050900D0050900C7050910
:1026400000BE050900B5050800AD050800A505098F
:10265000009C050800940508008C05080084050806
:10266000007C050800740508006C05070065050876
:10267000005D050700560508004E050700470507E1
:10268000004005080038050700310507002A050746
:1026900000230507001C050600160507000F0507A7
:1026A000000805060002050700FB040600F5040704
:1026B00000EE040600E8040600E2040700DB04065E
:1026C00000D5040600CF040600C9040600C30406B2
:1026D00000BD040600B7040600B1040500AC040602
:1026E00000A6040600A00405009B0406009504054E
:1026F00000900406008A0405008504050080040695
:10270000007A04050075040500700405006B0405DB
:102710000066040500610405005C0405005704051B
:1027200000520405004D040500480405004304055B
:10273000003E0404003A040500350405003004049A
:10274000002C04050027040400230405001E0404D3
:10275000001A04040016040500110404000D04040A
:1027600000090405000404040000040400FC030440
:1027700000F8030400F4030400F0030400EC030475
:1027800000E8030400E4030400E0030400DC0304A5
:1027900000D8030400D4030400D0030400CC0304D5
:1027A00000C8030300C503030024F404D9201BC49C
:1027B0000C5C0E9804C4095F0265077101F405F909
:1027C00000FB04B30048048700C1036900580355A7
:1027D0000003034500BE023A008402310053022A7E
:1027E000002902250004022000E4011C00C8011990
:1027F00000AF01170098011400840113007101104B
:10280000006101100051010E0043010D0036010B63
:10281000002B010B0020010B00150109000C010920
:102820000003010800FB000800F3000800EB0007AC
:1028300000E4000600DE000600D8000600D2000614
:1028400000CC000500C7000500C2000500BD000463
:1028500000B9000400B5000400B1000400AD00049C
:1028600000A9000400A5000300A20003009F0004CB
:10287000009B0003009800030095000200930003F2
:1028800000900003008D0002008B0003008800020E
:10289000008600020084000300810002007F000225
:1028A000007D0002007B0002007900020077000139
:1028B0000076000200740002007200010071000244
:1028C000006F0002006D0001006C0002006A000150
:1028D0000069000200670001006600010065000158
:1028E000006400020062000100610001006000015C
:1028F000005F0002005D0001005C0001005B000160
:10290000005A000100590001005800010057000161
:102910000056000100550001005400010053000062
:10292000005300010052000100510001005000015D
:10293000004F0001004E0000004E0001004D00015C
:10294000004C0001004B0000004B0001004A000158
:102950000049000100480000004800010047000154
:10296000004600000046000100450000004500014F
:102970000044000100430000004300010042000049
:102980000042000100410000004100010040000140
:10299000003F0000003F0001003E0000003E00013B
:1029A000003D0000003D0001003C0000003C000034
:1029B000003C0001003B0000003B0001003A000029
:1029C000003A000100390000003900010038000021
:1029D0000038000000380001003700000037000117
:1029E000003600000036000000360001003500000F
:1029F0000035000000350001003400000034000004
:102A000000340001003300000033000000330001F7
:102A100000320000003200000032000100310000EE
:102A200000310000003100010030000000300000E3
:102A300000300001002F0000002F0000002F0000D8
:102A4000002F0001002E0000002E0000002E0001CB
:102A5000002D0000002D0000002D0000002D0001C1
:102A6000002C0000002C0000002C0000002C0001B5
:102A7000002B0000002B0000002B0000002B0001A9
:102A8000002A0000002A0000002A0000002A00019D
:102A90000029000000290000002900000029000092
:102AA0000029000100280000002800000028000084
:102AB0000028000000280001002700000027000077
:102AC000002700000027000000270001002600006A
:102AD000002600000026000000260000002600015D
:102AE0000025000000250000002500000025000052
:102AF0000025000000250001002400000024000043
:102B00000024000000240000002400010023000035
:102B10000023000000230000002300000023000029
:102B2000002300000023000100220000002200001A
:102B3000002200000022000000220000002200010C
:102B40000021000000210000002100000021000001
:102B500000210000002100000021000100200000F1
:102B600000200000002000000020000000200000E5
:102B7000002000000020000000200001001F0000D5
:102B8000001F0000001F0000001F0000001F0000C9
:102B9000001F0000001F0001001E0000001E0000BA
:102BA000001E0000001E0000007C3C3E5E2B3D3FEE
:102BB0002F5B5D3B2C2A225C000000211042206329
:102BC000308440A550C660E770088129914AA16B06
:102BD000B18CC1ADD1CEE1EFF1311210027332529E
:102BE00022B5529442F772D662399318837BB35A56
:102BF000A3BDD39CC3FFF3DEE3622443342004016E
:102C000014E664C774A44485546AA54BB5288509A5
:102C100095EEE5CFF5ACC58DD5533672261116303D
:102C200006D776F6669556B4465BB77AA7199738F5
:102C300087DFF7FEE79DD7BCC7C448E5588668A77D
:102C4000784008611802282338CCC9EDD98EE9AF45
:102C5000F9488969990AA92BB9F55AD44AB77A96DD
:102C60006A711A500A333A122AFDDBDCCBBFFB9E95
:102C7000EB799B588B3BBB1AABA66C877CE44CC5AD
:102C80005C222C033C600C411CAEED8FFDECCDCDE5
:102C9000DD2AAD0BBD688D499D977EB66ED55EF47D
:102CA0004E133E322E511E700E9FFFBEEFDDDFFC35
:102CB000CF1BBF3AAF599F788F8891A981CAB1EBDA
:102CC000A10CD12DC14EF16FE18010A100C230E303
:102CD000200450254046706760B9839893FBA3DABF
:102CE000B33DC31CD37FE35EF3B1029012F322D253
:102CF000323542145277625672EAB5CBA5A895894F
:102D0000856EF54FE52CD50DC5E234C324A01481A2
:102D1000046674476424540544DBA7FAB79987B85E
:102D2000975FE77EF71DC73CD7D326F2369106B0F2
:102D30001657667676154634564CD96DC90EF92F5E
:102D4000E9C899E9898AB9ABA94458654806782742
:102D500068C018E1088238A3287DCB5CDB3FEB1EFE
:102D6000FBF98BD89BBBAB9ABB754A545A376A1692
:102D70007AF10AD01AB32A923A2EFD0FED6CDD4D8E
:102D8000CDAABD8BADE89DC98D267C076C645C45E2
:102D90004CA23C832CE01CC10C1FEF3EFF5DCF7C9E
:102DA000DF9BAFBABFD98FF89F176E367E554E7432
:102DB0005E932EB23ED10EF01E4D3834205820596D
:102DC000205A20450043616E6E6F7420656E7465F5
:102DD00072207375626469723A20004563686F3AC5
:102DE00020004372656174696F6E206661696C656D
:102DF00064004469726563746F72792063726561FF
:102E000074656400446F6E6520736176696E672037
:102E100066696C652E0044656C6574696F6E20662A
:102E200061696C65640046696C652064656C6574F5
:102E300065640046696C652064656C657465640052
:102E400057726974696E6720746F2066696C653AA1
:102E500020006F70656E206661696C65642C204689
:102E6000696C653A20004572726F723A20004E6FAD
:102E700074205344207072696E74696E67002F006D
:102E80005344207072696E74696E6720627974654C
:102E900020006F70656E206661696C65642C204649
:102EA000696C653A200046696C652073656C6563E2
:102EB000746564002053697A653A200046696C6540
:102EC000206F70656E65643A20006572726F7220C3
:102ED00077726974696E6720746F2066696C65002B
:102EE0004572726F723A200053442063617264200D
:102EF0006F6B004563686F3A2000534420696E6928
:102F000074206661696C004572726F723A20004DE0
:102F1000494E54454D502074726967676572656407
:102F2000004D494E54454D50204552524F5200627B
:102F30006564002C2073797374656D2073746F70F1
:102F400070656421204865617465725F49443A2068
:102F5000004572726F723A20004D415854454D50F1
:102F600020747269676765726564004D4158544505
:102F70004D50204552524F5200204B643A200020C1
:102F80004B693A20004B703A20004563686F3A2045
:102F900000504944204175746F74756E65206669F0
:102FA0006E697368656421205075742074686520AB
:102FB0006C617374204B702C204B6920616E64200F
:102FC0004B6420636F6E7374616E74732066726FEE
:102FD0006D2061626F766520696E746F20436F6E3D
:102FE00066696775726174696F6E2E68206F7220F2
:102FF00073656E6420636F6D6D616E64204D353056
:103000003020666F72207361766520696E204545B9
:1030100050524F4D20746865206E65772076616C44
:10302000756521004563686F3A200050494420418E
:1030300075746F74756E65206661696C65642120B6
:1030400074696D656F7574004572726F723A200015
:10305000504944204175746F74756E6520666169CE
:103060006C6564212054656D70657261747572655C
:1030700020746F6F2068696768004572726F723ADA
:103080002000204B643A2000204B693A20004B700E
:103090003A200020436C61737369632050494420D7
:1030A000002054753A2000204B753A2000206D61B5
:1030B000783A2000206D696E3A200020643A2000A2
:1030C00020626961733A2000204379636C65733A2A
:1030D00020002054656D703A2000486F74656E645E
:1030E0003A20004563686F3A2000504944204175FA
:1030F000746F74756E6520737461727400456368D3
:103100006F3A2000504944204175746F74756E65A4
:10311000206661696C656421204261642065787471
:103120007275646572206E756D62657200457272AB
:103130006F723A200010001900F03F190000000AD9
:103140000B02090C0D0E080703040100000000002B
:10315000000000000000000000000000000000006F
:10316000000000000000000000121110000000002C
:10317000000000000000000000000000000000004F
:1031800000000001021020200808102040102040FC
:10319000800201020108040201010204081020401B
:1031A0008080402010080402018004020180402039
:1031B0001008040201080402010102040810204062
:1031C0008001020408102040800505050507050858
:1031D000080808020202020A0A080804040404019A
:1031E00001010101010101030303030303030304BC
:1031F0000707070C0C0C0C0C0C0C0C02020202064C
:10320000060606060606060B0B0B0B0B0B0B0B003C
:103210000020002300260029002C002F003200008F
:103220000100000301060109010000220025002819
:10323000002B002E003100340002010000050108BF
:10324000010B0100002100240027002A002D00307E
:1032500000330001010000040107010A014E414E44
:10326000494E495459494E46CDCCCC3D0AD7233C12
:1032700017B7D13877CC2B329595E6241FB14F0A7A
:10328000000020410000C84200401C4620BCBE4C4B
:10329000CA1B0E5AAEC59D74B9509687F2D311243D
:1032A0001FBECFEFD1E2DEBFCDBF00E00CBF14E008
:1032B000A0E0B2E0EAE5F2EC01E00BBF02C007904B
:1032C0000D92A836B107D9F720E2A8E6B4E001C014
:1032D0001D92AF31B207E1F712E3CEE9D2E300E08D
:1032E00006C022970109FE010BBF0E94E9D9C83927
:1032F000D10780E00807A9F70E94C1D40C942BE104
:103300000C9400002F923F924F925F926F927F92A7
:103310008F929F92AF92BF92CF92DF92EF92FF92E5
:103320001F93CF93DF93CDB7DEB7C656D1090FB643
:10333000F894DEBF0FBECDBF8CE1E4EAF2E0DE011F
:10334000D99601900D928A95E1F78CE1E0ECF2E0DC
:10335000DE015D9601900D928A95E1F78CE1ECED2E
:10336000F2E0DE01119601900D928A95E1F720912D
:103370001B1B30911C1B40911D1B50911E1B40902C
:103380000B1B50900C1B60900D1B70900E1B8090BF
:10339000A5049090A604A090A704B090A804C090A3
:1033A000A904D090AA04E090AB04F090AC04809102
:1033B000AD049091AE04A091AF04B091B0046D96AD
:1033C0008CAF9DAFAEAFBFAF6D971E0199E3290ED5
:1033D000311CA7E3BBE16F96BFAFAEAF6F97FE01A5
:1033E0007D96A396FFAFEEAFA39787E49BE1679628
:1033F0009FAF8EAF6797DE011196A196BFAFAEAFBC
:10340000A197E7E2FBE16996FFAFEEAF699710E0A5
:10341000F10181919191A191B1911F016F96EEAD52
:10342000FFAD6F9781939193A193B1936F96FFAF87
:10343000EEAF6F97A396EEADFFADA39781919191FB
:10344000A191B191A396FFAFEEAFA3976796EEADB2
:10345000FFAD679781939193A193B1936796FFAF67
:10346000EEAF6797A196AEADBFADA1976D917D917F
:103470008D919D91A196BFAFAEAFA197A4962FAFAE
:10348000A497A5963FAFA597A6964FAFA697A796E8
:103490005FAFA7970E941CD66996EEADFFAD699706
:1034A00061937193819391936996FFAFEEAF6997A2
:1034B000A4962FADA497A5963FADA597A6964FAD20
:1034C000A697A7965FADA797111115C06D961CAE74
:1034D0001DAE1EAE1FAE6D97C12CD12C76014601DC
:1034E0005701412C512C88E4682E82E4782E20E08C
:1034F00030E44CE156E41F5F143009F089CF20938B
:103500001B1B30931C1B40931D1B50931E1B409292
:103510000B1B50920C1B60920D1B70920E1B809225
:10352000A5049092A604A092A704B092A804C09209
:10353000A904D092AA04E092AB04F092AC046D9678
:103540008CAD9DADAEADBFAD6D978093AD04909346
:10355000AE04A093AF04B093B0040E94069780E03D
:1035600090E0AAE7B4E480931F1B9093201BA093E4
:10357000211BB093221B8093171B9093181BA093C1
:10358000191BB0931A1B1092231B1092241B10922C
:10359000251B1092261B80E29EE4A0E0B0E0809301
:1035A000571B9093581BA093591BB0935A1B109212
:1035B000071B1092081B1092091B10920A1B80E037
:1035C00090E0A8EDB1E48093131B9093141BA0939B
:1035D000151BB093161B8DEC9CECACECBEE38093FA
:1035E0000F1B9093101BA093111BB093121B1092F2
:1035F000B9041092BA041092BB041092BC04109249
:10360000B5041092B6041092B7041092B804109248
:10361000B1041092B2041092B3041092B404109248
:103620006D0410926E0410926F04109270048EEB71
:1036300090E09093770C8093760C2CE330E03093FD
:10364000750C2093740C8FEF90E09093730C809323
:10365000720C40EF50E05093710C4093700C44E6B4
:1036600050E050936F0C40936E0C90936D0C8093D0
:103670006C0C46EE50E050936B0C40936A0C309308
:10368000690C2093680C9093670C8093660C80E023
:1036900090E0A0E2B2E480931F1F9093201FA093BC
:1036A000211FB093221F60E070E080EE90E40E9442
:1036B000B8C960931B1F70931C1F80931D1F9093AC
:1036C0001E1F60E070E080E792E40E94C4C960932E
:1036D000171F7093181F8093191F90931A1F80E073
:1036E00090E0A8ECB2E48093131F9093141FA09372
:1036F000151FB093161F0E94B9C01092BD040E94FE
:10370000524BE9E0F6E08491882341F09091C000AB
:1037100095FFFCCF8093C6003196F5CFE7EEF5E03C
:103720008491882341F09091C00095FFFCCF809355
:10373000C6003196F5CF82EB98E0CA59DF4F0FB63D
:10374000F894DEBF0FBECDBFDF91CF911F91FF90E8
:10375000EF90DF90CF90BF90AF909F908F907F9031
:103760006F905F904F903F902F900C9472528F9279
:103770009F92AF92BF92CF92DF92EF92FF920F9300
:103780001F93CF93DF93CDB7DEB7EC970FB6F894C6
:10379000DEBF0FBECDBF182F81111EC0E2E5F2E0E3
:1037A0008491882341F09091C00095FFFCCF8093D5
:1037B000C6003196F5CFE3E4F2E08491882341F02E
:1037C0009091C00095FFFCCF8093C6003196F5CF55
:1037D00082EB98E00E947252C0907504D0907604FB
:1037E000E0907704F09078042CE3822E912CA12CA9
:1037F000B12CC701B601A50194010E9486D9CA0166
:10380000B901A50194010E9486D97F936F93C701E6
:10381000B60120E13EE040E050E00E9486D9CA01B6
:10382000B90128E130E040E050E00E9486D97F9362
:103830006F93C701B60120E831E541E050E00E94F6
:1038400086D93F932F9385E292E09F938F937E01D9
:103850008FE1E80EF11CFF92EF920E9466DE0FB638
:10386000F894DEBF0FBECDBFEEE1F2E08491882375
:1038700041F09091C00095FFFCCF8093C600319637
:10388000F5CFF7018191882339F09091C00095FF21
:10389000FCCF8093C600F6CF82EB98E00E94725274
:1038A00011111EC0E7E1F2E08491882341F090916C
:1038B000C00095FFFCCF8093C6003196F5CFE5E0C0
:1038C000F2E08491882341F09091C00095FFFCCFF5
:1038D0008093C6003196F5CF82EB98E00E94725239
:1038E00060917104709172048091730490917404DA
:1038F0000E9417D66B017C012AE030E040E050E0E6
:103900000E94A8D97F936F93CA01B90124E630E0E1
:1039100040E050E00E94A8D97F936F9398EE892EE3
:1039200093E0992EA12CB12CC701B601A5019401F9
:103930000E94A8D9CA01B901A50194010E94A8D981
:103940007F936F93C701B60120E432E44FE050E06B
:103950000E94A8D93F932F938CEE91E09F938F9371
:103960008E010F5F1F4F1F930F930E9466DE0FB6ED
:10397000F894DEBF0FBECDBFE5EEF1E08491882361
:1039800041F09091C00095FFFCCF8093C600319626
:10399000F5CFF8018191882339F09091C00095FF0F
:1039A000FCCF8093C600F6CF82EB98E00E94725263
:1039B000EC960FB6F894DEBF0FBECDBFDF91CF916E
:1039C0001F910F91FF90EF90DF90CF90BF90AF903D
:1039D0009F908F900895CF93C82F81111EC0EEED58
:1039E000F5E08491882341F09091C00095FFFCCFD1
:1039F0008093C6003196F5CFEEECF5E084918823F4
:103A000041F09091C00095FFFCCF8093C6003196A5
:103A1000F5CF82EB98E00E947252E5ECF5E08491DC
:103A2000882341F09091C00095FFFCCF8093C600A1
:103A30003196F5CFEDEBF5E08491882341F090913C
:103A4000C00095FFFCCF8093C6003196F5CF409122
:103A5000371B5091381B6091391B70913A1B22E043
:103A600030E082EB98E00E945153EAEBF5E084915C
:103A7000882341F09091C00095FFFCCF8093C60051
:103A80003196F5CF40913B1B50913C1B60913D1B03
:103A900070913E1B22E030E082EB98E00E9451538F
:103AA000E7EBF5E08491882341F09091C00095FF09
:103AB000FCCF8093C6003196F5CF40913F1B5091CB
:103AC000401B6091411B7091421B22E030E082EB71
:103AD00098E00E945153E4EBF5E08491882341F093
:103AE0009091C00095FFFCCF8093C6003196F5CF32
:103AF0004091431B5091441B6091451B7091461BA4
:103B000022E030E082EB98E00E94515382EB98E093
:103B10000E947252C1111EC0EBEAF5E08491882325
:103B200041F09091C00095FFFCCF8093C600319684
:103B3000F5CFE1E9F5E08491882341F09091C00050
:103B400095FFFCCF8093C6003196F5CF82EB98E0CD
:103B50000E947252E8E8F5E08491882341F0909148
:103B6000C00095FFFCCF8093C6003196F5CFEFE7FC
:103B7000F5E08491882341F09091C00095FFFCCF3F
:103B80008093C6003196F5CF4091471B5091481B5A
:103B90006091491B70914A1B22E030E082EB98E073
:103BA0000E945153ECE7F5E08491882341F0909115
:103BB000C00095FFFCCF8093C6003196F5CF4091B1
:103BC0004B1B50914C1B60914D1B70914E1B22E082
:103BD00030E082EB98E00E945153E9E7F5E08491F0
:103BE000882341F09091C00095FFFCCF8093C600E0
:103BF0003196F5CF40914F1B5091501B6091511B56
:103C00007091521B22E030E082EB98E00E94515309
:103C1000E6E7F5E08491882341F09091C00095FF9C
:103C2000FCCF8093C6003196F5CF4091531B509145
:103C3000541B6091551B7091561B22E030E082EBC3
:103C400098E00E94515382EB98E00E947252C11199
:103C50001EC0EDE6F5E08491882341F09091C0000C
:103C600095FFFCCF8093C6003196F5CFEFE4F5E0E9
:103C70008491882341F09091C00095FFFCCF809300
:103C8000C6003196F5CF82EB98E00E947252E6E4CE
:103C9000F5E08491882341F09091C00095FFFCCF1E
:103CA0008093C6003196F5CFEDE3F5E0849188234B
:103CB00041F09091C00095FFFCCF8093C6003196F3
:103CC000F5CF4091271B5091281B6091291B7091C3
:103CD0002A1B2AE030E082EB98E00E94B252EAE32D
:103CE000F5E08491882341F09091C00095FFFCCFCE
:103CF0008093C6003196F5CF40912B1B50912C1B21
:103D000060912D1B70912E1B2AE030E082EB98E031
:103D10000E94B252E7E3F5E08491882341F090914C
:103D2000C00095FFFCCF8093C6003196F5CF40913F
:103D30002F1B5091301B6091311B7091321B2AE078
:103D400030E082EB98E00E94B252E4E3F5E0849127
:103D5000882341F09091C00095FFFCCF8093C6006E
:103D60003196F5CF4091331B5091341B6091351B38
:103D70007091361B2AE030E082EB98E00E94B2524C
:103D800082EB98E00E94725282EB98E00E9472529D
:103D9000C1111EC0EBE2F5E08491882341F09091BF
:103DA000C00095FFFCCF8093C6003196F5CFE6EFBB
:103DB000F4E08491882341F09091C00095FFFCCFFE
:103DC0008093C6003196F5CF82EB98E00E94725244
:103DD000EDEEF4E08491882341F09091C00095FFCE
:103DE000FCCF8093C6003196F5CFE4EEF4E08491E9
:103DF000882341F09091C00095FFFCCF8093C600CE
:103E00003196F5CF40911F1B5091201B6091211BD3
:103E10007091221B22E030E082EB98E00E94515327
:103E2000E1EEF4E08491882341F09091C00095FF89
:103E3000FCCF8093C6003196F5CF4091171B50916F
:103E4000181B6091191B70911A1B22E030E082EB65
:103E500098E00E94515382EB98E00E947252E8ED84
:103E6000F4E08491882341F09091C00095FFFCCF4D
:103E70008093C6003196F5CFEFECF4E0849188236F
:103E800041F09091C00095FFFCCF8093C600319621
:103E9000F5CF4AE050E060E070E082EB98E00E94ED
:103EA0008652ECECF4E08491882341F09091C000BC
:103EB00095FFFCCF8093C6003196F5CF40911B1B38
:103EC00050911C1B60911D1B70911E1B22E030E065
:103ED00082EB98E00E94515382EB98E00E9472526C
:103EE000C1111EC0E3ECF4E08491882341F090916D
:103EF000C00095FFFCCF8093C6003196F5CFE0E17E
:103F0000F4E08491882341F09091C00095FFFCCFAC
:103F10008093C6003196F5CF82EB98E00E947252F2
:103F2000E7E0F4E08491882341F09091C00095FF90
:103F3000FCCF8093C6003196F5CFEEEFF3E084918D
:103F4000882341F09091C00095FFFCCF8093C6007C
:103F50003196F5CF4091231B5091241B6091251B76
:103F60007091261B22E030E082EB98E00E945153D2
:103F7000EBEFF3E08491882341F09091C00095FF2E
:103F8000FCCF8093C6003196F5CF4091071B50912E
:103F9000081B6091091B70910A1B22E030E082EB44
:103FA00098E00E945153E8EFF3E08491882341F0B8
:103FB0009091C00095FFFCCF8093C6003196F5CF5D
:103FC0004091571B5091581B6091591B70915A1B7F
:103FD0002AE030E082EB98E00E94B252E5EFF3E095
:103FE0008491882341F09091C00095FFFCCF80938D
:103FF000C6003196F5CF4091131B5091141B609170
:10400000151B7091161B22E030E082EB98E00E94B5
:104010005153E2EFF3E08491882341F09091C00086
:1040200095FFFCCF8093C6003196F5CF40910F1BD2
:104030005091101B6091111B7091121B22E030E017
:1040400082EB98E00E945153EFEEF3E084918823D5
:1040500041F09091C00095FFFCCF8093C60031964F
:10406000F5CF40910B1B50910C1B60910D1B709173
:104070000E1B22E030E082EB98E00E94515382EB6D
:1040800098E00E947252C1111EC0E6EEF3E08491E6
:10409000882341F09091C00095FFFCCF8093C6002B
:1040A0003196F5CFE4EDF3E08491882341F09091CF
:1040B000C00095FFFCCF8093C6003196F5CF82EB10
:1040C00098E00E947252EBECF3E08491882341F077
:1040D0009091C00095FFFCCF8093C6003196F5CF3C
:1040E000E2ECF3E08491882341F09091C00095FFC9
:1040F000FCCF8093C6003196F5CF4091B10450912A
:10410000B2046091B3047091B40422E030E082EB19
:1041100098E00E945153EFEBF3E08491882341F043
:104120009091C00095FFFCCF8093C6003196F5CFEB
:104130004091B5045091B6046091B7047091B804F1
:1041400022E030E082EB98E00E945153ECEBF3E088
:104150008491882341F09091C00095FFFCCF80931B
:10416000C6003196F5CF4091B9045091BA046091E0
:10417000BB047091BC0422E030E082EB98E00E9426
:10418000515382EB98E00E947252C1111EC0E3EBC2
:10419000F3E08491882341F09091C00095FFFCCF1B
:1041A0008093C6003196F5CFEFE9F3E08491882340
:1041B00041F09091C00095FFFCCF8093C6003196EE
:1041C000F5CF82EB98E00E947252E6E9F3E0849129
:1041D000882341F09091C00095FFFCCF8093C600EA
:1041E0003196F5CFEDE8F3E08491882341F090918A
:1041F000C00095FFFCCF8093C6003196F5CF4AE012
:1042000050E060E070E082EB98E00E948652EAE8BD
:10421000F3E08491882341F09091C00095FFFCCF9A
:104220008093C6003196F5CF4091A5045091A60425
:104230006091A7047091A80422E030E082EB98E03E
:104240000E945153E7E8F3E08491882341F0909174
:10425000C00095FFFCCF8093C6003196F5CF40910A
:10426000A9045091AA046091AB047091AC0422E0BF
:1042700030E082EB98E00E945153E4E8F3E084914F
:10428000882341F09091C00095FFFCCF8093C60039
:104290003196F5CF4091AD045091AE046091AF04DA
:1042A0007091B00422E030E082EB98E00E9451531C
:1042B00082EB98E00E947252C1111EC0EBE7F3E05E
:1042C0008491882341F09091C00095FFFCCF8093AA
:1042D000C6003196F5CFEFE5F3E08491882341F0F5
:1042E0009091C00095FFFCCF8093C6003196F5CF2A
:1042F00082EB98E00E947252E6E5F3E08491882315
:1043000041F09091C00095FFFCCF8093C60031969C
:10431000F5CFEAE4F3E08491882341F09091C00066
:1043200095FFFCCF8093C6003196F5CF6091760C57
:104330007091770C4AE050E082EB98E00E94865240
:10434000E7E4F3E08491882341F09091C00095FF69
:10435000FCCF8093C6003196F5CF6091740C7091BC
:10436000750C4AE050E082EB98E00E948652E4E44B
:10437000F3E08491882341F09091C00095FFFCCF39
:104380008093C6003196F5CF6091720C7091730CDA
:104390004AE050E082EB98E00E948652E4E3F3E0CA
:1043A0008491882341F09091C00095FFFCCF8093C9
:1043B000C6003196F5CF82EB98E00E947252EBE294
:1043C000F3E08491882341F09091C00095FFFCCFE9
:1043D0008093C6003196F5CFEFE1F3E08491882316
:1043E00041F09091C00095FFFCCF8093C6003196BC
:1043F000F5CF6091700C7091710C4AE050E082EB47
:1044000098E00E948652ECE1F3E08491882341F029
:104410009091C00095FFFCCF8093C6003196F5CFF8
:1044200060916E0C70916F0C4AE050E082EB98E066
:104430000E948652E9E1F3E08491882341F0909153
:10444000C00095FFFCCF8093C6003196F5CF6091F8
:104450006C0C70916D0C4AE050E082EB98E00E9489
:104460008652E9E0F3E08491882341F09091C00006
:1044700095FFFCCF8093C6003196F5CF82EB98E094
:104480000E947252E0E0F3E08491882341F0909121
:10449000C00095FFFCCF8093C6003196F5CFE4EFC6
:1044A000F2E08491882341F09091C00095FFFCCF09
:1044B0008093C6003196F5CF60916A0C70916B0CB9
:1044C0004AE050E082EB98E00E948652E1EFF2E091
:1044D0008491882341F09091C00095FFFCCF809398
:1044E000C6003196F5CF6091680C7091690C4AE076
:1044F00050E082EB98E00E948652EEEEF2E084916A
:10450000882341F09091C00095FFFCCF8093C600B6
:104510003196F5CF6091660C7091670C4AE050E0DF
:1045200082EB98E00E948652EEEDF2E084918823BF
:1045300041F09091C00095FFFCCF8093C60031966A
:10454000F5CF82EB98E00E947252C1111EC0E5EDDA
:10455000F2E08491882341F09091C00095FFFCCF58
:104560008093C6003196F5CFE7ECF2E08491882382
:1045700041F09091C00095FFFCCF8093C60031962A
:10458000F5CF82EB98E00E947252EEEBF2E084915C
:10459000882341F09091C00095FFFCCF8093C60026
:1045A0003196F5CFE5EBF2E08491882341F09091CC
:1045B000C00095FFFCCF8093C6003196F5CF40E058
:1045C00050E060E082EB98E00E94BD52E2EBF2E046
:1045D0008491882341F09091C00095FFFCCF809397
:1045E000C6003196F5CF40911F1F5091201F60915A
:1045F000211F7091221F22E030E082EB98E00E94A0
:104600005153EFEAF2E08491882341F09091C00089
:1046100095FFFCCF8093C6003196F5CF60911B1FAC
:1046200070911C1F80911D1F90911E1F0E94BEC97A
:10463000AB01BC0122E030E082EB98E00E945153D4
:10464000ECEAF2E08491882341F09091C00095FF5C
:10465000FCCF8093C6003196F5CF6091171F709103
:10466000181F8091191F90911A1F0E94CAC9AB018F
:10467000BC0122E030E082EB98E00E94515382EBD3
:1046800098E00E9472528091BD04882309F449C0C9
:10469000C1111EC0E3EAF2E08491882341F09091B9
:1046A000C00095FFFCCF8093C6003196F5CFE0E9BE
:1046B000F2E08491882341F09091C00095FFFCCFF7
:1046C0008093C6003196F5CF82EB98E00E9472523B
:1046D000E7E8F2E08491882341F09091C00095FFD3
:1046E000FCCF8093C6003196F5CFEEE7F2E08491DF
:1046F000882341F09091C00095FFFCCF8093C600C5
:104700003196F5CF40912302509124026091250209
:104710007091260222E030E082EB98E00E94515333
:104720001CC0C1111EC0E5E7F2E08491882341F06E
:104730009091C00095FFFCCF8093C6003196F5CFD5
:10474000E9E5F2E08491882341F09091C00095FF63
:10475000FCCF8093C6003196F5CF82EB98E00E94A3
:1047600072528C2FCF9103C8109275041092760468
:1047700010927704109278041092710410927204CF
:104780001092730410927404E1EEF1E08491882396
:1047900041F09091C00095FFFCCF8093C600319608
:1047A000F5CFECEBF1E08491882341F09091C000CB
:1047B00095FFFCCF8093C6003196F5CF82EB98E051
:1047C0000C947252FC0165917591859194910895B4
:1047D0000E94FACF609386047093870480938804C4
:1047E000909389040895CF93DF93FC0120812B33AC
:1047F00009F464C020914406309145062430310507
:104800000CF05CC0209146063091470640E6429F7E
:10481000E001439FD00D1124CC53DB4FBC01CE01EE
:104820000E9445DEE5EDFEE08491882341F0909101
:10483000C00095FFFCCF8093C6003196F5CFE8EC21
:10484000FEE08491882371F09091C00095FFFCCF29
:104850008093C6003196F5CF9091C00095FFFCCFB4
:104860008093C60089918111F7CFE6ECFEE0849138
:10487000882341F09091C00095FFFCCF8093C60043
:104880003196F5CF82EB98E00E94725280914606F5
:1048900090914706019664E070E00E9473D990936E
:1048A00047068093460680914406909145060196FE
:1048B000909345068093440681E001C080E0DF913B
:1048C000CF910895DF92EF92FF920F931F93CF93B2
:1048D000DF93CDB7DEB76E970FB6F894DEBF0FBE8D
:1048E000CDBF60918A0470918B0461157105A1F0B0
:1048F0004DE150E08E010F5F1F4FC8010E94E1DDC6
:104900001E8EF8017F01E01AF10AD190DD2031F00E
:104910008AE0D812F7CF02C080E01DC0F801EE0D8A
:10492000FF1D1082C8015FDF8823A1F0DD2071F038
:104930008FEFE81AF80A80918A0490918B048E0D0B
:104940009F1D90938B0480938A0404C010928B0463
:1049500010928A0481E06E960FB6F894DEBF0FBE07
:10496000CDBFDF91CF911F910F91FF90EF90DF901E
:10497000089590938B0480938A04A4CF40E052EC76
:1049800061E070E082EB98E00E946A5161E070E0C3
:1049900080E090E00E9429D0E0ECFEE08491882342
:1049A00041F09091C00095FFFCCF8093C6003196F6
:1049B000F5CF82EB98E00E9472520E94BD50E3EB6B
:1049C000FEE08491882341F09091C00095FFFCCFD8
:1049D0008093C6003196F5CF82EB98E00E94725228
:1049E000ECE6FEE08491882341F09091C00095FFB1
:1049F000FCCF8093C6003196F5CF82EB98E00E9401
:104A00007252E6E5FEE08491882341F09091C00067
:104A100095FFFCCF8093C6003196F5CF82EB98E0EE
:104A20000E947252E8E4FEE08491882341F0909164
:104A3000C00095FFFCCF8093C6003196F5CF0E9451
:104A40001C514AE050E0BC0182EB98E00E94865283
:104A5000E2E3FEE08491882341F09091C00095FF4D
:104A6000FCCF8093C6003196F5CF4AE050E060E578
:104A70007EE082EB98E00E94865282EB98E00E94F2
:104A800072521092690410926A0410926B04109290
:104A90006C046ADE0E94821980E00E94EB1C0E9476
:104AA000786C0E94EFC20E94508B0E9425A10C944A
:104AB000A1550F931F93CF93DF9300918C04109116
:104AC0008D0465E470E0C8010E9431DEEC01C8018C
:104AD0000196209761F0188260E070E00E9420DB70
:104AE00025E42883DF91CF911F910F91089560E015
:104AF00070E0DF91CF911F910F910C9420DB80919A
:104B00008C0490918D044AE050E060E070E00196E2
:104B10000C9488DC80918C0490918D044AE050E0E4
:104B200060E070E001960E9488DCCB010895682F58
:104B3000772767FD709580914A0690914B060E94F9
:104B400031DE90938D0480938C0421E0892B09F44D
:104B500020E0822F08954F925F926F927F92AF92E2
:104B6000CF92DF92EF92FF920F931F9328013901AA
:104B7000FC012191CF01222339F03091C00035FF93
:104B8000FCCF2093C600F4CFE4EBFCE084918823B3
:104B900041F09091C00095FFFCCF8093C600319604
:104BA000F5CF22E030E082EB98E00E945153E1EB38
:104BB000FCE08491882341F09091C00095FFFCCFE8
:104BC0008093C6003196F5CF22E030E0B301A20118
:104BD00082EB98E00E945153EEEAFCE08491882336
:104BE00041F09091C00095FFFCCF8093C6003196B4
:104BF000F5CF22E030E0B701A60182EB98E00E94F9
:104C00005153ECEAFCE08491882341F09091C0007C
:104C100095FFFCCF8093C6003196F5CFAA2079F09E
:104C200082EB98E01F910F91FF90EF90DF90CF9073
:104C3000AF907F906F905F904F900C9472521F9145
:104C40000F91FF90EF90DF90CF90AF907F906F909B
:104C50005F904F900895AF92CF92DF92EF92FF92C4
:104C60000F931F93FB01A42EC084D184E284F384AC
:104C70000481158126813781408151816281738150
:104C80006ADF1F910F91FF90EF90DF90CF90AF9070
:104C900008950F931F93CF93DF9300D000D0CDB72B
:104CA000DEB78C0186E0E8EFF2E0DE0111960190BC
:104CB0000D928A95E1F7F801EE0FFF1F81E090E079
:104CC0008C0F9D1FE80FF91F608171811616170662
:104CD00004F1E2E9FBE08491882341F09091C00067
:104CE00095FFFCCF8093C6003196F5CFEBE5FBE056
:104CF0008491882341F09091C00095FFFCCF809370
:104D0000C6003196F5CF82EB98E00E9472526AE0BD
:104D100070E0000F111F000F111F035D1D4F88274A
:104D200077FD8095982F0E944AD69B01AC01F8012F
:104D300060817181828193810E94AFD560933D0231
:104D400070933E0280933F029093400226960FB6E6
:104D5000F894DEBF0FBECDBFDF91CF911F910F91B1
:104D60000895AF92CF92EF92FF920F931F9320E09E
:104D700030E040E752E460913D0270913E02809144
:104D80003F02909140020E94AFD5A0909604C0903F
:104D900098047B018C0125E936E041E956E06DE895
:104DA00076E089E896E00E94A08B1F910F91FF901A
:104DB000EF90CF90AF9008954F925F926F927F9255
:104DC000AF92CF92DF92EF92FF920F931F93CF9308
:104DD000DF93CDB7DEB72C970FB6F894DEBF0FBECA
:104DE000CDBF2B013C0129833A834B835C83ED8249
:104DF000FE820F83188780913D0290913E02A09120
:104E00003F02B091400289879A87AB87BC87809127
:104E1000350290913602A0913702B091380280930A
:104E20003D0290933E02A0933F02B09340028091D6
:104E3000410281FF1CC0E6EDFBE08491882341F034
:104E40009091C00095FFFCCF8093C6003196F5CFBE
:104E5000AA24A394CD80DE80EF80F88409811A8192
:104E60002B813C81B301A2018EEF92E074DE8D8133
:104E70009E81AF81B8858093910690939206A0930E
:104E80009306B09394066DDF0E94AEA160910B0271
:104E900070910C02882777FD8095982F0E944AD642
:104EA00060933D0270933E0280933F0290934002D4
:104EB0004092890650928A0660928B0670928C0608
:104EC00089819A81AB81BC8180938D0690938E06F7
:104ED000A0938F06B093900644DF0E94AEA189850F
:104EE0009A85AB85BC8580933D0290933E02A0934A
:104EF0003F02B09340022C960FB6F894DEBF0FBE6F
:104F0000CDBFDF91CF911F910F91FF90EF90DF9078
:104F1000CF90AF907F906F905F904F900895AF9239
:104F2000CF92EF92FF920F931F9320E030E040E783
:104F300052E40E94AFD5A0909604C09098047B01E3
:104F40008C0125E836E041E856E06DE776E089E738
:104F500096E00E94A08B1F910F91FF90EF90CF9051
:104F6000AF90089560913D0270913E0280913F02A2
:104F700090914002D4CF25E936E041E956E06DE852
:104F800076E089E896E00C9410964F925F926F92CB
:104F90007F928F929F92AF92BF92CF92DF92EF92C9
:104FA000FF920F931F93CF93DF938C018091410267
:104FB00081FF34C0EFECFBE08491882341F09091B5
:104FC000C00095FFFCCF8093C6003196F5CFE1EC91
:104FD000FBE08491882341F09091C00095FFFCCFC5
:104FE0008093C6003196F5CFA80160E070E02AE01A
:104FF00030E082EB98E00E94B252EFEBFBE084914C
:10500000882341F09091C00095FFFCCF8093C600AB
:105010003196F5CF82EB98E00E9472520330110571
:1050200008F05AC1F801E452F14FF490E801CC0FB6
:10503000DD1FCC0FDD1F9E012757394F6901F90194
:10504000108211821282138296DFCE018950914F15
:10505000B9DB2B013C016F2D772767FD7095872FFA
:10506000972F0E944AD64B015C019E012758394F69
:10507000790120E030E040EC5FE3C301B2010E941F
:105080007DD8A50194010E947DD8F70160837183CA
:1050900082839383FE01E35DFD4F80819181A28134
:1050A000B38180933D0290933E02A0933F02B09360
:1050B000400258DF0E94AEA1F601108211821282D6
:1050C000138259DF80E00E940D989E012152314FDA
:1050D0006901C90177DB9058A50194010E947DD830
:1050E000F70160837183828393833CDF0E94AEA1CA
:1050F00081E00E940D98C801CCDDC60163DB9B01F5
:10510000AC010E94CFD4A50194010E947DD8F70183
:10511000608371838283938325DF0E94AEA1809197
:10512000410281FF13C0E8EBFBE08491882341F04A
:105130009091C00095FFFCCF8093C6003196F5CFCB
:1051400041E069E876E082E193E085DDCE018D5FA4
:10515000904F38DB9E012757394F6901FE01EF540C
:10516000FB4F7F0120813181428153810E94CFD446
:10517000F6016083718382839383CE018551914FC1
:1051800021DB9E0127563B4F6901F70120813181C8
:10519000428153810E94CFD4F60160837183828360
:1051A0009383CE01815F904F0DDB9E012D5E3D4FBD
:1051B0006901F70120813181428153810E94CFD45E
:1051C000F60160837183828393838091410281FF22
:1051D00043C0E4E5FBE08491882341F09091C00056
:1051E00095FFFCCF8093C6003196F5CFEFE3FBE04F
:1051F0008491882341F09091C00095FFFCCF80936B
:10520000C6003196F5CFA80160E070E02AE030E0FA
:1052100082EB98E00E94B252E7E2FBE0849188239F
:1052200041F09091C00095FFFCCF8093C60031966D
:10523000F5CFFE01EF54FB4F4081518162817381B4
:1052400022E030E082EB98E00E94515341E069E8AF
:1052500076E087E393E0FFDC8EDE8091410281FF00
:1052600013C0E1EBFBE08491882341F09091C000F2
:1052700095FFFCCF8093C6003196F5CF41E069E8F9
:1052800076E08CE493E0E7DCFE01E758F94FC7577E
:10529000D94F88819981AA81BB8180839183A28320
:1052A000B38310923D0210923E0210923F02109280
:1052B00040020E944E9781E090E0002E01C0880FCE
:1052C0000A94EAF790917706982B9093770690913D
:1052D0007806982B909378068091410281FF44C014
:1052E000EAEAFBE08491882341F09091C00095FFA9
:1052F000FCCF8093C6003196F5CFECE9FBE08491BA
:10530000882341F09091C00095FFFCCF8093C600A8
:105310003196F5CFA80160E070E02AE030E082EB42
:1053200098E00E94B252EAE9FBE08491882341F0C0
:105330009091C00095FFFCCF8093C6003196F5CFC9
:1053400082EB98E0DF91CF911F910F91FF90EF904A
:10535000DF90CF90BF90AF909F908F907F906F9095
:105360005F904F900C947252DF91CF911F910F91EB
:10537000FF90EF90DF90CF90BF90AF909F908F9075
:105380007F906F905F904F90089580E1E9E7F6E09D
:10539000A9E8B6E001900D928A95E1F70895E9EA4F
:1053A000FCE08491882341F09091C00095FFFCCFF0
:1053B0008093C6003196F5CF4091511F5091521FF6
:1053C0006091531F7091541F21E030E082EB98E010
:1053D0000E945153E6EAFCE08491882341F09091C9
:1053E000C00095FFFCCF8093C6003196F5CF609149
:1053F0006B1F70916C1F882777FD8095982F0E94F6
:105400004AD6AB01BC0121E030E082EB98E00E947B
:105410005153E2EAFCE08491882341F09091C0006E
:1054200095FFFCCF8093C6003196F5CF809179042B
:1054300090E00E94D0C04AE050E0BC0182EB98E0CE
:105440000C9486528F929F92AF92BF92CF92DF922E
:10545000EF92FF920F931F93CF93DF9353EFC52EDD
:1054600053E0D52E69E7E62E66E0F62E09E816E051
:10547000C0E0D0E0F60181916F0159DB882359F13A
:1054800018DBFE01E054FB4F2081211104C0209164
:105490009204222331F0F80120813181428153812D
:1054A00012C020919804FE01E20FF11DEE0FFF1FC4
:1054B000EE0FFF1FEB55FB4F80809180A280B380E1
:1054C000A501940150580E94CFD4F70160837183E5
:1054D000828393830AC0F80180819181A281B38184
:1054E000F70180839183A283B3832196F4E0EF0ECA
:1054F000F11C0C5F1F4FC230D10509F0BBCF85E412
:1055000016DB882301F1D5DA2091C304211104C0F0
:1055100020919204222349F020919506309196061D
:10552000409197065091980603C020E030E0A90111
:105530000E94CFD460938506709386068093870679
:105540009093880610C08091950690919606A09140
:105550009706B09198068093850690938606A0934F
:105560008706B093880686E4E2DA882391F0A1DA10
:105570006B017C0120E030E0A9010E94ABD7181636
:1055800044F4C0923D02D0923E02E0923F02F0927B
:10559000400280E5CCDA882381F18BDA6B017C0153
:1055A000E0919704F0E0EE0FFF1FE95DFD4F608191
:1055B0007181882777FD8095982F0E944AD69B019C
:1055C000AC01C701B6010E947DD820E030E048EC74
:1055D00052E40E94AFD520919506309196064091F5
:1055E0009706509198060E94CFD4609385067093D9
:1055F00086068093870690938806209195063091C1
:105600009606409197065091980660918506709194
:10561000860680918706909188060E94CED49B01D1
:10562000AC01609171047091720480917304909147
:1056300074040E94CFD460937104709372048093B9
:10564000730490937404DF91CF911F910F91FF9099
:10565000EF90DF90CF90BF90AF909F908F90089584
:10566000EAE9FCE08491882341F09091C00095FF25
:10567000FCCF8093C6003196F5CFE7E8FCE084913B
:10568000882341F09091C00095FFFCCF8093C60025
:105690003196F5CFE0914C06F0914D06819188232B
:1056A00039F09091C00095FFFCCF8093C600F6CFF3
:1056B00082EB98E00C947252CF93DF9383E537DA54
:1056C000882321F0F6D90E9417D602C060E070E06E
:1056D0006230710518F1EFE1FBE08491882341F01D
:1056E0009091C00095FFFCCF8093C6003196F5CF16
:1056F000E3E0FBE08491882341F09091C00095FFA6
:10570000FCCF8093C6003196F5CF4AE050E062E0CE
:1057100070E082EB98E00E948652A7C0EB01E4E0C3
:10572000CC0FDD1FEA95E1F7DE01AA5AB94F80E1FF
:10573000E9E8F6E001900D928A95E1F781E0809327
:105740007606ECEFFAE08491882341F09091C00056
:1057500095FFFCCF8093C6003196F5CFEDEEFAE0D1
:105760008491882341F09091C00095FFFCCF8093F5
:10577000C6003196F5CFEAEEFAE08491882341F035
:105780009091C00095FFFCCF8093C6003196F5CF75
:105790004AE050E082EB98E00E948652E5EEFAE0A3
:1057A0008491882341F09091C00095FFFCCF8093B5
:1057B000C6003196F5CFFE01EA5AF94F408151817A
:1057C0006281738122E030E082EB98E00E945153C5
:1057D000E1EEFAE08491882341F09091C00095FFBA
:1057E000FCCF8093C6003196F5CFFE01EA5AF94FFF
:1057F000448155816681778122E030E082EB98E038
:105800000E945153EDEDFAE08491882341F090918C
:10581000C00095FFFCCF8093C6003196F5CFFE0106
:10582000EA5AF94F408551856285738522E030E060
:1058300082EB98E00E945153E9EDFAE084918823CD
:1058400041F09091C00095FFFCCF8093C600319647
:10585000F5CFCA5AD94F4C855D856E857F8522E08C
:1058600030E082EB98E00E94515382EB98E0DF91A8
:10587000CF910C947252BF92CF92DF92EF92FF922F
:105880000F931F93CF93DF9300D01F92CDB7DEB756
:1058900085E44DD9811102C00E94AEA1F3EFCF2E55
:1058A000F3E0DF2EA9E8EA2EA6E0FA2E00E010E0F1
:1058B000B12CF60181916F013AD98823A1F0F9D872
:1058C000F701608371838283938369837A838B83F7
:1058D0009C830330110529F4CE0101960E94E196C4
:1058E00002C0BB24B3940F5F1F4FF4E0EF0EF11C16
:1058F00004301105F1F6B1103EDB0F900F900F90C0
:105900000F90DF91CF911F910F91FF90EF90DF905B
:10591000CF90BF90089580919D068823E1F010926A
:105920009D06E9E5FAE08491882341F09091C0005A
:1059300095FFFCCF8093C6003196F5CFEBE4FAE0FB
:1059400084918823A9F09091C00095FFFCCF8093AB
:10595000C6003196F5CF81E080939D06E4E4FAE03D
:105960008491811109C0E5E3FAE0849181110CC0B2
:1059700082EB98E00C9472529091C00095FFFCCF9E
:105980008093C6003196ECCF9091C00095FFFCCF7C
:105990008093C6003196E9CFECE1FAE08491882348
:1059A00041F09091C00095FFFCCF8093C6003196E6
:1059B000F5CF82EB98E00E9472528EE996E00E9449
:1059C00056BAEEE0FAE08491882341F09091C0004D
:1059D00095FFFCCF8093C6003196F5CF82EB98E01F
:1059E0000C9472520F931F93CF93DF93CDB7DEB712
:1059F0006E970FB6F894DEBF0FBECDBF0E94FACFF0
:105A000060937A0470937B0480937C0490937D046C
:105A100000917E0410917F042091800430918104D4
:105A2000601B710B820B930B28EE33E040E050E0DB
:105A30000E9486D9CA01B9012CE330E040E050E071
:105A40000E9486D97F936F933F932F938FEF99E0B6
:105A50009F938F938E010F5F1F4F1F930F930E9491
:105A600066DE0FB6F894DEBF0FBECDBFE8EFF9E0FB
:105A70008491882341F09091C00095FFFCCF8093E2
:105A8000C6003196F5CFF8018191882339F09091C5
:105A9000C00095FFFCCF8093C600F6CF82EB98E064
:105AA0000E94725260E0C8010E94F6680E94B8C06D
:105AB0006E960FB6F894DEBF0FBECDBFDF91CF91CB
:105AC0001F910F9108950F931F93CF93DF9383E559
:105AD0002ED88823A9F11ED88C0180E528D88823E8
:105AE00021F00F3F110541F138F1CDE0D0E0E1ECBC
:105AF000F3E0819191918C179D0711F183E0E33FD1
:105B0000F807B9F7C930D10529F41093950400932B
:105B1000940402C0D7FD14C061E08C2F0E94E5D12F
:105B2000602F8C2F0E941ED2B8018C2FDF91CF9155
:105B30001F910F910C94CDD00E948A25EC01D7CFF4
:105B4000DF91CF911F910F91089583E50E949725D2
:105B5000882399F00E94592520E030E04AE754E478
:105B60000E947DD80E941CD660930F027093100291
:105B70008093110290931202089588E50E94972560
:105B8000811114C089E50E94972581110FC08AE513
:105B90000E94972581110AC085E40E9497258111F2
:105BA00005C00E94AEA1129A0C942DA20E94AEA133
:105BB00088E50E949725882331F05F9A80917806C6
:105BC0008E7F8093780689E50E949725882331F09F
:105BD0008A9A809178068D7F809378068AE50E9464
:105BE0009725882369F09FB7F89480910801816018
:105BF000809308019FBF809178068B7F8093780601
:105C000085E40E949725882311F0129A089508953B
:105C100083E50E949725882319F00E948A2501C0F8
:105C200082E18093410280FF1EC0EFEBF9E0849196
:105C3000882341F09091C00095FFFCCF8093C6006F
:105C40003196F5CFECEAF9E08491882341F0909108
:105C5000C00095FFFCCF8093C6003196F5CF82EB54
:105C600098E00E9472528091410281FF1EC0E5EAD5
:105C7000F9E08491882341F09091C00095FFFCCF1A
:105C80008093C6003196F5CFE2E9F9E0849188234C
:105C900041F09091C00095FFFCCF8093C6003196F3
:105CA000F5CF82EB98E00E9472528091410283FF0F
:105CB00020C0EBE8F9E08491882341F09091C00086
:105CC00095FFFCCF8093C6003196F5CFE6E7F9E06B
:105CD0008491882341F09091C00095FFFCCF809380
:105CE000C6003196F5CF82EB98E00E9472520E9476
:105CF0006FC38091410285FF1EC0EFE6F9E08491F9
:105D0000882341F09091C00095FFFCCF8093C6009E
:105D10003196F5CFE1E6F9E08491882341F0909146
:105D2000C00095FFFCCF8093C6003196F5CF82EB83
:105D300098E00C94725208958F929F92AF92BF9206
:105D4000CF92DF92EF92FF92E5E5F9E0849188230C
:105D500041F09091C00095FFFCCF8093C600319632
:105D6000F5CF4091890650918A0660918B0670911B
:105D70008C0622E030E082EB98E00E945153E1E58E
:105D8000F9E08491882341F09091C00095FFFCCF09
:105D90008093C6003196F5CF40918D0650918E06C6
:105DA00060918F067091900622E030E082EB98E0DF
:105DB0000E945153EDE4F9E08491882341F09091E1
:105DC000C00095FFFCCF8093C6003196F5CF40917F
:105DD000910650919206609193067091940622E08C
:105DE00030E082EB98E00E945153E9E4F9E08491BD
:105DF000882341F09091C00095FFFCCF8093C600AE
:105E00003196F5CF40919506509196066091970690
:105E10007091980622E030E082EB98E00E945153A6
:105E20008FB7F89440915B1B50915C1B60915D1B98
:105E300070915E1B80905F1B9090601BA090611B17
:105E4000B090621BC090631BD090641BE090651BF8
:105E5000F090661B8FBFEFE3F9E08491882341F057
:105E60009091C00095FFFCCF8093C6003196F5CF8E
:105E70002AE030E082EB98E00E945B52EBE3F9E02D
:105E80008491882341F09091C00095FFFCCF8093CE
:105E9000C6003196F5CF2AE030E0B501A40182EBCF
:105EA00098E00E945B52E7E3F9E08491882341F097
:105EB0009091C00095FFFCCF8093C6003196F5CF3E
:105EC0002AE030E0B701A60182EB98E00E945B5225
:105ED00082EB98E0FF90EF90DF90CF90BF90AF9073
:105EE0009F908F900C947252E5E7F8E0849188239C
:105EF00041F09091C00095FFFCCF8093C600319691
:105F0000F5CFECE5F8E08491882341F09091C00052
:105F100095FFFCCF8093C6003196F5CF82EB98E0D9
:105F20000E947252E4E5F8E08491882341F0909158
:105F3000C00095FFFCCF8093C6003196F5CF659BDE
:105F400003C0EFE7F3E009C0EBE7F3E006C0909190
:105F5000C00095FFFCCF8093C60081918111F7CFDF
:105F600082EB98E00E947252ECE4F8E0849188237E
:105F700041F09091C00095FFFCCF8093C600319610
:105F8000F5CF8091030181FF03C0EFE7F3E009C083
:105F9000EBE7F3E006C09091C00095FFFCCF809343
:105FA000C60081918111F7CF82EB98E00E94725276
:105FB000E4E4F8E08491882341F09091C00095FFDB
:105FC000FCCF8093C6003196F5CF4B9B03C0EFE723
:105FD000F3E009C0EBE7F3E006C09091C00095FF45
:105FE000FCCF8093C60081918111F7CF82EB98E0BE
:105FF0000E94725282EB98E00C947252CF93DF931E
:1060000088E40E949725882359F00E9459250E9410
:1060100017D6EB011C161D062CF4E9E3F7E0C0C00F
:10602000C0E0D0E080E50E949725882369F00E94B7
:106030005925FE01EE0FFF1FEE0FFF1FE15EF04E30
:10604000608371838283938389E40E9497258823E8
:1060500079F00E9459250E94B8C9FE01EE0FFF1F7A
:10606000EE0FFF1FE55EF04E6083718382839383A2
:1060700084E40E949725882379F00E9459250E9484
:10608000C4C9FE01EE0FFF1FEE0FFF1FE95EF04EC9
:1060900060837183828393830E94B9C0E0E5F7E057
:1060A0008491882341F09091C00095FFFCCF8093AC
:1060B000C6003196F5CFEDE4F7E08491882341F0F6
:1060C0009091C00095FFFCCF8093C6003196F5CF2C
:1060D0004AE050E0BE0182EB98E00E948652E9E47B
:1060E000F7E08491882341F09091C00095FFFCCFA8
:1060F0008093C6003196F5CFCC0FDD1FCC0FDD1F8E
:10610000FE01E15EF04E408151816281738122E0A7
:1061100030E082EB98E00E945153E5E4F7E084918F
:10612000882341F09091C00095FFFCCF8093C6007A
:106130003196F5CFFE01E55EF04E6081718182817E
:1061400093810E94BEC9AB01BC0122E030E082EB2A
:1061500098E00E945153E1E4F7E08491882341F0F4
:106160009091C00095FFFCCF8093C6003196F5CF8B
:10617000C95ED04E688179818A819B810E94CAC99B
:10618000AB01BC0122E030E082EB98E00E94515369
:1061900017C09091C00095FFFCCF8093C600319648
:1061A00084918111F6CFE8E2F7E08491882341F0F1
:1061B0009091C00095FFFCCF8093C6003196F5CF3B
:1061C00082EB98E0DF91CF910C9472520F931F9362
:1061D000CF93DF9388E40E949725882321F00E94C3
:1061E0008A25EC0102C0C0E0D0E083E40E9497253C
:1061F000882321F00E948A258C0102C005E010E06E
:1062000083E50E949725882319F00E94592506C02E
:10621000D7FD09C060E070E086E193E4209739F48F
:106220001092790404C060E070E08CE892E4980178
:10623000AE01DF91CF911F910F910C94E3C32F9288
:106240003F924F925F926F927F928F929F92AF9206
:10625000BF92CF92DF92EF92FF920F931F93CF9353
:10626000DF93CDB7DEB768970FB6F894DEBF0FBEE9
:10627000CDBF8CE0E9E8F6E0DE01119601900D92C9
:106280008A95E1F78CE0E1EBF4E0DE011D960190E8
:106290000D928A95E1F74E018DE0880E911CFE016A
:1062A00031961F0100E010E0A12CB12C80917806FE
:1062B00090E00A2C02C0959587950A94E2F780FF3A
:1062C00081C0F1014080518062807380F801ED5EF1
:1062D000FD4F2081318142815381F801E756FB4F08
:1062E00060817181828193810E94CFD420E030E06F
:1062F00040E05FE30E947DD89B01AC01C301B20185
:106300000E94ABD7181644F4C8018D5F904F0E94CD
:10631000E2236B017C0103C0C12CD12C7601A701C3
:106320009601C301B2010E94CED42B013C0120E0B2
:1063300030E040EA51EC0E94ABD7181654F420E04C
:1063400030E040EA51E4C301B2010E94A8D587FDC4
:1063500003C0E0E2F7E01BC0A3019201F4016081F9
:106360007181828193810E94CED4F4016083718314
:1063700082839383F101C082D182E282F38222C0C0
:106380009091C00095FFFCCF8093C6003196849118
:106390008111F6CFE3E0F7E08491882341F09091FA
:1063A000C00095FFFCCF8093C6003196F5CF82EBFD
:1063B00098E00E94725285EF96E00E94EB6B87EEA8
:1063C00096E049C0FFEFAF1ABF0A84E0880E911C27
:1063D0000C5F1F4F94E0290E311CE3E0AE16B104B0
:1063E00009F064CF8CE0FE013196A9E8B6E0019097
:1063F0000D928A95E1F78CE0FE013D96A1EBB4E0A9
:1064000001900D928A95E1F70E94BB27E0EEF6E03D
:106410008491882341F09091C00095FFFCCF809338
:10642000C6003196F5CFE0EDF6E08491882341F087
:106430009091C00095FFFCCF8093C6003196F5CFB8
:1064400082EB98E00E94725260E080EC96E00E943D
:10645000E56B82EA96E090938B0480938A046896B9
:106460000FB6F894DEBF0FBECDBFDF91CF911F9165
:106470000F91FF90EF90DF90CF90BF90AF909F90E3
:106480008F907F906F905F904F903F902F900C94E3
:106490006224CF92DF92EF92FF92CF9383E50E9426
:1064A0009725882321F080914202811148C08CE415
:1064B0000E949725882321F08091420281114CC0CF
:1064C00080E50E949725882321F080914202811166
:1064D00059C084E40E949725882321F080914202CC
:1064E00081115BC082E40E949725882321F080916E
:1064F0004202811160C082E50E949725882321F025
:106500008091420281115FC086E40E949725882312
:1065100009F464C00E9459256B017C0120E030E041
:10652000A9010E94ABD718160CF058C0C0923D02CA
:10653000D0923E02E0923F02F09240024FC00E9491
:1065400059250E9417D670933A09609339097093C0
:10655000DC096093DB09ABCF0E9459250E9417D656
:1065600097FF07C090958095709561957F4F8F4FED
:106570009F4F60933F097093400980934109909326
:1065800042099ECF0E94592560933B0970933C09B4
:1065900080933D0990933E099CCF0E945925C1E00C
:1065A00020E030E0A9010E94A8D5811101C0C0E01F
:1065B000C0934E0997CF0E9459250E9417D6CB0150
:1065C0000E94F25598CF0E9459256093E10970937B
:1065D000E2098093E3099093E40996CFCF91FF906D
:1065E000EF90DF90CF900895CF92DF92EF92FF92DD
:1065F000882319F0EBE9F6E024C01092790486E4D0
:106600000E949725882309F449C00E9459256B01EF
:106610007C0120E030E0A9010E94ABD718160CF0F5
:106620003DC0C0923D02D0923E02E0923F02F09205
:10663000400234C02091C00025FFFCCF9093C600DB
:10664000319694919111F6CFE9E9F6E0949199236E
:1066500041F02091C00025FFFCCF9093C6003196F9
:10666000F5CF682F70E04AE050E082EB98E00E949E
:106670008652E7E8F6E08491882341F09091C000CB
:1066800095FFFCCF8093C6003196F5CF82EB98E062
:10669000FF90EF90DF90CF900C947252FF90EF90AC
:1066A000DF90CF90089582EB98E00E94BC51EEE716
:1066B000F6E08491882341F09091C00095FFFCCFD3
:1066C0008093C6003196F5CF40914E0650914F060B
:1066D00060915006709151064F5F5F4F6F4F7F4F33
:1066E0002AE030E082EB98E00E945B5282EB98E077
:1066F0000E947252EAE7F6E08491882341F090917B
:10670000C00095FFFCCF8093C6003196F5CF089569
:10671000CF93C62FE2E2FEE02491222341F0309194
:10672000C00035FFFCCF2093C6003196F5CFFC01A9
:106730008191882339F09091C00095FFFCCF809320
:10674000C600F6CF40914E0650914F06609150061C
:10675000709151062AE030E082EB98E00E945B5293
:1067600082EB98E00E947252C1119DDF109290045A
:1067700010928F04CF9108950E94E823E09148067B
:10678000F0914906E759FB4F8081811111C0E6E77E
:10679000F6E08491882341F09091C00095FFFCCFF2
:1067A0008093C6003196F5CF82EB98E00C9472523C
:1067B0000895CF92DF92EF92FF92CF93DF93EC0197
:1067C00080910D02882309F48BC0C0909904D09069
:1067D0009A04E0909B04F0909C04A70196016881C4
:1067E00079818A819B810E94A8D587FF04C0C882D5
:1067F000D982EA82FB82C0909D04D0909E04E090F2
:106800009F04F090A004A70196016C817D818E8188
:106810009F810E94A8D587FF04C0CC82DD82EE82D2
:10682000FF8220E030E0A9016091A1047091A204F0
:106830008091A3049091A4040E94CFD46B017C01A9
:106840009B01AC01688579858A859B850E94A8D5C6
:1068500087FF04C0C886D986EA86FB86C0901302EB
:10686000D0901402E0901502F0901602A701960154
:10687000688179818A819B810E94ABD7181624F4A4
:10688000C882D982EA82FB82C0901702D090180297
:10689000E0901902F0901A02A70196016C817D81A7
:1068A0008E819F810E94ABD7181624F4CC82DD82A2
:1068B000EE82FF82C0901B02D0901C02E0901D026D
:1068C000F0901E02A7019601688579858A859B85CF
:1068D0000E94ABD7181624F4C886D986EA86FB86B0
:1068E000DF91CF91FF90EF90DF90CF9008952091AE
:1068F0008506309186064091870650918806609102
:1069000095067091960680919706909198060E9440
:10691000A8D5882391F12091790630917A0640918B
:106920007B0650917C066091890670918A06809161
:106930008B0690918C060E94A8D5811114C02091DD
:106940007D0630917E0640917F06509180066091D1
:106950008D0670918E0680918F06909190060E9410
:10696000A8D5882391F081E0809347098CE090E0DE
:10697000909338098093370908C080913709909126
:1069800038090C9711F4109247092091790630913B
:106990007A0640917B0650917C0660918906709141
:1069A0008A0680918B0690918C060E94A8D5811151
:1069B00017C020917D0630917E0640917F06509150
:1069C000800660918D0670918E0680918F06909161
:1069D00090060E94A8D5811103C00E94B2271CC056
:1069E00060912B0270912C02882777FD8095982F5B
:1069F0000E944AD620913D0230913E0240913F02D2
:106A0000509140020E947DD820E030E048EC52E4F2
:106A10000E94AFD50E948F2781E0089589E796E014
:106A2000C8DE0E94E82363DF81110C94C529089514
:106A3000CF93DF93C82F80914202882309F481C04D
:106A40000E94222ACC23B1F183E50E949725882356
:106A500021F080914202811134C08CE40E9497257C
:106A6000882321F080914202811134C080E50E9488
:106A70009725882321F080914202811141C084E44E
:106A80000E949725882321F080914202811143C002
:106A900082E40E949725882321F08091420281118F
:106AA00048C081E0809347098AE090E090933809DC
:106AB00080933709B3DFCC2309F443C01092470910
:106AC00040C00E9459250E9417D670933A096093DE
:106AD0003909C3CF0E9459250E9417D697FF07C0D6
:106AE00090958095709561957F4F8F4F9F4F6093E4
:106AF0003F09709340098093410990934209B6CFB2
:106B00000E94592560933B0970933C0980933D098D
:106B100090933E09B4CF0E945925D1E020E030E0A7
:106B2000A9010E94A8D5811101C0D0E0D0934E09DF
:106B3000AFCF0E9459250E9417D6CB010E94F25573
:106B4000B0CFDF91CF910895CF92DF92EF92FF9275
:106B5000CF938CE40E949725882341F00E94592509
:106B60000E9417D67093E6096093E50984E20E94BB
:106B70009725882399F10E945925C1E020E030E053
:106B8000A9010E94A8D5811101C0C0E0C093E90904
:106B90002091DD093091DE094091DF095091E00933
:106BA0006091E1097091E2098091E3099091E40913
:106BB0000E947DD89B01AC0160918D0670918E067C
:106BC00080918F06909190060E94CFD460937D06AD
:106BD00070937E0680937F069093800684E40E94E3
:106BE0009725882391F04091E5095091E60960913D
:106BF0008C0470918D046F5F7F4F83E599E00E9454
:106C0000B9539093E8098093E7098091E90960916D
:106C1000E7097091E809F0904E09811141C0882779
:106C200077FD8095982F0E944AD62091E1093091F6
:106C3000E2094091E3095091E4090E947DD89B014B
:106C4000AC016091890670918A0680918B069091C3
:106C50008C060E94CED46093790670937A06809356
:106C60007B0690937C06FF2009F45FC0E0E7FCE020
:106C70008491882341F09091C00095FFFCCF8093D0
:106C8000C6003196F5CFEBE5FCE084918823C1F195
:106C90009091C00095FFFCCF8093C6003196F5CF50
:106CA000882777FD8095982F0E944AD62091E10988
:106CB0003091E2094091E3095091E4090E947DD8A6
:106CC0009B01AC016091890670918A0680918B06C8
:106CD00090918C060E94CFD46093790670937A06C7
:106CE00080937B0690937C06FF20F9F0E4E5FCE0BE
:106CF000849181110AC0EFE3FCE0849181110DC001
:106D000082EB98E00E94725210C09091C00095FFF3
:106D1000FCCF8093C6003196EBCF9091C00095FFD9
:106D2000FCCF8093C6003196E8CF2091E1093091E5
:106D3000E2094091E3095091E40960E070E080E8E5
:106D40009FE30E94AFD56B017C0160933B09709378
:106D50003C0980933D0990933E0920E030E040E7F4
:106D600052E460913D0270913E0280913F02909109
:106D700040020E94AFD59B01AC0160E074E284E761
:106D800099E40E94AFD5A70196010E94AFD50E9459
:106D90001CD660933F0970934009809341099093FA
:106DA000420982E08093490981E08093470982E0AB
:106DB00090E09093380980933709CF91FF90EF903E
:106DC000DF90CF902BCEAF92BF92CF92DF92EF9217
:106DD000FF920F931F93CF93DF93809176068823C2
:106DE00009F410C183E50E949725882331F00E94A1
:106DF00059250E9417D6EB0102C0C0E0D0E0C23096
:106E0000D10518F4EEEAFAE037C0E1EDFAE084913A
:106E1000882341F09091C00095FFFCCF8093C6007D
:106E20003196F5CFE5EBFAE08491882341F090911B
:106E3000C00095FFFCCF8093C6003196F5CF4AE0A5
:106E400050E062E070E082EB98E00E94865282EBB4
:106E500098E0DF91CF911F910F91FF90EF90DF901D
:106E6000CF90BF90AF900C9472529091C00095FF5C
:106E7000FCCF8093C600319684918111F6CFEBE967
:106E8000FAE08491882341F09091C00095FFFCCFF7
:106E90008093C6003196F5CFE8E9FAE08491882323
:106EA00041F09091C00095FFFCCF8093C6003196D1
:106EB000F5CF4AE050E0BE0182EB98E00E94865296
:106EC000E5E9FAE08491882341F09091C00095FFB4
:106ED000FCCF8093C6003196F5CF86E40E949725BB
:106EE000882399F00E9459256B017C0120E030E055
:106EF000A9010E94ABD7181644F4C0923D02D0926B
:106F00003E02E0923F02F092400209E716E053EFA2
:106F1000E52E53E0F52E6E0164E0CC0CDD1C6A9585
:106F2000E1F7C6018A5A994F6C01C0E0D0E05701E1
:106F3000F70180810E949725882389F00E945925B6
:106F4000F601EC0FFD1F20813181428153810E94A7
:106F5000CFD4F80160837183828393830CC0FE01D8
:106F6000E757F94F80819181A281B381F801808335
:106F70009183A283B383E3E9FAE08491882341F00B
:106F80009091C00095FFFCCF8093C6003196F5CF5D
:106F9000FFEFEF1AFF0A40E050E0F501608182EB5D
:106FA00098E00E946A52E1E9FAE08491882341F076
:106FB0009091C00095FFFCCF8093C6003196F5CF2D
:106FC000F80141915191619171918F0122E030E07E
:106FD00082EB98E00E9451532496C031D10509F00C
:106FE000A6CF82EB98E00E94725218DDDF91CF911C
:106FF0001F910F91FF90EF90DF90CF90BF90AF90D7
:107000000C94AEA1DF91CF911F910F91FF90EF9063
:10701000DF90CF90BF90AF900895CF9383E50E940B
:107020009725882321F080914202811131C08CE4A0
:107030000E949725882321F080914202811131C05E
:1070400080E50E949725882321F0809142028111DA
:107050003EC084E40E949725882321F0809142025B
:10706000811140C082E40E949725882321F08091FD
:107070004202811145C081E0809347098BE090E096
:1070800090933809809337090E94936CCF91C6CCB6
:107090000E9459250E9417D670933A0960933909C6
:1070A000C6CF0E9459250E9417D697FF07C090951A
:1070B0008095709561957F4F8F4F9F4F60933F09EB
:1070C000709340098093410990934209B9CF0E947F
:1070D000592560933B0970933C0980933D09909337
:1070E0003E09B7CF0E945925C1E020E030E0A90158
:1070F0000E94A8D5811101C0C0E0C0934E09B2CF53
:107100000E9459250E9417D6CB010E94F255B3CF99
:107110002F923F924F925F926F927F928F929F92A7
:10712000AF92BF92CF92DF92EF92FF920F931F9395
:10713000CF93DF93CDB7DEB7C654D1090FB6F8941D
:10714000DEBF0FBECDBF1C017EA76DA7142FDB01D4
:1071500014968D909D90AD90BC901797CD90DD903A
:10716000ED90FC90A5019401C701B6010E94B8D72B
:1071700023966CAF7DAF8EAF9FAF2397809189062A
:1071800090918A06A0918B06B0918C06898F9A8F78
:10719000AB8FBC8FA7019601BC01CD010E94CFD45B
:1071A0006FAB78AF89AF9AAF80918D0690918E06C4
:1071B000A0918F06B09190068D8F9E8FAF8FB8A350
:1071C000A5019401BC01CD010E94CFD46BAF7CAF6F
:1071D0008DAF9EAF8091910690919206A0919306FB
:1071E000B091940689A39AA3ABA3BCA39C01AD0163
:1071F000D10118966D917D918D919C911B970E9464
:10720000CED46DA37EA38FA398A7D1011C968D9198
:107210009D910D90BC91A02D27968CAF9DAFAEAFE8
:10722000BFAF27978091950690919606A0919706FB
:10723000B091980689A79AA7ABA7BCA7D701C601AA
:10724000B0588D8B9E8BAF8BB88FD501C401B058D1
:10725000898B9A8BAB8BBC8BD1018D919D910D90BD
:10726000BC91A02D8FA798ABA9ABBAAB2FA938AD15
:1072700049AD5AADBC01CD010E94CED46B017C0159
:10728000D10114968D919D910D90BC91A02D8BAB49
:107290009CABADABBEAB2BAD3CAD4DAD5EADBC0163
:1072A000CD010E94CED44B015C01A70196016D89EE
:1072B0007E898F89988D0E947DD82B013C01A50184
:1072C000940169897A898B899C890E947DD89B0168
:1072D000AC01C301B2010E94CFD42B013C01A50136
:1072E00094016D897E898F89988D0E947DD84B018C
:1072F0005C01A701960169897A898B899C890E9422
:107300007DD89B01AC01C501B4010E94CED4A3017C
:1073100092010E9442D56B017C0120E030E0A9017E
:107320000E94A8D587FF0AC02BED3FE049EC50E44E
:10733000C701B6010E94CFD46B017C01112351F02B
:107340002BED3FE049EC50E4C701B6010E94CED4DA
:107350006B017C012FA538A949A95AA9698D7A8D9D
:107360008B8D9C8D0E94A8D581111FC02BA93CA993
:107370004DA95EA96D8D7E8D8F8D98A10E94A8D597
:10738000811113C020E030E0A901C701B6010E94BD
:10739000A8D581110AC02BED3FE049EC50E4C701AC
:1073A000B6010E94CFD46B017C0123962CAD3DAD7C
:1073B0004EAD5FAD2397C701B6010E947DD82DA1C8
:1073C0003EA14FA158A55F770E94B8D74B015C0141
:1073D0002FE632E143E85AE30E94A8D587FDB8C101
:1073E000C501B4010E9485D60E941CD67A8F698F90
:1073F000FB01EF2B21F421E030E03A8F298FA98D9A
:10740000BA8DBD0180E090E00E9448D64B015C013E
:107410009B01AC01C701B6010E94AFD52B013C0115
:10742000A50194016DA17EA18FA198A50E94AFD561
:107430006FA778AB89AB9AAB29A53AA54BA55CA5FC
:1074400027966CAD7DAD8EAD9FAD27970E94CED4B3
:10745000A50194010E94AFD56BAB7CAB8DAB9EAB0D
:1074600020E030E040E05FE3C301B2010E947DD83C
:10747000A30192010E947DD89B01AC0160E070E005
:1074800080E89FE30E94CED46DA37EA38FA398A72C
:1074900089A19AA1ABA1BCA189879A87AB87BC8738
:1074A00089A59AA5ABA5BCA58D879E87AF87B88B0C
:1074B00060912B0270912C02882777FD8095982F80
:1074C0000E944AD620913D0230913E0240913F02F7
:1074D000509140020E947DD820E030E040E752E425
:1074E0000E94AFD520E030E048EC52E40E94AFD5D6
:1074F00069A37AA38BA39CA3B12CA1E0B0E0BE8FBB
:10750000AD8F2D8D3E8D898D9A8D2817390708F006
:1075100009C1B8E1BB150CF444C02DA13EA14FA197
:1075200058A569897A898B899C890E947DD86B01CD
:107530007C01A30192016D897E898F89988D0E94BB
:107540007DD8A70196010E94CFD4A62E172F982E82
:10755000892E2DA13EA14FA158A56D897E898F89C5
:10756000988D0E947DD86B017C01A30192016989ED
:107570007A898B899C890E947DD89B01AC01C701C7
:10758000B6010E94CED46D8B7E8B8F8B988FB39477
:107590008A2D912FA92DB82D898B9A8BAB8BBC8B03
:1075A0006BC0ED8DFE8DBF0180E090E00E9448D65B
:1075B000A30192010E947DD86B017C010E94ACD591
:1075C000698B7A8B8B8B9C8BC701B6010E94E0D8AC
:1075D0004B015C01ADA5BEA5CD90DD90ED90FC907A
:1075E0001397F7FAF094F7F8F09414968D919D9113
:1075F0000D90BC91A02D89A79AA7ABA7BCA72989FC
:107600003A894B895C89C701B6010E947DD86D8B90
:107610007E8B8F8B988FA501940169A57AA58BA588
:107620009CA50E947DD89B01AC016D897E898F89C4
:10763000988D0E94CFD46D8B7E8B8F8B988FA501F8
:107640009401C701B6010E947DD86B017C01298994
:107650003A894B895C8969A57AA58BA59CA50E946E
:107660007DD89B01AC01C701B6010E94CED4698BC5
:107670007A8B8B8B9C8BB12C2D893E894F89588DB1
:107680006FA978AD89AD9AAD0E94CFD469837A8312
:107690008B839C8329893A894B895C896BAD7CAD4E
:1076A0008DAD9EAD0E94CFD46D837E838F839887EE
:1076B0002FA538A949A95AA969857A858B859C8502
:1076C0000E94CFD469877A878B879C872BA93CA996
:1076D0004DA95EA96D857E858F8598890E94CFD43E
:1076E0006D877E878F87988BCE01019662D8A09098
:1076F0009604C0909804E9A0FAA00BA11CA19E01D9
:10770000235F3F4FAE01475F5F4FBE016B5F7F4F0F
:10771000CE0101960E94A08BED8DFE8D3196FE8FDD
:10772000ED8FEFCE9101245F3F4FA101485F5F4F86
:10773000B1016C5F7F4FA0909604C0909804E9A0BF
:10774000FAA00BA11CA1C1010E94A08B0E94C52917
:10775000CA5BDF4F0FB6F894DEBF0FBECDBFDF911F
:10776000CF911F910F91FF90EF90DF90CF90BF903E
:10777000AF909F908F907F906F905F904F903F90D1
:107780002F9008950F931F93CF93DF93CDB7DEB75C
:1077900028970FB6F894DEBF0FBECDBF182F80918B
:1077A0004202882309F4A2C00E94222A83E50E9493
:1077B0009725882321F080914202811157C08CE4E3
:1077C0000E949725882321F080914202811157C0A1
:1077D00080E50E949725882321F080914202811143
:1077E00064C084E40E949725882321F0809142029E
:1077F000811166C082E40E949725882321F0809140
:10780000420281116BC081E0809347098AE090E0D9
:10781000909338098093370989E40E94972588233B
:1078200019F00E94592503C060E070E0CB01698324
:107830007A838B839C838AE40E949725882319F09E
:107840000E94592503C060E070E0CB016D837E8308
:107850008F839887412FBE016F5F7F4F89E796E046
:1078600057DC0E94E8231092470940C00E94592526
:107870000E9417D670933A0960933909A0CF0E94ED
:1078800059250E9417D697FF07C09095809570954F
:1078900061957F4F8F4F9F4F60933F0970934009D1
:1078A000809341099093420993CF0E945925609398
:1078B0003B0970933C0980933D0990933E0991CF19
:1078C0000E94592501E020E030E0A9010E94A8D5DE
:1078D000811101C000E000934E098CCF0E94592510
:1078E0000E9417D6CB010E94F2558DCF28960FB675
:1078F000F894DEBF0FBECDBFDF91CF911F910F91E6
:1079000008950E94EB6BF8940E946FC30E9412A22C
:107910000E94A155E5E6F6E08491882341F090911C
:10792000C00095FFFCCF8093C6003196F5CFE6E40A
:10793000F6E08491882341F09091C00095FFFCCF40
:107940008093C6003196F5CF82EB98E00E94725288
:107950007894C6E0D0E0219749F068EC70E080E0D0
:1079600090E00E9429D00E94936CF5CFF894FFCF4D
:107970002F923F924F925F926F927F928F929F923F
:10798000AF92BF92CF92DF92EF92FF920F931F932D
:10799000CF93DF93CDB7DEB76E970FB6F894DEBF07
:1079A0000FBECDBF0E9462248111E9C2A0E69A2ECB
:1079B000B4E0AB2EB12C772473948091330990916D
:1079C00034092091350930913609821B930B8F774A
:1079D0009927892B39F080914406909145060497A8
:1079E0000CF448C08091FC06882309F4C8C2809139
:1079F0008F0490919004892B09F0C1C280914406B4
:107A000090914506892B11F410926804ECE3CE2E78
:107A1000D12CE12CF12CF0E14F2EFEE05F2E612CF9
:107A2000712C8E010F5F1F4F70E6272E3324339485
:107A30004091030750910407609105077091060774
:107A40008091FF0690910007A0910107B091020775
:107A5000481759076A077B0708F091C280914406CE
:107A60009091450604970CF08AC2809168048111B8
:107A700086C25FC182EB98E00E94A051809391047E
:107A800020918F04309190048A3031F08D3021F0B4
:107A90002F3531050CF408C110928E0421153105E3
:107AA00009F46DC24091460650914706949EC0016C
:107AB000959E900D11248C539B4FFC01E20FF31FF8
:107AC0001082FA01E759FB4F10828C01DC012C91E6
:107AD00001962032D1F378012E3411F000E010E04D
:107AE0006AE270E0C7010E9431DE6C0101151105E8
:107AF00009F478C06DE17EE0C7010E94F0DD8824C2
:107B00008394892B11F4812C09C06EE470E0C701C5
:107B100004960E9431DE009709F08C014AE050E0A3
:107B200060E070E0C80101960E9488DC6093520614
:107B300070935306809354069093550620914E06F9
:107B400030914F0640915006509151062F5F3F4FA4
:107B50004F4F5F4F621773078407950731F081100D
:107B600004C061E08AEE9DE022C0C114D10411F18D
:107B700080E010E0F701E80FF11D90819A3219F0D2
:107B80008F5F1927F7CF4AE050E060E070E0C60150
:107B900001960E9488DC012F10E020E030E06017A1
:107BA00071078207930769F061E08BEC9DE00E940A
:107BB0008833E5C10E151F0521F461E081EA9DE0DF
:107BC000F6CF8091520690915306A0915406B09141
:107BD000550680934E0690934F06A0935006B0939F
:107BE000510606C0009721F060E087E79DE0DFCFF7
:107BF00080914202811134C067E470E0C7010E94A5
:107C000031DE009769F14AE050E060E070E00196F3
:107C10000E9488DC6430710518F5EFE6FDE0849180
:107C2000882341F09091C00095FFFCCF8093C6005F
:107C30003196F5CFE9EFFCE08491882341F09091F3
:107C4000C00095FFFCCF8093C6003196F5CF82EB44
:107C500098E00E94725260E08FEE9CE00E94E56B1B
:107C600069E873E0C7010E943CDE892B19F486EEB7
:107C70009CE047DE80914606909147060196B5014B
:107C80000E9473D9909347068093460680914406DC
:107C90009091450601969093450680934406109274
:107CA000900410928F0489CE8C3529F58091330988
:107CB000909134092091350930913609821B930B3C
:107CC0008F779927892B09F478CE8091440690917B
:107CD000450604970CF071CE82EB98E00E94A0510B
:107CE00080939104409146065091470620918F045D
:107CF000309190040CC08B3311F470928E049091EB
:107D00008E0491115ACE4091460650914706B90112
:107D10006F5F7F4F7093900460938F04949EF00187
:107D2000959EF00D1124E20FF31FEC53FB4F80835F
:107D300044CE8091E9069091EA06A091EB06B091BD
:107D4000EC068093030790930407A0930507B09374
:107D500006078EED96E00E9497A940910307509187
:107D6000040760910507709106074F5F5F4F6F4FE3
:107D70007F4F409303075093040760930507709368
:107D80000607E82F809391048A30B1F0ED30A1F01E
:107D9000E33211F0EA3321F420918E04222361F0C2
:107DA00020918F04309190042F3531052CF48F3FB2
:107DB000BFEF9B0709F0C5C08091FF0690910007B7
:107DC000A0910107B0910207481759076A077B077E
:107DD00008F47BC0E3EDFCE08491882341F09091AE
:107DE000C00095FFFCCF8093C6003196F5CF82EBA3
:107DF00098E00E9472520E94FACF60937A047093C6
:107E00007B0480937C0490937D0480907E0490900A
:107E10007F04A0908004B0908104681979098A09D0
:107E20009B0928EE33E040E050E00E9486D94901EA
:107E30005A01CA01B901A70196010E9486D9CA0157
:107E4000B901A70196010E9486D97F936F93C5015E
:107E5000B401A30192010E9486D93F932F93AFEB07
:107E6000BCE0BF93AF931F930F930E9466DE0FB6E3
:107E7000F894DEBF0FBECDBFE8EBFCE08491882311
:107E800041F09091C00095FFFCCF8093C6003196E1
:107E9000F5CFF8018191882339F09091C00095FFCA
:107EA000FCCF8093C600F6CF82EB98E00E9472521E
:107EB00061E0C8010E94F6688EE996E00E94A0BFCA
:107EC00061E08EE996E00E9455BF80919104833273
:107ED00011F43092680420918F04309190042115A0
:107EE000310519F410928E044AC080914606909193
:107EF0004706289EF001299EF00D1124E20FF31F82
:107F0000EC53FB4F1082FC01E759FB4F308220916C
:107F10004406309145062F5F3F4F3093450620932E
:107F20004406019664E070E00E9473D9909347067E
:107F30008093460610928E041092900410928F0443
:107F400077CDEB3311F430928E0440918E044111C1
:107F50006BCD4091460650914706B9016F5F7F4F48
:107F60007093900460938F04249EF001259EF00D81
:107F70001124E20FF31FEC53FB4F808359CD6E9613
:107F80000FB6F894DEBF0FBECDBFDF91CF911F912A
:107F90000F91FF90EF90DF90CF90BF90AF909F90A8
:107FA0008F907F906F905F904F903F902F900895AB
:107FB000CF92DF92EF92FF920F931F93CF93C82F30
:107FC000809144069091450603970CF4D1DC0E9401
:107FD000FACFC0908204D0908304E0908404F090A3
:107FE0008504C114D104E104F104A1F000918604D8
:107FF0001091870420918804309189040C0D1D1D77
:108000002E1D3F1D061717072807390718F48DE6A0
:1080100096E077DCC0900F02D0901002E090110241
:10802000F0901202C114D104E104F10479F100913D
:1080300086041091870420918804309189040C0DE6
:108040001D1D2E1D3F1D0617170728073907F0F4C1
:10805000C1111CC09091A50C8091A40C981316C05E
:1080600080914F099091500980369A4E68F0809126
:1080700051099091520901969093520980935109A8
:108080001092500910924F090E94A155CF911F9153
:108090000F91FF90EF90DF90CF900C94848BCF9353
:1080A000DF931F92CDB7DEB789830E9476C28981A4
:1080B0007FDF0F90DF91CF910C94936C8F929F9202
:1080C000AF92BF92CF92DF92EF92FF924B015C0191
:1080D0000E94FACF6B017C01C80CD91CEA1CFB1C66
:1080E0000E94FACF6C157D058E059F0518F480E07F
:1080F000D6DFF6CFFF90EF90DF90CF90BF90AF909C
:108100009F908F9008958F929F92AF92BF92CF923F
:10811000DF92EF92FF9280E50E949725882329F055
:108120000E947F254B015C0103C0812C912C5401DE
:1081300083E50E949725882361F00E94592520E05D
:1081400030E04AE754E40E947DD80E941CD64B01DF
:108150005C010E94AEA10E94E823C0908604D090EA
:108160008704E0908804F0908904C80CD91CEA1CAC
:10817000FB1C0E94EF68811105C060E087E79CE06E
:108180000E94E56B0E94FACF6C157D058E059F0558
:1081900018F480E084DFF6CFFF90EF90DF90CF906F
:1081A000BF90AF909F908F9008952F923F924F92E3
:1081B0005F926F927F928F929F92AF92BF92CF9277
:1081C000DF92EF92FF920F931F93CF93DF93CDB780
:1081D000DEB728970FB6F894DEBF0FBECDBF8091F3
:1081E000410281FF1EC0E8E3FCE08491882341F056
:1081F0009091C00095FFFCCF8093C6003196F5CFDB
:10820000EAE2FCE08491882341F09091C00095FF60
:10821000FCCF8093C6003196F5CF82EB98E00E94A8
:1082200072520E94AEA180913D0290913E02A091B7
:108230003F02B09140028093990690939A06A093D2
:108240009B06B0939C0680912B0290912C029093F8
:10825000BF048093BE0484E690E090932C02809348
:108260002B020E94E82381E00E940D9880E1E9E85A
:10827000F6E0A9E7B6E001900D928A95E1F782E475
:108280000E949725C82E882341F180913D0290914C
:108290003E02A0913F02B091400289839A83AB8352
:1082A000BC834090890650908A0660908B0670903F
:1082B0008C0680908D0690908E06A0908F06B090D0
:1082C00090068091910690919206A0919306B091AC
:1082D00094068D839E83AF83B88710923D021092DF
:1082E0003E0210923F021092400288E50E949725BC
:1082F000282E89E50E949725382E8AE50E94972529
:10830000D82E85E40E949725211007C0311009C09E
:10831000D11007C091E0982705C0332011F09D2DA2
:1083200001C090E090930A02911102C02220E1F076
:1083300080E090E00E94C5278091410281FF14C037
:10834000E3E2FCE08491882341F09091C00095FF26
:10835000FCCF8093C6003196F5CF41E069E876E026
:108360008EE893E00E942B2680910A02811102C0C0
:108370003320E1F081E090E00E94C5278091410226
:1083800081FF14C0ECE1FCE08491882341F09091DE
:10839000C00095FFFCCF8093C6003196F5CF41E039
:1083A00069E876E086E993E00E942B268DE40E943E
:1083B0009725882309F44AC2211048C2311046C2C9
:1083C000E5E1FCE08491882341F09091C00095FFA5
:1083D000FCCF8093C6003196F5CFEDEFFBE08491A2
:1083E000882341F09091C00095FFFCCF8093C60098
:1083F0003196F5CF82EB98E00E9472520E944F6E48
:10840000811103C081E04BDEF9CF80913D02909154
:108410003E02A0913F02B091400280939906909352
:108420009A06A0939B06B0939C0680912B02909194
:108430002C029093BF048093BE0484E690E0909356
:108440002C0280932B020E94E82381E00E940D9869
:108450008091890690918A06A0918B06B0918C0636
:108460008093790690937A06A0937B06B0937C065E
:1084700080918D0690918E06A0918F06B091900606
:1084800080937D0690937E06A0937F06B09380062E
:108490008091910690919206A0919306B0919406D6
:1084A0008093810690938206A0938306B0938406FE
:1084B0008091950690919606A0919706B0919806A6
:1084C0008093850690938606A0938706B0938806CE
:1084D00010923D0210923E0210923F021092400212
:1084E00080E090E00E94C52781E090E00E94C527CF
:1084F00082E090E00E94C5270E94BB2780E00E9496
:108500000D988091990690919A06A0919B06B09142
:108510009C0680933D0290933E02A0933F02B0934D
:1085200040028091BE049091BF0490932C028093EE
:108530002B020E94E8230E944E970E94BB272091A5
:108540008D0630918E0640918F0650919006609175
:10855000890670918A0680918B0690918C06E12C99
:10856000F12C00EA10E40E94DC2681E090E00E94F9
:108570002A5AE0909106F09092060091930610918D
:10858000940620E030E040EA51E4CA01B9010E94BB
:10859000DC2620918D0630918E0640918F065091F9
:1085A00090066091890670918A0680918B06909161
:1085B0008C06E12CF12C87010E94DC260E944F6E74
:1085C000811103C081E06BDDF9CF82E090E00E9471
:1085D0002A5A20918D0630918E0640918F06509137
:1085E00090066091890670918A0680918B06909121
:1085F0008C06E12CF12C00EA10E40E94DC26E090CD
:108600009106F0909206009193061091940620E056
:1086100030E040EA51E460E070E084E393E40E94DB
:10862000DC2620918D0630918E0640918F06509168
:1086300090066091890670918A0680918B069091D0
:108640008C06E12CF12C87010E94DC260E944F6EE3
:10865000811103C081E023DDF9CF83E090E00E9427
:108660002A5A20918D0630918E0640918F065091A6
:1086700090066091890670918A0680918B06909190
:108680008C06E12CF12C00EA10E40E94DC26E0903C
:108690009106F0909206009193061091940620E0C6
:1086A00030E044E353E4CA01B9010E94DC26209182
:1086B0008D0630918E0640918F0650919006609104
:1086C000890670918A0680918B0690918C06E12C28
:1086D000F12C87010E94DC260E944F6E811103C09D
:1086E00081E0DDDCF9CF84E090E00E942A5A2091FD
:1086F0008D0630918E0640918F06509190066091C4
:10870000890670918A0680918B0690918C06E12CE7
:10871000F12C00EA10E40E94DC26E0909106F09033
:108720009206009193061091940620E030E044E315
:1087300053E460E070E080EA91E40E94DC2620913E
:108740008D0630918E0640918F0650919006609173
:10875000890670918A0680918B0690918C06E12C97
:10876000F12C87010E94DC260E944F6E811103C00C
:1087700081E095DCF9CF85E090E00E942A5A2091B3
:108780008D0630918E0640918F0650919006609133
:10879000890670918A0680918B0690918C06E12C57
:1087A000F12C00EA10E40E94DC26E0909106F090A3
:1087B0009206009193061091940620E030E046EE78
:1087C00052E460E070E088E293E40E94DC262091AD
:1087D0008D0630918E0640918F06509190066091E3
:1087E000890670918A0680918B0690918C06E12C07
:1087F000F12C87010E94DC260E944F6E811103C07C
:1088000081E04DDCF9CF86E090E00E942A5A209169
:108810008D0630918E0640918F06509190066091A2
:10882000890670918A0680918B0690918C06E12CC6
:10883000F12C00EA10E40E94DC2689EF9BE0909383
:108840008B0480938A040E94622406C080910A02ED
:108850008111C4C0D110C2C00E94BB2780E00E9419
:108860000D988091990690919A06A0919B06B091DF
:108870009C0680933D0290933E02A0933F02B093EA
:1088800040028091BE049091BF0490932C0280938B
:108890002B020E94E8230E944E97CC2009F464C06A
:1088A0002220D1F080912D0290912E02A0912F02D2
:1088B000B091300280933D0290933E02A0933F021C
:1088C000B09340024092790650927A0660927B06FD
:1088D00070927C060E940E353320D1F080913102D7
:1088E00090913202A0913302B091340280933D0204
:1088F00090933E02A0933F02B093400280927D0687
:1089000090927E06A0927F06B09280060E940E355D
:10891000DD20F1F08091350290913602A09137026E
:10892000B091380280933D0290933E02A0933F02A3
:10893000B09340028D819E81AF81B885809381067E
:1089400090938206A0938306B09384060E940E350E
:1089500089819A81AB81BC8180933D0290933E02D4
:10896000A0933F02B09340028091410281FF53C027
:10897000EBEEFBE08491882341F09091C00095FFDD
:10898000FCCF8093C6003196F5CFEDEDFBE08491EE
:10899000882341F09091C00095FFFCCF8093C600E2
:1089A0003196F5CF82EB98E028960FB6F894DEBFAB
:1089B0000FBECDBFDF91CF911F910F91FF90EF9030
:1089C000DF90CF90BF90AF909F908F907F906F90EF
:1089D0005F904F903F902F900C94725282E090E005
:1089E0000E94C5278091410281FF36CFE2EFFBE074
:1089F0008491882341F09091C00095FFFCCF809333
:108A0000C6003196F5CF41E069E876E08EE993E063
:108A10000E942B2621CF28960FB6F894DEBF0FBEFA
:108A2000CDBFDF91CF911F910F91FF90EF90DF901D
:108A3000CF90BF90AF909F908F907F906F905F90FE
:108A40004F903F902F9008958F929F92AF92BF9238
:108A5000CF92DF92EF92FF921F93CF93DF93C0915B
:108A60004A06D0914B0680E50E949725882379F02D
:108A70000E948A256C01EE24D7FCE094FE2C11E0C4
:108A8000C114D104E104F10431F410E004C010E099
:108A9000C12CD12C760183E50E9497258823D9F03B
:108AA0000E94592520E030E04AE754E40E947DD836
:108AB0000E941CD66B017C0111110FC0611571055C
:108AC0008105910551F48881882339F061E0CE0158
:108AD0000E94F66807C01123B1F360E080E89AE0D5
:108AE0000E94E56B81E00E94A0680E94AEA10E94F6
:108AF000E823C114D104E104F104C1F0809086049C
:108B000090908704A0908804B09089048C0C9D1CE0
:108B1000AE1CBF1C0E94FACF681579058A059B051B
:108B200080F40E944F6E81110CC025C00E944D6ED2
:108B3000882321F10E944F6E811106C080E0AFDAD8
:108B4000F9CF80E00E94A0688091FC0660E0882355
:108B500019F081E79AE002C080E69AE0DF91CF91B8
:108B60001F91FF90EF90DF90CF90BF90AF909F90BC
:108B70008F900C94E56B80E092DACCCFDF91CF91AF
:108B80001F91FF90EF90DF90CF90BF90AF909F909C
:108B90008F9008954F925F926F927F928F929F92E3
:108BA000AF92BF92CF92DF92EF92FF920F931F93FB
:108BB00080910E028823B9F060916B1F70916C1F39
:108BC000882777FD8095982F0E944AD62091511FC3
:108BD0003091521F4091531F5091541F0E94ABD7A8
:108BE00018160CF0C1C0109293040E94FACF4B01EA
:108BF0005C012B013C0188EE480E83E0581E611C8D
:108C0000711CCC24CA94DC2C7601809193048111D0
:108C100094C0F7FE86C00E94FACF4B015C01461655
:108C200057066806790608F043C02B013C0188EE20
:108C3000480E83E0581E611C711C0E94CF29E6ED8E
:108C4000F9E08491882341F09091C00095FFFCCF1A
:108C50008093C6003196F5CFF7FE03C0E4EDF9E04E
:108C600020C0C701B601605F784D8F4F9F4F6819D4
:108C700079098A099B0928EE33E040E050E00E9420
:108C800086D9BA01A9012AE030E082EB98E00E947F
:108C90005B520AC09091C00095FFFCCF8093C60044
:108CA000319684918111F6CF82EB98E00E94725246
:108CB00080E0F5D960916B1F70916C1F882777FD5C
:108CC0008095982F0E944AD69B01AC016091511F5C
:108CD0007091521F8091531F9091541F0E94CED4C7
:108CE0000E9417D697FF07C0909580957095619563
:108CF0007F4F8F4F9F4FF7FE05C001E010E020E04F
:108D000030E004C003E010E020E030E00617170771
:108D1000280739070CF079CF0E94FACF6B017C014C
:108D200074CFD701C601805F984DAF4FBF4F8816F3
:108D30009906AA06BB0608F46ECF60E086EC99E0BF
:108D40000E94E56B0E94E82380918604909187043D
:108D5000A0918804B091890480937E0490937F044D
:108D6000A0938004B09381041F910F91FF90EF9026
:108D7000DF90CF90BF90AF909F908F907F906F903B
:108D80005F904F900895CF92DF92EF92FF92CF9332
:108D9000DF9380E50E949725882309F44FC00E9445
:108DA00059256B017C0183E50E949725882331F0CA
:108DB0000E9459250E9417D6EB0102C0CFEFDFEFCA
:108DC000CE0101960397D0F5C701B6010E9417D6D0
:108DD000F62E262F372FE1ECF3E041915191421707
:108DE000530761F183E0E33FF807B9F737FD26C089
:108DF0000E94AEA1EF2C60E08F2D0E94E5D1CF3F05
:108E00008FEFD80729F0219771F0C0E0D0E00DC0B6
:108E10008F2D0E9453D231E020E0892B09F030E001
:108E2000C32FD22F02C0C1E0D0E08E2D0E9453D2BA
:108E30008C179D0719F080E032D9F7CFDF91CF91E1
:108E4000FF90EF90DF90CF90089567707727E82F1D
:108E5000F0E0E35CFE4C849190E0FC013797EC304D
:108E6000F10578F5EE58FF4F0C94C4D98091B1000C
:108E7000887F8093B1008091B100862B8093B100F0
:108E8000089580919100887F809391008091910056
:108E9000862B8093910008958091A100887F809314
:108EA000A1008091A100862B8093A100089580915C
:108EB0002101887F8093210180912101862B80935D
:108EC00021010895CF93DF93EC0180919804809362
:108ED000790484E50E949725811102C080E041C099
:108EE0000E948A25809379048823C1F3EEE3F6E09B
:108EF0008491882341F09091C00095FFFCCF80932E
:108F0000C6003196F5CFECE3F6E08491882341F07A
:108F10009091C00095FFFCCF8093C6003196F5CFAD
:108F20004AE050E0BE0182EB98E00E948652EAE2FD
:108F3000F6E08491882341F09091C00095FFFCCF2A
:108F40008093C6003196F5CF40E050E060917904FF
:108F500082EB98E00E94BD5282EB98E00E94725230
:108F600081E0DF91CF910895CF92DF92EF92FF924F
:108F70000F931F93CF93DF938CE590E0A3DF8111D4
:108F800041C0C3EFEC2EC3E0FC2E07E31BE1C0E0C1
:108F9000D0E0F70181917F010E9497258823C1F0DD
:108FA000C33079F4809179046E01C80ED11C0E94FF
:108FB0005925F601EE0FFF1FEE0FFF1FE95CF44E7F
:108FC00003C00E945925F8016083718382839383D3
:108FD00021960C5F1F4FC430D105D9F60E94AEA177
:108FE00025E936E041E956E06DE876E089E896E06B
:108FF000DF91CF911F910F91FF90EF90DF90CF9075
:109000000C941096DF91CF911F910F91FF90EF90EC
:10901000DF90CF90089588E690E054DF811117C06B
:109020008091410283FD13C090917904809198044E
:1090300098130DC083E50E949725882341F00E9474
:1090400059250E9417D670936C1F60936B1F08956B
:109050008DE690E037DF811125C08091410283FDCC
:1090600021C0909179048091980498131BC060E00E
:109070008AED99E00E94E56B83E50E949725809335
:109080000E02811106C082E50E949725811101C060
:1090900081CD0E9459250E9417D670936C1F609352
:1090A0006B1FF6CF0895CF92DF92EF92FF920F934E
:1090B0001F93CF93DF938BEC90E004DF81112DC0E1
:1090C00033EFE32E33E0F32E07E41BE1C0E0D0E002
:1090D000F70181917F010E9497258823C1F0C33059
:1090E00079F4809179046E01C80ED11C0E94592533
:1090F000F601EE0FFF1FEE0FFF1FE95BF44E03C0FA
:109100000E945925F801608371838283938321969D
:109110000C5F1F4FC430D105D9F6DF91CF911F915D
:109120000F91FF90EF90DF90CF900895CF93DF9352
:109130008CEC90E0C7DE811102C183E50E94972587
:10914000882309F43EC00E94592560931F1B709329
:10915000201B8093211B9093221B6093171B7093FD
:10916000181B8093191B90931A1BE8E0F8E0849178
:10917000882341F09091C00095FFFCCF8093C600FA
:109180003196F5CFE0EEF7E08491882341F090919D
:10919000C00095FFFCCF8093C6003196F5CF40917B
:1091A0001F1B5091201B6091211B7091221B22E0FC
:1091B00030E082EB98E00E94515382EB98E00E94ED
:1091C000725280E50E9497258823B1F10E945925AB
:1091D00060931F1B7093201B8093211B9093221B75
:1091E000E9EDF7E08491882341F09091C00095FF6C
:1091F000FCCF8093C6003196F5CFECEBF7E084917D
:10920000882341F09091C00095FFFCCF8093C60069
:109210003196F5CF40911F1B5091201B6091211B6F
:109220007091221B22E030E082EB98E00E945153C3
:1092300082EB98E00E94725282E50E949725882373
:1092400009F440C0C0917904D0E00E945925FE0184
:10925000EE0FFF1FEE0FFF1FE55EF44E608371837C
:1092600082839383E5EBF7E08491882341F090912A
:10927000C00095FFFCCF8093C6003196F5CFE6E99C
:10928000F7E08491882341F09091C00095FFFCCFD6
:109290008093C6003196F5CFE091790484E0E89F91
:1092A000F0011124E55EF44E4081518162817381A9
:1092B00022E030E082EB98E00E94515382EB98E08C
:1092C0000E94725286E50E9497258823C1F10E9470
:1092D00059256093171B7093181B8093191B90934B
:1092E0001A1BEFE8F7E08491882341F09091C000C9
:1092F00095FFFCCF8093C6003196F5CFE1E7F7E00C
:109300008491882341F09091C00095FFFCCF809319
:10931000C6003196F5CF4091171B5091181B6091F4
:10932000191B70911A1B22E030E082EB98E00E943A
:10933000515382EB98E0DF91CF910C947252DF9100
:10934000CF910895CF93DF938DEC90E0BBDD811139
:1093500062C083E50E949725882351F00E94592519
:109360006093231B7093241B8093251B9093261BD3
:1093700086E50E949725882351F00E945925609325
:10938000071B7093081B8093091B90930A1B82E4B0
:109390000E949725882361F00E9459250E941CD6BF
:1093A0006093571B7093581B8093591B90935A1BC3
:1093B00088E50E949725882351F00E9459256093E3
:1093C000131B7093141B8093151B9093161B8AE537
:1093D0000E949725882351F00E94592560930F1B06
:1093E0007093101B8093111B9093121B85E40E94B5
:1093F0009725882381F0C0917904D0E00E945925F7
:10940000FE01EE0FFF1FEE0FFF1FE55FF44E6083BE
:10941000718382839383DF91CF910895CF93DF93FC
:10942000EC01809198048093790488E40E94972548
:10943000811102C080E041C00E948A258093790496
:109440008823C1F3E2E2F6E08491882341F0909111
:10945000C00095FFFCCF8093C6003196F5CFE0E2C7
:10946000F6E08491882341F09091C00095FFFCCFF5
:109470008093C6003196F5CF4AE050E0BE0182EB02
:1094800098E00E948652E0E1F6E08491882341F062
:109490009091C00095FFFCCF8093C6003196F5CF28
:1094A00040E050E06091790482EB98E00E94BD5268
:1094B00082EB98E00E94725281E0DF91CF91089593
:1094C000CF93DF938AED90E0A9DF8111AFC088E5EB
:1094D0000E949725882381F0C0917904D0E00E94F2
:1094E0005925FE01EE0FFF1FEE0FFF1FEB55FB4F3F
:1094F000608371838283938389E50E949725882303
:1095000081F0C0917904D0E00E945925FE01EE0F50
:10951000FF1FEE0FFF1FE755FB4F608371838283B0
:1095200093838AE50E949725882381F0C09179046E
:10953000D0E00E945925FE01EE0FFF1FEE0FFF1F26
:10954000E355FB4F6083718382839383EAE6F7E000
:109550008491882341F09091C00095FFFCCF8093C7
:10956000C6003196F5CFEAE5F7E08491882341F013
:109570009091C00095FFFCCF8093C6003196F5CF47
:10958000E8E5F7E08491882341F09091C00095FFD1
:10959000FCCF8093C6003196F5CF4091A504509141
:1095A000A6046091A7047091A80422E030E082EB49
:1095B00098E00E945153E6E5F7E08491882341F05A
:1095C0009091C00095FFFCCF8093C6003196F5CFF7
:1095D0004091A9045091AA046091AB047091AC042D
:1095E00022E030E082EB98E00E945153E4E5F7E09E
:1095F0008491882341F09091C00095FFFCCF809327
:10960000C6003196F5CF4091AD045091AE04609103
:10961000AF047091B00422E030E082EB98E00E9449
:10962000515382EB98E0DF91CF915CC7DF91CF91EE
:109630000895CF92DF92EF92FF926B017C018091AF
:10964000BD04882331F120E030E0A901C701B60153
:109650000E94A8D58823E9F020E030E040E05FE3F5
:10966000C701B6010E947DD86B017C012BED3FE064
:1096700049E450E40E947DD8A70196010E947DD85C
:109680009B01AC0160E070E080E89FE30E94AFD5F1
:1096900004C060E070E080E89FE3FF90EF90DF900F
:1096A000CF90089560912302709124028091250249
:1096B00090912602BEDF60931F0270932002809378
:1096C0002102909322020895CF92DF92EF92FF92AF
:1096D000CF9388EC90E0F6DB811194C084E40E9483
:1096E00097258823D9F00E9459256B017C01C1E0A0
:1096F00020E030E0A9010E94A8D5811101C0C0E09E
:10970000C093BD04E091790484E0E89FF001112446
:10971000ED5DFD4FC082D182E282F38283E50E943B
:109720009725882379F00E94592520E030E0A9018F
:109730000E94A8D5882321F081E08093BD0402C057
:109740001092BD048091BD04811103C0E3E2F8E0F2
:1097500040C0EDE3F8E08491882341F09091C0008F
:1097600095FFFCCF8093C6003196F5CFEAE2F8E092
:109770008491882341F09091C00095FFFCCF8093A5
:10978000C6003196F5CF82EB98E0ACD620E030E011
:10979000A901609123027091240280912502909189
:1097A00026020E94A8D5811127C080E090E0A0EE9B
:1097B000BFE38093230290932402A0932502B093E9
:1097C00026021AC09091C00095FFFCCF8093C6007E
:1097D000319684918111F6CFEFE0F8E084918823EF
:1097E00041F09091C00095FFFCCF8093C600319668
:1097F000F5CF82EB98E076D6CF91FF90EF90DF9097
:10980000CF9050CFCF91FF90EF90DF90CF90089501
:109810000F931F93CF93DF93209148063091490611
:1098200040E6429FC001439F900D11248C539B4FF3
:1098300090934D0680934C068091410280FF1EC09C
:10984000E0E8FCE08491882341F09091C00095FF0E
:10985000FCCF8093C6003196F5CFE0914C06F09195
:109860004D068191882339F09091C00095FFFCCF7F
:109870008093C600F6CF82EB98E034D680914C06F8
:1098800090914D06FC01208101962032D9F3F0938E
:109890004D06E0934C062F7D2E3461F0C0914C06AE
:1098A000D0914D066AE270E0CE010E9431DE009751
:1098B000D1F420C0818190ED980F9A3010F08D3254
:1098C00069F73296DF0131962C9120532A30D0F37C
:1098D000CD01FC01019620812032D9F3F0934D0691
:1098E000E0934C06DBCFFC0131968291803251F03F
:1098F0008A3241F01881898180538A3008F0CBC3C5
:109900009E0102C01082F1CFF9012F5F3F4F4081CD
:109910004F7DD1F7CF01FC01019620812032D9F390
:10992000F0934B06E0934A06D0938D04C0938C04C9
:109930000E948A25143509F492C334F4173469F06F
:109940001D3409F454C0A7C31D3609F450C01437A0
:1099500009F485C3173609F09EC387309105A9F134
:1099600094F4843091054CF48230910534F597FDE0
:1099700078C381700E94183574C3049709F071C3CD
:109980000E9483406EC38D33910539F14CF48C31C4
:109990009105F1F0CC9709F064C30E945C2B61C380
:1099A0008B359105E9F08C359105F1F08A359105FB
:1099B00009F057C31092920454C321E0029709F0B2
:1099C00020E0822F0E94C23B4CC30E94A43549C3B1
:1099D0000E94D5400E949C2E44C30E94E33641C39E
:1099E00081E0809392043DC30E943B2C3AC38D36A4
:1099F000910509F420C20CF09DC08B31910509F44A
:109A000078C10CF04EC08231910509F4BFC11CF53C
:109A10008430910509F43BC164F497FD22C3823080
:109A200091050CF431C1039709F01BC30E940D3856
:109A300018C38B30910509F42DC18131910509F4CA
:109A40002CC1059709F00DC3109247090E94936C31
:109A50000E940E3506C38731910509F430C164F4C4
:109A60008531910509F421C10CF024C1449709F016
:109A7000F8C20E94CC2CF5C28931910509F429C1A4
:109A80000CF02CC18EE996E00E94F8BA0E94FACF41
:109A900060937E0470937F0480938004909381048C
:109AA000E0C28335910509F46DC124F5803291053A
:109AB00009F43AC19CF48E31910509F41FC10CF0F0
:109AC00030C14C9709F0CDC260914A0670914B06A7
:109AD00040E08EE996E00E9479BCC3C281359105D1
:109AE00009F434C10CF04BC18A9709F0BAC20E9444
:109AF000632DB7C28836910509F464C164F48535D5
:109B0000910509F446C10CF441C18C35910509F069
:109B1000A8C22ADAA6C28A36910509F470C10CF4EB
:109B200053C18B36910509F09CC210929504109296
:109B3000940497C28E3C910509F4E6C10CF049C02B
:109B40008937910509F492C134F58337910509F4F9
:109B500098C07CF48037910509F46FC18237910574
:109B600009F46FC18F36910509F07BC20E94082E5F
:109B700078C28737910509F472C10CF073C185373B
:109B8000910509F06EC260E080914A0690914B0603
:109B90000E94F66866C2893C910509F496C16CF48E
:109BA0008C38910509F47CC1883C910509F48BC17E
:109BB0008A37910509F055C25DC18C3C910509F4C5
:109BC0009FC10CF09FC18B3C910509F04AC26BDA32
:109BD00048C28F3221E0920709F417C20CF58E3D7E
:109BE000910509F4D1C164F48C3D910509F4A3C138
:109BF0000CF0B0C18A3D910509F033C261DC31C27D
:109C00008C32F1E09F0709F4D9C18D3221E092072F
:109C100009F4F8C1823E910509F023C2B4D821C2EB
:109C2000853FE1E09E0709F4F9C18CF48A3921E00F
:109C3000920709F4EDC18C3AE1E09E0709F4EBC10B
:109C40008039914009F00DC20E94AEA10AC2873F3F
:109C500021E0920709F4EBC10CF4E6C18938F2E087
:109C60009F0709F4F9C1873E934009F0FAC181E0EA
:109C70008093420210929D060E94086C0E9453330A
:109C8000F0C1ECE7F8E0E7C00E942445EAC10E9479
:109C90000D38E7C10E948B2CE4C160E08CE29AE0B1
:109CA0000E94E56B0E9406A2DCC18EE996E00E944C
:109CB000F0BAD7C18EE996E00E94F1BAD2C16091A4
:109CC0004A0670914B0640E08EE996E00E9475BB13
:109CD000C8C18EE996E00E9402BBC3C18091FD0617
:109CE000882309F4BEC183E50E9497258111BFC175
:109CF000B8C18EE996E00E9429BCB3C18091FD06EF
:109D0000882309F4AEC160E08EE996E00E943FBF6F
:109D100060914A0670914B068EE996E00E9400BD64
:109D2000A0C10E94F22C9DC18091FD06882309F4F8
:109D300098C160914A0670914B068EE996E00E94A8
:109D400097BD8EE996E00E94F0BA8BC10E946FC366
:109D50000E94AEA1129A0E942DA210929504109218
:109D6000940468EE73E080E090E00E945E4060E062
:109D700089EE99E00E94E56B0E94936C72C110928B
:109D8000C3046FC181E08093C3046BC10E94A52D01
:109D900068C183E50E949725882309F462C10E9467
:109DA000592520E030E04AE754E40E947DD80E9423
:109DB0001CD66093820470938304809384049093F0
:109DC00085044FC128D94DC189E690E07BD8811127
:109DD00065C1E5EEF9E08491882341F09091C000DF
:109DE00095FFFCCF8093C6003196F5CF0E94CF2916
:109DF00082EB98E0DF91CF911F910F9173C383E5C0
:109E00000E949725811103C08FEF90E00FC00E9440
:109E10008A2597FD09C00E948A258F3F910509F088
:109E20009CF70E948A2502C080E090E09093950400
:109E30008093940416C10CD914C188E599E00E945E
:109E4000813C0E949C2E0DC19091C00095FFFCCFDB
:109E50008093C600319684918111F6CF02C10E9491
:109E6000742FFFC081E00E940D98FBC080E00E942B
:109E70000D98F7C083E50E949725882309F4F1C067
:109E80000E94592520E030E0A9010E94A8D5811147
:109E900003C010920D02E5C081E080930D02E1C085
:109EA0008091410283FDDDC083E50E9497258823D0
:109EB00009F4D7C00E9459250E9417D670936A1FD3
:109EC0006093691FCEC000DCCCC0C3EFD3E007E2D3
:109ED0001BE189910E949725882349F00E9459250A
:109EE0000E941CD6F80160837183828393830C5F88
:109EF0001F4FF3E0C73FDF0761F70E940697B1C02D
:109F000015D9AFC01FDAADC0C3EFD3E001EB14E049
:109F100089910E949725882339F00E945925F801DC
:109F200060837183828393830C5F1F4FF3E0C63F8E
:109F3000DF0771F796C083E50E949725882309F40F
:109F400090C00E9459250E9417D670932C026093EE
:109F50002B0287C08DED90E00E946247811181C085
:109F600083E50E949725882309F47BC0C09179047A
:109F7000D0E00E945925CC0FDD1FC75DDD4F0E9448
:109F800017D6798368836DC08EED90E00E9462479A
:109F9000811167C083E50E949725882309F461C079
:109FA000C0917904D0E00E945925CC0FDD1FC95D16
:109FB000DD4F0E9417D67983688353C083E50E94E2
:109FC0009725882321F00E948A25EC0102C0C4E66F
:109FD000D0E080E50E949725882369F00E947F25C4
:109FE000693823E172078105910548F068E873E15B
:109FF00080E090E004C068EE73E080E090E0AE01A5
:10A0000002D62FC00E94FE2F2CC00E94E63029C02D
:10A010000E942FA226C00E941F3123C00E948219D5
:10A0200080E00E94EB1C1DC00E9482191AC083E5CB
:10A030000E949725882361F00E945925C1E020E005
:10A0400030E0A9010E94A8D58111C0E08C2F01C089
:10A0500080E00E94EB1C05C00E94493202C00E94B1
:10A06000F432DF91CF911F910F910C94BC330E9479
:10A070008A25AC01662757FD6095762F409303072C
:10A080005093040760930507709306078EED96E0E2
:10A090000E9497AAE6CF0E94302BE3CFDF91CF91A9
:10A0A0001F910F910895CF93DF9380914406909173
:10A0B0004506039714F40E94B83C60E08EE996E0F0
:10A0C0000E9455BF8091440690914506892B09F462
:10A0D00049C08091FB06882371F1809148069091D8
:10A0E000490620E6289FE001299FD00D1124CC537A
:10A0F000DB4F6EE27EE0CE010E94F0DD892B29F07D
:10A100008EE996E00E9469BD17C0BE018EE996E017
:10A110000E9409BBEAE2FEE08491882341F090911D
:10A12000C00095FFFCCF8093C6003196F5CF82EB3F
:10A1300098E0D8D101C06CDB80914406909145062F
:10A14000019790934506809344068091480690912C
:10A150004906019664E070E00E9473D99093490625
:10A16000809348060E94519780E0DF91CF910C9434
:10A170004F408EE996E00C945BB9CF93C4B7C0FF13
:10A1800010C0E8E5FFE08491882341F09091C00081
:10A1900095FFFCCF8093C6003196F5CF82EB98E017
:10A1A000A1D1C1FF10C0E9E4FFE08491882341F010
:10A1B0009091C00095FFFCCF8093C6003196F5CFFB
:10A1C00082EB98E08FD1C2FF10C0E9E3FFE08491F9
:10A1D000882341F09091C00095FFFCCF8093C6008A
:10A1E0003196F5CF82EB98E07DD1C3FF10C0EAE253
:10A1F000FFE08491882341F09091C00095FFFCCF4F
:10A200008093C6003196F5CF82EB98E06BD1C5FF05
:10A2100010C0EBE1FFE08491882341F09091C000F1
:10A2200095FFFCCF8093C6003196F5CF82EB98E086
:10A2300059D114BECF9108951F93CF93DF931FB7C9
:10A24000F89484E090E00E94F9D9EC010E9491DA40
:10A250008DB79EB71FBF8C1B9D0BDF91CF911F91B8
:10A2600008951F920F920FB60F9211240BB60F9202
:10A270002F933F934F935F936F938F939F93EF939E
:10A28000FF936091C6002091330930913409C901D0
:10A2900001968F7799274091350950913609841797
:10A2A000950741F0F901ED54F74F6083909334091D
:10A2B00080933309FF91EF919F918F916F915F91FF
:10A2C0004F913F912F910F900BBE0F900FBE0F90AB
:10A2D0001F9018959A01AB01211581EE38074105B1
:10A2E000510549F182E08093C00060E079E08DE3A0
:10A2F00090E00E94A8D92150310941095109CA01B1
:10A30000B90122E030E040E050E00E94A8D930934B
:10A31000C5002093C4008091C10080618093C1007A
:10A320008091C10088608093C1008091C1008068E5
:10A330008093C10008951092C00020E130E0E7CF83
:10A340002091350930913609809133099091340973
:10A350008217930771F0F901ED54F74F80812F5F59
:10A360003F4F2F773327309336092093350990E0FC
:10A3700008958FEF9FEF08958091350990913609E8
:10A38000909334098093330908954F925F926F92AE
:10A390007F928F929F92AF92BF92CF92DF92EF9275
:10A3A000FF920F931F93CF93DF93CDB7DEB7A097A4
:10A3B0000FB6F894DEBF0FBECDBF5C01411551054D
:10A3C00061057105E9F420E030E040E350E060E031
:10A3D00070E0A0960FB6F894DEBF0FBECDBFDF9140
:10A3E000CF911F910F91FF90EF90DF90CF90BF9092
:10A3F000AF909F908F907F906F905F904F905BC0D9
:10A400008E010F5F1F4FC12CD12C76014801422EC7
:10A41000512C612C712C8FEFC81AD80AE80AF80A5F
:10A42000CB01BA01A30192010E9486D9CA01F801A9
:10A4300061938F01A901BC014115510561057105A9
:10A4400051F7F1E0CF1AD108E108F108F401EC0D61
:10A45000FD1D80818A3010F440E301C047E3480FBE
:10A46000552747FD5095652F752F20E030E0C50139
:10A4700022D081E0C81AD108E108F108EFEFCE162A
:10A48000DE06EE06FE0611F7A0960FB6F894DEBFC4
:10A490000FBECDBFDF91CF911F910F91FF90EF9035
:10A4A000DF90CF90BF90AF909F908F907F906F90F4
:10A4B0005F904F9008952115310539F48091C000C7
:10A4C00085FFFCCF4093C60008952A30310509F47A
:10A4D00024C05BCF9A01462F552747FD5095652F25
:10A4E000752FE9CFCF93DF93EC0120E030E04DE012
:10A4F00050E060E070E0DFDF20E030E04AE050E074
:10A5000060E070E0CE01DF91CF91D5CF9A01AB0131
:10A51000662757FD6095762FCECFCF92DF92EF92D0
:10A52000FF92CF93DF93EC016A017B0177FF0FC0AD
:10A5300020E030E04DE250E060E070E0BCDFF094FD
:10A54000E094D094C094C11CD11CE11CF11C2AE001
:10A55000B701A601CE01DF91CF91FF90EF90DF9080
:10A56000CF9013CF2115310539F48091C00085FFBC
:10A57000FCCF4093C600089508CF9A01462F50E0C3
:10A5800060E070E0EFCF9A01AB0160E070E0EACFED
:10A590008F929F92AF92BF92CF92DF92EF92FF92F3
:10A5A0001F93CF93DF93EC016A017B01122F20E010
:10A5B00030E0A901C701B6010E94A8D587FF0CC0F1
:10A5C00020E030E04DE250E060E070E0CE0173DF6B
:10A5D000F7FAF094F7F8F094B12C60E070E080E0C6
:10A5E0009FE3B11641F020E030E040E251E40E94E8
:10A5F000AFD5B394F6CF9B01AC01C701B6010E9461
:10A60000CFD46B017C010E941CD64B015C010E94DF
:10A6100048D69B01AC01C701B6010E94CED46B01A4
:10A620007C012AE0B501A401CE01AFDE112341F087
:10A6300020E030E04EE250E060E070E0CE013BDF31
:10A64000112319F120E030E040E251E4C701B601E6
:10A650000E947DD86B017C010E9417D64B01AA2471
:10A6600097FCA094BA2CB501A401CE0156DFC50118
:10A67000B4010E944AD69B01AC01C701B6010E94F9
:10A68000CED46B017C011150DBCFDF91CF911F91B4
:10A69000FF90EF90DF90CF90BF90AF909F908F9002
:10A6A000089576CFDC01FB0120813181220F331F19
:10A6B000220F331F428153814073552794E05595F3
:10A6C00047959A95E1F7240F351F11963C932E93E9
:10A6D0002281338144E0220F331F4A95E1F733276B
:10A6E000448155814C735527559547955595479508
:10A6F000240F351F13963C932E9312972481358196
:10A7000076E0220F331F7A95E1F733278681978110
:10A71000280F391F15963C932E93149708959FEB9D
:10A72000980F9A3130F4992787FD909581549109BB
:10A7300008959FE9980F9A3130F4992787FD9095F5
:10A7400087549109089590ED980F9A3028F499272D
:10A7500087FD9095049608958B3229F08F3231F45D
:10A760008FE390E008958EE390E008958FEF9FEFE0
:10A7700008956F927F928F929F92AF92BF92CF92E5
:10A78000DF92EF92FF920F931F93CF93DF93CDB79A
:10A79000DEB72E970FB6F894DEBF0FBECDBF6C01AB
:10A7A0005A017B01A60EB71E00E010E080E090E0A9
:10A7B0004E0129E0820E911CEA14FB0429F0F701F6
:10A7C00041917F014D3389F478015C01009709F4D0
:10A7D0008BC0AC01440F551F21E030E02C0F3D1F12
:10A7E000420F531F20E030E041C09C012F5F3F4FDC
:10A7F000FC01EE0FFF1F81E090E08C0F9D1FE80F22
:10A80000F91F842F992787FD9095918380832430A9
:10A81000310551F5FE0131963F01F30180817FDF63
:10A82000F301819391933F01E815F905B1F7BE015A
:10A830006F5F7F4FC40136DFF401C801880F991F95
:10A840008C0D9D1D20E030E041915191DC01A20F63
:10A85000B31F4D935C932E5F3F4F26303105A1F718
:10A860000D5F1F4F20E030E0C901A6CF8430910575
:10A870004CF4FA01E20FF31F1182108201962E5F51
:10A880003F4FF4CFCE0101964C013E0199E0690E95
:10A89000711CF401808143DFF401819391934F0196
:10A8A000E615F705B1F7BE016F5F7F4FCF01FADE06
:10A8B000D4019801220F331F2C0D3D1D80E090E044
:10A8C000F1E0AF1AB1088C010E0D1F1D8A159B0512
:10A8D0005CF44D915D91FC01EE0FFF1FE20FF31F41
:10A8E000518340830196EFCFF801EE0FFF1FEC0D6F
:10A8F000FD1D11821082C8012E960FB6F894DEBF9E
:10A900000FBECDBFDF91CF911F910F91FF90EF90C0
:10A91000DF90CF90BF90AF909F908F907F906F907F
:10A920000895CF93C82F61E00E94E5D161E070E007
:10A930008C2F0E94CDD0E1EAF0E0108282E8809373
:10A94000A00080E491E09093A7008093A6008FE39D
:10A9500091E09093A9008093A80089E18083F89406
:10A960008081887F808380E491E09093A50080932C
:10A97000A4009093A7008093A600808181608083CB
:10A980007894CF910895CF93DF93EC0181E0809389
:10A9900048090E9406D060934A0970934B0980933E
:10A9A0004C0990934D09BE01882777FD8095982F1B
:10A9B0000E944AD620E030E44CE156E40E94ABD736
:10A9C00018162CF0D7FF05C0C0E0D0E002C0C0E1EF
:10A9D000D7E261E085E00E94E5D1BE01882777FDDE
:10A9E0008095982F0E944AD620E030E44CE156E44E
:10A9F0000E94AFD520E030E040EA53E40E947DD8C9
:10AA00000E9417D697FF07C0909580957095619525
:10AA10007F4F8F4F9F4F86E00E94CDD060E085E052
:10AA20000E941ED280914E098823F9F0E6E8FFE0EB
:10AA30008491882341F09091C00095FFFCCF8093D2
:10AA4000C6003196F5CFEAE7FFE08491882341F014
:10AA50009091C00095FFFCCF8093C6003196F5CF52
:10AA600082EB98E0DF91CF913DCDDF91CF910895BA
:10AA70008F929F92AF92BF92CF92DF92EF92FF920E
:10AA800080914809882309F453C01092480961E075
:10AA900085E00E941ED20E94FACF4B015C01C0905B
:10AAA0004F09D0905009E12CF12C60914A09709126
:10AAB0004B0980914C0990914D0928EE33E040E01C
:10AAC00050E00E9486D9C21AD30AE40AF50AC80CDB
:10AAD000D91CEA1CFB1CD0925009C0924F098091EE
:10AAE0004E09882329F1E3E7FFE08491882341F0B0
:10AAF0009091C00095FFFCCF8093C6003196F5CFB2
:10AB0000E0E6FFE08491882341F09091C00095FF3A
:10AB1000FCCF8093C6003196F5CF82EB98E0FF9092
:10AB2000EF90DF90CF90BF90AF909F908F90DACC56
:10AB3000FF90EF90DF90CF90BF90AF909F908F905D
:10AB4000089586E090E0EDDE61E085E00E941ED28F
:10AB500061E085E00E94E5D184E690E090933A09B7
:10AB60008093390910923B0910923C0910923D09DB
:10AB700010923E0910923F0910924009109241092B
:10AB800010924209109247091092480910924909FF
:10AB900010924A0910924B0910924C0910924D09DB
:10ABA00010924E091092500910924F0980E090E0E7
:10ABB000A0E8BFE38093DD099093DE09A093DF094D
:10ABC000B093E0098DEC9CECACE4BEE38093E1092A
:10ABD0009093E209A093E309B093E40981E08093A4
:10ABE000E90946CF8130910541F08230910539F075
:10ABF000892B41F410924909089581E001C082E057
:10AC00008093490908958F929F92AF92BF92CF92FD
:10AC1000DF92EF92FF920F931F93CF93DF9300D0B9
:10AC20001F92CDB7DEB76B017C014115510591F143
:10AC3000389A4A01A12CB12C60E271EA87E090E0D9
:10AC4000A50194010E94A8D98901A7019601C50117
:10AC5000B4010E9443D928EE33E040E050E00E9466
:10AC6000A8D9E12CF12CE216F30641F1409AC80173
:10AC700029833A834B835C830E9460D04098C8014B
:10AC80000E9460D08FEFE81AF80A5C814B813A810C
:10AC90002981E9CF882799270F900F900F900F9067
:10ACA000DF91CF911F910F91FF90EF90DF90CF90A8
:10ACB000BF90AF909F908F900C9429D00F900F90E1
:10ACC0000F900F90DF91CF911F910F91FF90EF9018
:10ACD000DF90CF90BF90AF909F908F90089598E0B5
:10ACE0000BC0F894209102012E7F209302013FBFF8
:10ACF000880F119A915079F011983FB787FFF1CFE3
:10AD0000F894209102012160209302013FBF880F37
:10AD1000119A915089F7089508958F929F92AF925A
:10AD2000BF92CF92DF92EF92FF920F931F93CF9338
:10AD3000DF93EB0147015801609144027091450295
:10AD400070930F0A60930E0A6091180A7091190AA5
:10AD500070930D0A60930C0A62E06093430260EE08
:10AD60007AE7709345026093440290930B0A8093B4
:10AD70000A0AD093090AC093080ACA01B9010E94BD
:10AD800017D66093040A7093050A8093060A90937D
:10AD9000070A0E944AD66B017C019B01AC01C501E8
:10ADA000B4010E94CED40E9417D66093000A70931B
:10ADB000010A8093020A9093030AA7019601688111
:10ADC00079818A819B810E94CED40E941CD6609397
:10ADD000180A7093190A80931A0A90931B0ADF913C
:10ADE000CF911F910F91FF90EF90DF90CF90BF9088
:10ADF000AF909F908F9008954F925F926F927F9245
:10AE00008F929F92AF92BF92CF92DF92EF92FF927A
:10AE10000F931F93CF93DF93EB0129013A01470171
:10AE20005801209144023091450230930F0A20933B
:10AE30000E0A2091180A3091190A30930D0A2093B6
:10AE40000C0A22E02093430225E937E830934502BB
:10AE50002093440290930B0A80930A0A7093090A84
:10AE60006093080A20E030E048EC52E4C301B201EC
:10AE70000E947DD80E9417D66093040A7093050A39
:10AE80008093060A9093070A0E944AD66B017C01C0
:10AE900020E030E048EC52E4C501B4010E947DD8C6
:10AEA000A70196010E94CED40E9417D66093000A93
:10AEB0007093010A8093020A9093030A20E030E025
:10AEC00048EC52E4688179818A819B810E947DD817
:10AED000A70196010E94CED40E941CD66093180A46
:10AEE0007093190A80931A0A90931B0ADF91CF91ED
:10AEF0001F910F91FF90EF90DF90CF90BF90AF9098
:10AF00009F908F907F906F905F904F900895CF9318
:10AF1000DF93EC01262F4CAD6BAD04960E9497CBCE
:10AF20002BAD992787FD9095820F911D8BAF81E006
:10AF300090E0DF91CF9108956F927F928F929F92D0
:10AF4000AF92BF92CF92DF92EF92FF920F931F9337
:10AF5000CF93DF935C017B01942E69018AE048174F
:10AF600009F478C0A5E14A1350C0DB011296ED91B7
:10AF7000FC9113978280C681D7819FB7F894809106
:10AF800002018260809302019FBF0E9461CA80EE2D
:10AF9000782E780C90E2692E680C88EFA0DE0E9473
:10AFA00061CABFE1B81508F444C0882D8077806875
:10AFB00096DE882D8295807F92DE0E9461CA80E8AD
:10AFC0008EDE80E08CDE0E9461CA8AEF88DE0E94FD
:10AFD00061CA8E01005F1F4F8881807F80DE89916A
:10AFE0008295807F7CDE0C171D07B1F7E8010E9477
:10AFF00061CA839473948610D0CF9FB7F8948091E0
:10B0000002018D7F809302019FBF9601492DB701F8
:10B01000C501DF91CF911F910F91FF90EF90DF90CD
:10B02000CF90BF90AF909F908F907F906F900C9437
:10B0300087CE872D8077806852DE872D8295807F2E
:10B040004EDE0E9461CA80E84ADE80E848DE0E9447
:10B0500061CABBCF809101018260809301019FB7DB
:10B06000F894809102018D7F809302019FBF8091AF
:10B0700001018160809301019FB7F89480910201E2
:10B080008E7F809302019FBF099A119A9FB7F8940F
:10B09000809102018260809302019FBF0E9461CA79
:10B0A00088E790E00E9457CA88EF19DE0E9461CAC3
:10B0B00080E015DE80E813DE0E9461CA80E00FDECA
:10B0C00080E10DDE0E9461CA8FE090E00E9457CAC5
:10B0D00080E305DE80EE03DE0E9461CAD0E08D2FA2
:10B0E00080778068FCDD8D2F8295807FF8DD0E945F
:10B0F00061CA80E8F4DD80E0F2DD0E9461CA8AEF77
:10B10000EEDD0E9461CAC0E280E0E9DD80E0E7DDBB
:10B110000E9461CAC150C1F788EFE1DD0E9461CA97
:10B12000DF5FD032E1F680E0DADD80ECD8DD0E942E
:10B1300061CA63CFEDE4F2E19491992361F0EDE40B
:10B14000F2E18091C00085FFFCCF9093C60031965C
:10B1500094919111F6CF82EB98E0C4D987E492E103
:10B160000E94B9241092790C1092780C80914402BC
:10B1700090914502805F9C4579F080EF9CE590932B
:10B180004502809344021092180A1092190A1092F4
:10B190001A0A10921B0A089508950F931F93CF93D4
:10B1A000C82F8B0189E390E10E94B9248C2F90E095
:10B1B000EADBB801882777FD8095982F0E9429D077
:10B1C000CF911F910F9154CC91E0811101C090E07B
:10B1D000892F089508950895CF92DF92EF92FF92FC
:10B1E000CF93DF93EB01609144027091450270931D
:10B1F0000F0A60930E0A6091180A7091190A7093F1
:10B200000D0A60930C0A62E06093430269E17DE7F6
:10B21000709345026093440290930B0A80930A0A4C
:10B22000D093090AC093080ACA01B9010E9448D6FE
:10B230002AE037ED43E25CE30E947DD80E9417D6F6
:10B240006093040A7093050A8093060A9093070A94
:10B250000E944AD66B017C019B01AC0160E070E862
:10B2600087E794E40E94CED40E9417D66093000A28
:10B270007093010A8093020A9093030A688179818E
:10B280008A819B810E9448D62AE037ED43E25CE345
:10B290000E947DD8A70196010E94CED40E941CD6A0
:10B2A0006093180A7093190A80931A0A90931B0AE4
:10B2B000DF91CF91FF90EF90DF90CF900895CF92E4
:10B2C000DF92EF92FF92CF93DF93EB0169017A0156
:10B2D000209144023091450230930F0A20930E0AC8
:10B2E0002091180A3091190A30930D0A20930C0A04
:10B2F00022E02093430224E53CE73093450220936B
:10B30000440290930B0A80930A0A7093090A60938F
:10B31000080A2AE037ED43E25CE3C701B6010E9468
:10B320007DD80E9417D66093040A7093050A809313
:10B33000060A9093070A0E944AD66B017C019B0182
:10B34000AC0160E070E887E794E40E94CED40E94EC
:10B3500017D66093000A7093010A8093020A9093B3
:10B36000030A2AE037ED43E25CE3688179818A8150
:10B370009B810E947DD8A70196010E94CED40E9495
:10B380001CD66093180A7093190A80931A0A909336
:10B390001B0ADF91CF91FF90EF90DF90CF9008953F
:10B3A000209144023091450230930F0A20930E0AF7
:10B3B0002091180A3091190A30930D0A20930C0A33
:10B3C00022E0209343022DE73EE73093450220938D
:10B3D000440290930B0A80930A0A7093090A6093BF
:10B3E000080A82E390E0A0E0B0E08093040A909322
:10B3F000050AA093060AB093070A84E696E8A1E03E
:10B40000B0E08093000A9093010AA093020AB093DF
:10B41000030A20E030E040E251E4FB0160817181E9
:10B42000828193810E947DD820E030E048E452E49C
:10B430000E94CED40E941CD66093180A7093190AF9
:10B4400080931A0A90931B0A0895BC0180E090E053
:10B450000C9429D09093790C8093780C0895FC017A
:10B460001382128289E294E09183808313AE14AE3A
:10B4700015AECF0104960C9460CDFC0163AF44AFD0
:10B480000895CF93DF93FC0185ADEF0124968111E0
:10B4900005C081E085AFCE010E9450CDCE01DF9185
:10B4A000CF910C946FCD04960C9473CD0F931F9392
:10B4B000CF93DF931F92CDB7DEB7FC0185AD8F012F
:10B4C0000C5F1F4F811107C081E085AFC801698300
:10B4D0000E9450CD6981C8010F90DF91CF911F91DB
:10B4E0000F910C9481CD04960C949DCD04960C94F0
:10B4F00086CD0F9304960E9444CF0F9108950F9329
:10B5000004960E9494CF0F9108950F93CF93C82F64
:10B51000611112C061E087E29AE0E5DF8C2F90E0D4
:10B520000196482F440F480F440F440F60E087E214
:10B530009AE0CF910F91A1CF61E087E29AE0D3DF4B
:10B540004C2F440F4C0F440F440F4D5F0CE020E88C
:10B5500060E087E29AE0D3DF60E087E29AE0C3DF51
:10B56000DDCFEF92FF920F9304960E94FFC90F91D7
:10B57000FF90EF90089504960C943ACC66E675E13E
:10B5800087E29AE0F8DF81E08093230A0895CF9361
:10B59000C82F823091F06CF0833011F0843039F490
:10B5A00066E675E187E29AE0E6DFC093230ACF9171
:10B5B00008958130E1F7CF91E1CF66E87FE187E23E
:10B5C0009AE0D9DFC093230ACF91089504960C9492
:10B5D000B5CBDF92EF92FF920F931F93CF93DF9340
:10B5E0006091250A87E29AE061DF80912B0AF2DD03
:10B5F000C82FD0E0BE016057710977FD56C0759520
:10B600006795D62EEC97D695C79587E29AE039DFF5
:10B6100005C087E29AE047DF8823B1F180914602B6
:10B620008823B9F326E4E22E20E2F22E06E22EE091
:10B6300040E06D2D87E29AE094DF84E0A8DF8091FE
:10B640002B0AC8DD182F80912C0AC5DD4EEE480F5D
:10B6500027EF33E06C2F87E29AE0B8DF80912C0A65
:10B66000BADD4AEF480F212F30E0B9016857710960
:10B670007695679522E034E087E29AE0A7DF87E2DB
:10B680009AE011DF8111CACF80914602882329F008
:10B6900088E893E1DADE10924602DF91CF911F91A4
:10B6A0000F91FF90EF90DF9008956F5F7F4FA7CFCE
:10B6B000CF93DF93EC0167E472E0D1DE81E394E0A5
:10B6C00099838883DF91CF910895CF93C82F8FEF0F
:10B6D0008C0F893040F06C2F87E29AE00E9474D47E
:10B6E00081E0CF91089566E87FE187E29AE043DF49
:10B6F0006C2F87E29AE00E9474D48091230A47DF7E
:10B7000081E0CF910895FF920F931F93CF93DF9322
:10B71000062FEA01F22E682F802FF7DEFE018491BA
:10B72000882351F114E1D1DF181B2196FE01849189
:10B730008111F9CFCFEFC10F111102C007C0C92F7E
:10B7400080E2C3DF9FEF9C0FC111F9CF602F70E043
:10B750006F5F7F4F462F440F460F440F440F6AE739
:10B7600087E29AE08ADE8F2DB0DF80E2DF91CF9111
:10B770001F910F91FF90A9CFC3E1E2CFEF92FF920B
:10B780001F93CF93DF931F92CDB7DEB7982F862FED
:10B79000692F4983BADE4981442311F082E095DFA5
:10B7A00065EBE62E6DE1F62E15E1F70181917F0143
:10B7B000882319F08ADF181BF8CF112321F080E2CB
:10B7C00084DF1150FACF0F90DF91CF911F91FF903E
:10B7D000EF9008951F93CF93DF93EC018881882326
:10B7E00061F0219610E071DF180F89918111FBCF74
:10B7F000812FDF91CF911F91089510E0F9CF8F92A3
:10B800009F92AF92BF92CF92DF92EF92FF920F93EF
:10B810001F93CF93DF93CDB7DEB7EC970FB6F894B5
:10B82000DEBF0FBECDBFC0907504D0907604E0900F
:10B830007704F09078047CE3872E912CA12CB12C16
:10B84000C701B601A50194010E9486D9CA01B901B8
:10B85000A50194010E9486D97F936F93C701B60119
:10B8600020E13EE040E050E00E9486D9CA01B901E3
:10B8700028E130E040E050E00E9486D97F936F934A
:10B88000C701B60120E831E541E050E00E9486D9C9
:10B890003F932F938CEC94E19F938F938E01015EE5
:10B8A0001F4F1F930F930E9466DE4EE065E087E214
:10B8B0009AE0E3DDC8018EDF60917104709172043B
:10B8C00080917304909174040E9417D66B017C01DF
:10B8D0002AE030E040E050E00E94A8D97F936F93C7
:10B8E000CA01B90124E630E040E050E00E94A8D946
:10B8F0007F936F93E8EE8E2EE3E09E2EA12CB12C69
:10B90000C701B601A50194010E94A8D9CA01B901D5
:10B91000A50194010E94A8D97F936F93C701B60136
:10B9200020E432E44FE050E00E94A8D93F932F93E7
:10B9300083EB94E19F938F930E5111091F930F9303
:10B940000E9466DE4AE265E087E29AE096DDC80181
:10B9500041DF8091220A0FB6F894DEBF0FBECDBF43
:10B9600082FF15C08091440290914502895099460A
:10B9700071F089E099E69093450280934402109219
:10B98000180A1092190A10921A0A10921B0AEC96C1
:10B990000FB6F894DEBF0FBECDBFDF91CF911F91E0
:10B9A0000F91FF90EF90DF90CF90BF90AF909F905E
:10B9B0008F9008951F93CF93DF93EC012196FC01A4
:10B9C000849110E0882339F080DE180FFE01849105
:10B9D00021968111F9CF812FDF91CF911F91089589
:10B9E0008091780C9091790C8730910508F008953A
:10B9F000FC01E258FF4F4EE065E087E29AE00C94CC
:10BA0000C4D93BDD80E691E1D5DF4CE165E087E21A
:10BA10009AE033DD8BE491E1CDCF2FDD86E391E138
:10BA2000C9DF4CE165E087E29AE027DD83E291E13E
:10BA3000C1DF88E893E109DD8FE191E10E94B9243B
:10BA400080914402909145028156934681F281E6AD
:10BA500093E690934502809344021092180A109244
:10BA6000190A10921A0A10921B0A089506DD82E341
:10BA700092E1A0DF4CE165E087E29AE0FEDC8DE137
:10BA800092E198CFFADC88E092E194DF4CE165E046
:10BA900087E29AE0F2DC83EF91E18CCFEEDC8EED71
:10BAA00091E188DF4CE165E087E29AE0E6DC89EC31
:10BAB00091E180CFE2DC84EB91E17CDF4CE165E059
:10BAC00087E29AE0DADC8FE991E174CFD6DC8AE88C
:10BAD00091E170DF4CE165E087E29AE0CEDC85E73A
:10BAE00091E168CFDF92EF92FF920F931F93CF9374
:10BAF000DF93E62EEA018901F9019081992309F487
:10BB00004EC0D901119640E050E007C02E2F9F2F64
:10BB1000422F592F9D91992361F0FA013196907C23
:10BB20009038A1F7242F952F422F592F9D919111D5
:10BB3000F4CFB4E1FB2ED22EDD0CD20EDD0CD1946D
:10BB4000F0E8DF0EF21A682F8E2DDFDCFE01849103
:10BB5000882339F0BADDF81A2196FE01849181110B
:10BB6000F9CF8AE3B2DDFF2029F0CF2D80E2ADDDF1
:10BB7000C150E1F7EE2DF0E031964E2F440F4E0FFD
:10BB8000440F440F6D2D87E29AE077DCC801DF9106
:10BB9000CF911F910F91FF90EF90DF901BCEF0E8B7
:10BBA000DF2EA4E1FA2ECFCF8F929F92AF92BF9259
:10BBB000CF92DF92EF92FF921F93CF93DF934C01CE
:10BBC000EB014881442309F490C0FB01319680E0E9
:10BBD00090E004C0C9014191442359F09C012F5FBA
:10BBE0003F4F407C4038B1F79C01C9014191411160
:10BBF000F5CF332764E170E0621B730B85E190E0C1
:10BC0000821B930B182F110F180F110F9401F401C1
:10BC10008491882309F466C0C40140E050E0F90132
:10BC20002491207C203811F04F5F5F4F01969C01DA
:10BC3000FC01A491A111F3CF641775070CF04BC060
:10BC400083E0E82EF12C92E0A92EB12C80912C0AF1
:10BC5000C2DA90E0B7010E9473D9882777FD8095FA
:10BC6000982F0E944AD66B017C0120E030E040EC26
:10BC700050E40E94CFD40E941CD6462F60E087E299
:10BC80009AE0FBDBC40196DE8AE31FDDB50188275D
:10BC900077FD8095982F0E944AD6A70196010E94B1
:10BCA0007DD820E030E040EC50E40E94CFD40E94E8
:10BCB0001CD6462F612F87E29AE0DFDBCE01DF91B1
:10BCC000CF911F91FF90EF90DF90CF90BF90AF90FA
:10BCD0009F908F907FCD22E0E22EF12CAA24A39496
:10BCE000B12CB4CF40E050E0A7CF1EE764E170E094
:10BCF0008DCF84EA9FE00E94B92480914402909104
:10BD000045028C5E954771F08CEE95E79093450265
:10BD1000809344021092180A1092190A10921A0A7B
:10BD200010921B0A08950E946FC3109295041092FE
:10BD3000940480914402909145028C5E954771F085
:10BD40008CEE95E790934502809344021092180A76
:10BD50001092190A10921A0A10921B0A0895AF92B3
:10BD6000CF92EF92FF920F931F9320E030E040E7D5
:10BD700052E40E94AFD5A0909604C09098047B0135
:10BD80008C0125E936E041E956E06DE876E089E886
:10BD900096E00E94A08B1F910F91FF90EF90CF90A3
:10BDA000AF90089582E0809343020E94FACF6C50D6
:10BDB0007E4F8F4F9F4F60931D0A70931E0A809392
:10BDC0001F0A9093200A40ED57E068E770E080E09A
:10BDD00090E00C9403566F927F928F929F92AF9255
:10BDE000BF92CF92DF92EF92FF920F931F93CF9368
:10BDF000DF93CDB7DEB76F970FB6F894DEBF0FBEF7
:10BE0000CDBF80914302811119C08091220A82FD29
:10BE100015C06F960FB6F894DEBF0FBECDBFDF9191
:10BE2000CF911F910F91FF90EF90DF90CF90BF9037
:10BE3000AF909F908F907F906F9008958EE996E0DD
:10BE40000E9427BE8C0110927E0C8091180A90915E
:10BE5000190AA0911A0AB0911B0A813020E89207B2
:10BE6000A105B10508F08AC0782EB090210A7B1494
:10BE700018F47092210AB72C9090220A92FA992411
:10BE800090F8A12C88248394680121E0C21AD1087B
:10BE9000B11051C091E0711090E080914302811186
:10BEA000A4C0911085C065EB7DE186E497E00E9417
:10BEB00062A78091B51D8F3209F495C082E001150B
:10BEC000110589F07B1409F4A2C0760166246394FD
:10BED0006B0C91105DC0B81609F4F2C08F5F21E0C1
:10BEE000E21AF108C0F7781680F090E00197AC01F3
:10BEF000662757FD6095762F4093180A5093190ACC
:10BF000060931A0A70931B0A782E2091210A30E060
:10BF10002C5F3F4F472D50E0241735070CF041C0F0
:10BF20006CEFB62EB70CB092210A80924302A12C7E
:10BF3000BB2009F4AFCF65EB7DE186E497E00E947A
:10BF400062A78091B51D8F3209F44DC0F1E0BF1298
:10BF5000B5CF91E0791290E08091430281114EC0FB
:10BF6000992009F4ABCF992309F4A8CF1BDF8EE900
:10BF700096E00E9413BF1092210A4BCF1092180A2C
:10BF80001092190A10921A0A10921B0A712C6DCF86
:10BF9000B81609F47FC08F5FE1E0EE1AF108C0F730
:10BFA000A2CFA394B394F4E0FA1508F071CF31CF87
:10BFB000992309F478CFF6DE8091440290914502EE
:10BFC0008950994609F425CF89E099E69093450276
:10BFD000809344021092180A1092190A10921A0AB9
:10BFE00010921B0A16CF81E06ACF24E04DEE54E197
:10BFF0006A2D892F9F8F87DB9F8D53CF20E249EEDB
:10C0000054E16A2D892F9F8F7EDB9F8DA9CF9920C8
:10C01000A1F120E030E007C08F5F2F5F3F4F201776
:10C02000310709F460CF8B11F7CFB8016150710966
:10C03000621B730B40E050E08EE996E00E94E1BD88
:10C040008091FE06882309F451C080914302882321
:10C0500021F041E06A2D81E091DBA4DE65EB7DE11A
:10C060008EE996E00E9470BE1092180A1092190A8A
:10C0700010921A0A10921B0ACCCE760166246394A1
:10C08000670CB81609F480C08F5F21E0E21AF1084E
:10C09000C0F729CF40E050E0B7018EE996E00E945A
:10C0A000E1BD8091FE06882309F496C08091430289
:10C0B000882321F041E06A2D80E060DB862D6CCF83
:10C0C00040E050E0B7018EE996E00E94E1BD80912A
:10C0D000FE06882309F476C080914302882309F480
:10C0E00079C041E06A2D80E049DB74C08091430251
:10C0F000882321F040E06A2D81E040DB53DE85EBB0
:10C100009DE19F938F9382EE94E19F938F938E0195
:10C110000F5F1F4F1F930F930E9466DE8D810F905C
:10C120000F900F900F900F900F90882379F07E0161
:10C13000F5E0EF0EF11C992787FD90950E94C1DD77
:10C14000F70181937F0180818111F5CFC8010E94A1
:10C15000F3238EED94E10E94B924809144029091E2
:10C1600045028C5E954709F454CE8CEE95E790938A
:10C170004502809344021092180A1092190A1092F4
:10C180001A0A10921B0A45CE40E050E0B7018EE932
:10C1900096E00E94E1BD8091FE0681110AC0809167
:10C1A0004302882321F040E06A2D81E0E7DA862D02
:10C1B0006CCF809143028823D1F341E06A2D81E066
:10C1C000DDDAF5CF80914302882321F040E06A2D2B
:10C1D00080E0D4DA862D83CE80914302882309F44F
:10C1E0006DCF40E06A2D80E0C9DA68CFAF92BF9290
:10C1F000CF92DF92EF92FF920F931F93CF93DF9333
:10C200001F921F92CDB7DEB710927E0C8091180A54
:10C210009091190AA0911A0AB0911B0A813020E866
:10C220009207A105B10508F0B5C0782FA090210AAA
:10C230007A1518F47093210AA72E0091220A02FBA6
:10C24000002700F910E0BB24B394F7E0CF2ED12CE7
:10C25000E12CF12CA11021C091E0711190E08091AE
:10C260004302811176C0002311F091119DC07830F6
:10C2700040F5472F50E02091210A30E02C5F3F4FDE
:10C28000241735078CF5ECEFAE2EA70EA092210AED
:10C29000B092430210E0AA20F9F2F1E0AF1236C0EA
:10C2A00091E0713009F090E08091430281115CC00F
:10C2B0000023E9F29923D9F275DD62E370E080E2B0
:10C2C0003AC0C092180AD092190AE0921A0AF09263
:10C2D0001B0A47E050E077E02091210A30E02C5F14
:10C2E0003F4F241735077CF21F5FA394153008F4E5
:10C2F000B1CF0F900F90DF91CF911F910F91FF90D1
:10C30000EF90DF90CF90BF90AF90089522E0A212FF
:10C3100063C091E0723009F090E080914302811196
:10C320002EC0002309F4A3CF992309F4A0CF3ADD4E
:10C3300064E670E080E20F900F90DF91CF911F9143
:10C340000F91FF90EF90DF90CF90BF90AF900C9443
:10C35000CD5824E042E950E1612F892F79839A83F7
:10C36000D2D99A8179817FCF20E247E850E1612FCD
:10C37000892F79839A83C7D99A81798199CF20E2CD
:10C380004CE750E1612F892F79839A83BCD99A8138
:10C390007981C7CF1092180A1092190A10921A0ABE
:10C3A00010921B0A70E042CFFDDC80914402909114
:10C3B0004502805C974609F49CCF80EC97E6909309
:10C3C0004502809344021092180A1092190A1092A2
:10C3D0001A0A10921B0A8DCF83E0A8121EC091E0AA
:10C3E000733009F090E08091430281110BC000236B
:10C3F00009F43DCF992309F43ACFD4DC62E370E02D
:10C4000088EE99CF20E241E750E1612F892F7983AF
:10C410009A8379D99A817981EACFE4E0AE1213C088
:10C4200091E0743009F090E080914302811137C0AF
:10C43000002309F41CCF992309F419CFB3DC64E677
:10C4400070E088EE78CFF5E0AF1213C091E0753060
:10C4500009F090E08091430281112CC0002309F47F
:10C4600006CF992309F403CF9DDC62E370E08CEDE5
:10C4700062CF26E0A21234C091E0763009F090E05D
:10C4800080914302811121C0002309F4F0CE992349
:10C4900009F4EDCE87DC64E670E08CED4CCF20E251
:10C4A00046E650E1612F892F79839A832CD99A81AE
:10C4B0007981BECF20E24BE550E1612F892F79834E
:10C4C0009A8321D99A817981C9CF20E240E550E150
:10C4D000612F892F79839A8316D99A817981D4CF54
:10C4E00087E0A812C4CE91E0773009F090E0809107
:10C4F000430281110BC0002309F4B9CE992309F43A
:10C50000B6CE50DC60ED77E08FE015CF20E24DE352
:10C5100050E1612F892F79839A83F5D89A817981A7
:10C52000EACFAF92BF92CF92DF92EF92FF920F933A
:10C530001F93CF93DF9310927E0C8091180A9091F5
:10C54000190AA0911A0AB0911B0A813020E89207BB
:10C55000A105B10508F093C0D82F0091210AD0178A
:10C5600018F4D093210A0D2FB090220AB2FABB24FE
:10C57000B0F8A5E0AA2EA00EC02FB2E0CB2ED12C91
:10C58000E12CF12C19C011E0D11110E0809143028F
:10C59000811163C0BB2011F011117BC0D33048F072
:10C5A000C092180AD092190AE0921A0AF0921B0A55
:10C5B000D2E0CF5FCA1541F16C2F601BCC2319F379
:10C5C000C13069F511E0D13009F010E080914302EB
:10C5D000811149C0BB2011F3112301F3E3DB8091EA
:10C5E00044029091450288519F4771F088E19FE78E
:10C5F00090934502809344021092180A1092190AEF
:10C6000010921A0A10921B0ADF91CF911F910F917D
:10C61000FF90EF90DF90CF90BF90AF900895C23021
:10C6200009F0BCCF11E0D23009F010E08091430254
:10C6300081111FC0BB2009F4B1CF112309F4AECF83
:10C64000B1DBDF91CF911F910F91FF90EF90DF90C1
:10C65000CF90BF90AF900C94821924E04EEA54E141
:10C66000812F51D897CF23E047EA54E1812F4BD84F
:10C67000B1CF20E246E954E1812F45D8DBCF1092BB
:10C68000180A1092190A10921A0A10921B0AD0E086
:10C6900064CF88DB8091440290914502895099468D
:10C6A00009F4B2CF89E099E6909345028093440261
:10C6B0001092180A1092190A10921A0A10921B0A64
:10C6C000A3CFAF92BF92CF92DF92EF92FF920F93E0
:10C6D0001F93CF93DF931F921F92CDB7DEB71092B7
:10C6E0007E0C8091180A9091190AA0911A0AB091B3
:10C6F0001B0A813020E89207A105B10508F0BAC0F5
:10C70000782FA090210A7A1518F47093210AA72E89
:10C710000091220A02FB002700F910E0BB24B39429
:10C7200086E0C82ED12CE12CF12CA11022C091E082
:10C73000711190E080914302811178C0002311F0C3
:10C740009111A2C0773008F046C0472F50E02091E9
:10C75000210A30E02C5F3F4F2417350754F51CEFBA
:10C76000A12EA70EA092210AB092430210E0AA20A7
:10C77000F1F2F1E0AF123BC091E0713009F090E0CE
:10C780008091430281115EC00023E1F29923D1F22E
:10C7900009DB89E193E10F900F90DF91CF911F9119
:10C7A0000F91FF90EF90DF90CF90BF90AF900C94DF
:10C7B000B9241F5FA394153008F4B7CF0F900F90E2
:10C7C000DF91CF911F910F91FF90EF90DF90CF906D
:10C7D000BF90AF900895C092180AD092190AE092C3
:10C7E0001A0AF0921B0A46E050E076E0B0CF22E051
:10C7F000A21262C091E0723009F090E08091430291
:10C8000081112CC0002309F49DCF992309F49ACFFC
:10C81000C9DA0F900F90DF91CF911F910F91FF9088
:10C82000EF90DF90CF90BF90AF9063CA24E041E3D8
:10C8300053E1612F892F79839A830E94835B9A81C8
:10C8400079817CCF20E247E253E1612F892F798300
:10C850009A830E94835B9A81798196CF20E248E097
:10C8600053E1612F892F79839A830E94835B9A8198
:10C870007981C8CF1092180A1092190A10921A0AD8
:10C8800010921B0A70E03DCF8DDA809144029091A6
:10C8900045028950994609F491CF89E099E6909331
:10C8A0004502809344021092180A1092190A1092BD
:10C8B0001A0A10921B0A82CF83E0A81232C091E0BC
:10C8C000733009F090E08091430281111EC0002373
:10C8D00009F438CF992309F435CF64DA8091440202
:10C8E000909145028A59984509F468CF8AE998E5FC
:10C8F00090934502809344021092180A1092190AEC
:10C9000010921A0A10921B0A59CF23E044EF52E109
:10C91000612F892F79839A830E94835B9A81798121
:10C92000D6CFF4E0AF1226C091E0743009F090E069
:10C9300080914302811152C0002309F403CF99234F
:10C9400009F400CF2FDA8091440290914502825180
:10C95000954609F433CF82E195E6909345028093A2
:10C9600044021092180A1092190A10921A0A109290
:10C970001B0A24CF85E0A81212C091E0753009F09F
:10C9800090E080914302811135C0002309F4DACE92
:10C99000992309F4D7CE06DA85ED92E1FCCEE6E0E4
:10C9A000AE12D0CE91E0763009F090E08091430253
:10C9B00081112CC0002309F4C5CE992309F4C2CEFD
:10C9C000F1D90F900F90DF91CF911F910F91FF90B0
:10C9D000EF90DF90CF90BF90AF90A5C923E04AEED3
:10C9E00052E1612F892F79839A830E94835B9A8118
:10C9F0007981A2CF20E249ED52E1612F892F79831D
:10CA00009A830E94835B9A817981BFCF20E24CECAC
:10CA100052E1612F892F79839A830E94835B9A81E7
:10CA20007981C8CFAF92BF92CF92DF92EF92FF92FF
:10CA30000F931F93CF93DF9310927E0C8091180A6F
:10CA40009091190AA0911A0AB0911B0A813020E82E
:10CA50009207A105B10508F0A0C0D82FB090210A17
:10CA6000DB1518F4D093210ABD2E1091220A12FB77
:10CA7000112710F995E0A92EAB0CCB2D23E0C22E87
:10CA8000D12CE12CF12C19C001E0D11100E08091F2
:10CA9000430281116DC0112311F0011188C0D430FF
:10CAA00048F0C092180AD092190AE0921A0AF0923D
:10CAB0001B0AD3E0CF5FCA1541F16C2F6B19CC2351
:10CAC00019F3C13069F501E0D13009F000E080913F
:10CAD0004302811154C0112311F3002301F362D9E1
:10CAE0008091440290914502835B974671F083EBFD
:10CAF00097E690934502809344021092180A109290
:10CB0000190A10921A0A10921B0ADF91CF911F91F5
:10CB10000F91FF90EF90DF90CF90BF90AF9008956E
:10CB2000C23009F05CC001E0D23009F000E0809131
:10CB3000430281112BC0112309F4B1CF002309F462
:10CB4000AECF30D98091440290914502865A9746E3
:10CB5000E1F286EA97E690934502809344021092B0
:10CB6000180A1092190A10921A0A10921B0ACDCFB5
:10CB700024E045EC52E1802F0E94835B8CCF23E0C0
:10CB80004BEB52E1802F0E94835BA5CF23E042EB69
:10CB900052E1802F0E94835BCECF1092180A109230
:10CBA000190A10921A0A10921B0AD0E057CFFAD82D
:10CBB00080914402909145028156934609F4A5CF95
:10CBC00081E693E690934502809344021092180AFE
:10CBD0001092190A10921A0A10921B0A96CFC330AB
:10CBE00009F05DCF01E0D33009F000E0809143020D
:10CBF00081111EC0112309F452CF002309F44FCF35
:10CC0000D1D880914402909145028959974609F400
:10CC10007CCF89E997E69093450280934402109275
:10CC2000180A1092190A10921A0A10921B0A6DCF54
:10CC300023E047EA52E1802F0E94835BDBCFEF9233
:10CC4000FF920F931F93CF93DF931F92CDB7DEB761
:10CC500010927E0C8091180A9091190AA0911A0ADC
:10CC6000B0911B0A813020E89207A105B10508F0B8
:10CC7000DEC0182FF090210A1F1518F41093210A16
:10CC8000F12E0091220A02FB002700F9E12CF1109D
:10CC900037C091E0111190E0809143028111A9C049
:10CCA00001115BC020E030E040E251E46091FA09FC
:10CCB0007091FB098091FC099091FD090E94A8D513
:10CCC00087FD44C033E083E090E0A0E0B0E024E0E2
:10CCD000121748F08093180A9093190AA0931A0A21
:10CCE000B0931B0A132FE394F394F4E0FE1578F647
:10CCF0000F90DF91CF911F910F91FF90EF900895CA
:10CD0000F1E0FF124CC091E0113009F090E0809109
:10CD10004302811178C0002329F2992319F242D8E5
:10CD20008091440290914502885E9F4609F388EE07
:10CD30009FE690934502809344021092180A109245
:10CD4000190A10921A0A10921B0AD2CF34E084E01A
:10CD500090E0A0E0B0E025E0BBCF992309F4A2CF9A
:10CD600021D880914402909145028251954609F460
:10CD7000BFCF82E195E690934502809344021092E2
:10CD8000180A1092190A10921A0A10921B0A0F9090
:10CD9000DF91CF911F910F91FF90EF90089582E066
:10CDA000F8124FC091E0123009F090E080914302F8
:10CDB000811133C0002309F475CF992309F472CF90
:10CDC0000E94D25E80914402909145028F5E9F4600
:10CDD00009F48ECF8FEE9FE6909345028093440234
:10CDE0001092180A1092190A10921A0A10921B0A2D
:10CDF0007FCF24E04DE952E16E2D892F99830E9467
:10CE0000835B99814DCF23E046E952E16E2D892F56
:10CE100099830E94835B99817ECF23E04FE852E1A2
:10CE20006E2D892F99830E94835B9981C3CF1092C5
:10CE3000180A1092190A10921A0A10921B0A10E08E
:10CE400019CFF3E0FF1227C091E0133009F090E012
:10CE500080914302811159C0002309F423CF992303
:10CE600009F420CF0E94D25E809144029091450245
:10CE7000865F9F4609F43CCF86EF9FE6909345027C
:10CE8000809344021092180A1092190A10921A0AFA
:10CE900010921B0A2DCF20E030E040E251E4609177
:10CEA000FA097091FB098091FC099091FD090E949B
:10CEB000A8D587FF07CF84E0F81248CF91E014305F
:10CEC00009F090E080914302811129C0002309F408
:10CED0003DCF992309F43ACF0E94D25E809144025B
:10CEE00090914502875C9E4609F402CF87EC9EE64E
:10CEF00090934502809344021092180A1092190AE6
:10CF000010921A0A10921B0AF3CE23E048E852E16D
:10CF10006E2D892F99830E94835B99819DCF23E099
:10CF20004FE752E16E2D892F99830E94835B99818F
:10CF3000CDCF8DEC9CECACECBDE38093FA099093E3
:10CF4000FB09A093FC09B093FD0979CE80E090E045
:10CF5000A0E8BFE38093FA099093FB09A093FC0932
:10CF6000B093FD096CCE80E090E0A0E2B1E4809344
:10CF7000FA099093FB09A093FC09B093FD095FCED9
:10CF8000AF92BF92CF92DF92EF92FF920F931F93D7
:10CF9000CF93DF9310927E0C8091180A9091190A1A
:10CFA000A0911A0AB0911B0A813020E89207A105CE
:10CFB000B10508F0A2C0D82F0091210AD01718F4AB
:10CFC000D093210A0D2FB090220AB2FABB24B0F8F8
:10CFD00035E0A32EA00EC02F42E0C42ED12CE12CB0
:10CFE000F12C19C011E0D11110E0809143028111A0
:10CFF0006FC0BB2011F011118AC0D33048F0C0922D
:10D00000180AD092190AE0921A0AF0921B0AD2E08A
:10D01000CF5FCA1549F16C2F601BCC2319F3C130C7
:10D0200071F511E0D13009F010E0809143028111D7
:10D0300056C0BB2011F3112301F30E94D25E8091F0
:10D040004402909145028B5A944871F08BEA94E81F
:10D0500090934502809344021092180A1092190A84
:10D0600010921A0A10921B0ADF91CF911F910F9113
:10D07000FF90EF90DF90CF90BF90AF900895C230B7
:10D0800009F0BBCF11E0D23009F010E080914302EB
:10D0900081112CC0BB2009F4B0CF112309F4ADCF0E
:10D0A0000E94D25E8091440290914502865F904634
:10D0B000D9F286EF90E69093450280934402109255
:10D0C000180A1092190A10921A0A10921B0ACCCF51
:10D0D00024E046EB50E1812F0E94835B8ACF23E05E
:10D0E0004CEA50E1812F0E94835BA3CF23E042EA08
:10D0F00050E1812F0E94835BCDCF1092180A1092CD
:10D10000190A10921A0A10921B0AD0E055CF0E94F9
:10D11000D25E80914402909145028950994609F46B
:10D12000A3CF89E099E69093450280934402109240
:10D13000180A1092190A10921A0A10921B0A94CF18
:10D140008093110A1092100A0895FC012081222375
:10D1500059F1662371F140E030E002C0461710F546
:10D16000207C203809F04F5F3F5FFC01E30FF11D89
:10D1700020812111F3CF21E0240F461798F44FEFBF
:10D18000420F50E2431B01C0322F21E0230FFC016C
:10D19000E30FF11D5083342F320F3617A8F3FC0133
:10D1A000E20FF11D10820895FC0121E040E030E023
:10D1B000E4CFFC01F7CFCF93C62F42E450E0BC018F
:10D1C00085E592E00E94E1DD66E185E592E0BDDF64
:10D1D000C093650C82E080934302CF91089581E073
:10D1E00090915502911101C080E008952091650C45
:10D1F0002111089542E450E0BC0185E592E00E94CF
:10D200004CDE66E185E592E0A0DF82E08093430298
:10D210000895CF92DF92EF92FF920F931F93CF93D7
:10D22000DF931F921F92CDB7DEB710927E0C8091D4
:10D23000180A9091190AA0911A0AB0911B0A81301C
:10D2400020E89207A105B10508F084C2182FC0900C
:10D25000210A1C1518F41093210AC12EF090220AFD
:10D26000F2FAFF24F0F800E0EE24E394C1100BC0C2
:10D2700091E0111190E080914302811129C1FF20BA
:10D2800011F0911189C29091A50C8091A40C981B6A
:10D290009F7009F071C08091FC0681116DC021E082
:10D2A000C21609F41FC133E082E09091A50C2091D1
:10D2B000A40C921B9F7009F069C09091FC0691111B
:10D2C00065C08C1509F435C1C31609F49CC081E012
:10D2D000830F8C1509F4BCC062E0D62ED30E80916A
:10D2E000FD06882309F483C08091E1063A830E94F9
:10D2F000E4583A81882309F4D1C08091FC06882340
:10D3000009F463C1DC1409F4F0C13D5F3C1509F474
:10D3100093C121E0230F121788F030E0215031092A
:10D32000C901AA2797FDA095BA2F8093180A909358
:10D33000190AA0931A0AB0931B0A122F2091210AEE
:10D3400030E02C5F3F4F412F50E0241735070CF0A1
:10D3500054C05CEFC52EC10EC092210AE092430278
:10D3600000E0CC2009F484CF9091A50C8091A40C0E
:10D37000981B9F7009F48FCF32E081E09091A50C4B
:10D380002091A40C921B9F7009F497CF8C119CCF15
:10D3900091E01C1190E08091430281118EC1FF2029
:10D3A00009F492CF992309F48FCF0E94D25E809125
:10D3B000440290914502865D924771F086ED92E7B6
:10D3C00090934502809344021092180A1092190A11
:10D3D00010921A0A10921B0A0F900F90DF91CF91B2
:10D3E0001F910F91FF90EF90DF90CF900895DC1484
:10D3F00009F4C5C023E0230F8ECF0F5FC39405301F
:10D4000008F434CFE9CF91E01C1190E08091430201
:10D410008111FAC0FF2009F45ACF992309F457CF9C
:10D420000E94D25E809144029091450281599246B9
:10D4300099F281E992E6909345028093440210921A
:10D44000180A1092190A10921A0A10921B0AC4CFD5
:10D4500091E01C1190E0809143028111E1C0FF2016
:10D4600009F43ACF992309F437CF0E94D25E809114
:10D470004402909145028F5F9B4509F4ADCF8FEF39
:10D480009BE590934502809344021092180A1092F3
:10D49000190A10921A0A10921B0A9ECFDC10AACF0A
:10D4A00091E01C1190E08091430281113BC1FF206B
:10D4B00009F4A0CF992309F49DCF0E94D25E8091F8
:10D4C0004402909145028B5E9E4509F06FC084CF67
:10D4D00024E04AE555E1602F892F99830E94835B00
:10D4E0009981CDCE91E0113009F090E08091430216
:10D4F0008111CDC0FF2009F4D6CE992309F4D3CEF3
:10D500000E94D25E8091440290914502805C9746D1
:10D5100009F462CF80EC97E6909345028093440231
:10D520001092180A1092190A10921A0A10921B0AE5
:10D5300053CF91E01C1190E0809143028111B1C062
:10D54000FF2009F4C1CE992309F4BECE0E94D25E19
:10D5500080914402909145028156934609F43CCF54
:10D5600081E693E690934502809344021092180A54
:10D570001092190A10921A0A10921B0A2DCF91E0EC
:10D580001C1190E0809143028111A3C0FF2009F497
:10D5900031CF992309F42ECF0E94D25E80914402AC
:10D5A000909145028B5E9E4509F416CF8BEE9EE569
:10D5B00090934502809344021092180A1092190A1F
:10D5C00010921A0A10921B0A07CFDC109ECE91E02F
:10D5D0001C1190E0809143028111D2C0FF2009F418
:10D5E00094CE992309F491CE0E94D25E8EE996E002
:10D5F0000F900F90DF91CF911F910F91FF90EF90BF
:10D60000DF90CF900C94F8BA23E045E355E1602F0A
:10D61000892F3A8399830E94835B99813A81FACE5C
:10D6200023E04AE255E1602F892F3A8399830E94D3
:10D63000835B99813A8113CF91E0131390E080913D
:10D64000430281117BC0FF2009F463CE992309F4C2
:10D6500060CE0E94D25E0E942FA21092FC0660E073
:10D660008EE996E00E943FBF0E94B8C081E080939F
:10D67000930461E087E194E00F900F90DF91CF91E8
:10D680001F910F91FF90EF90DF90CF90AFCD23E0EF
:10D690004AE455E1602F892F99830E94835B998129
:10D6A00029CF23E04DE355E1602F892F3A839983F9
:10D6B0000E94835B99813A8143CF23E045E455E1A1
:10D6C000602F892F3A8399830E94835B99813A81E5
:10D6D00066CE23E042EF54E1602F892F3A8399838D
:10D6E0000E94835B99813A8151CF91E01C1190E0B7
:10D6F00080914302811138C0FF2009F406CE99239E
:10D7000009F403CE0E94D25E8EE996E00F900F904E
:10D71000DF91CF911F910F91FF90EF90DF90CF900D
:10D720000C9402BB23E048EF54E1602F892F3A8329
:10D7300099830E94835B99813A81B9CE20E246E0C9
:10D7400055E1602F892F3A8399830E94835B9981E9
:10D750003A8179CF1092180A1092190A10921A0A77
:10D7600010921B0A10E073CD20E24EE155E1602FCC
:10D77000892F3A8399830E94835B99813A81BCCF38
:10D7800020E241E155E1602F892F3A8399830E947D
:10D79000835B99813A8122CF0E94D25E80914402BC
:10D7A000909145028C5E954709F416CE8CEE95E774
:10D7B00090934502809344021092180A1092190A1D
:10D7C00010921A0A10921B0A07CE2091650C62175C
:10D7D00008F40895F0CC2091650C2230B0F08091CF
:10D7E0004402909145028C5E954771F08CEE95E76E
:10D7F00090934502809344021092180A1092190ADD
:10D8000010921A0A10921B0A089561E0D4DCE7CF47
:10D810001092650C08950F931F93CF93DF93369B5F
:10D820003AC084E025E091E0C0E0349932C0D22FC4
:10D83000C92F0E94FACF00911D0A10911E0A209153
:10D840001F0A3091200A061717072807390710F416
:10D85000329B26C0C093220A8091220A8170909147
:10D86000220A91FD826090911C0A891759F081303B
:10D8700071F1C0F0823031F1833021F4923061F1E6
:10D880009130A1F080931C0ADF91CF911F910F91ED
:10D890000895D82FCECF86E027E093E0C2E0C5CF31
:10D8A000CD2FD8CF9130C1F0923061F790917F0C9D
:10D8B000915090937F0C80931C0ADF91CF911F9120
:10D8C0000F910895992341F09330E1F6EFCF933013
:10D8D00019F0992359F3D6CF90917F0C9F5F9093C5
:10D8E0007F0C80931C0ADF91CF911F910F910895B7
:10D8F0000E94E95A3E983C98469A449A3A98429A2D
:10D9000060E081E30E94E5D19FB7F894EBE0F1E09D
:10D910008081816080839FBF82E08093170A7BDFD4
:10D9200010927F0C08954F925F926F927F928F9228
:10D930009F92AF92BF92CF92DF92EF92FF92CF93DE
:10D94000DF9369DFC0910901C095C170DC2FD170F0
:10D950008091170A8C17B1F082E0809343020E94F5
:10D96000E95AD111FEC08EE996E00E94F1BA809189
:10D97000170A823029F08091650C882309F481C14F
:10D98000C093170A0E94FACF6B017C018091130AA1
:10D990009091140AA091150AB091160A8C159D0554
:10D9A000AE05BF0508F0C9C0C0917F0C6C2F77276A
:10D9B00067FD709577FD00C1643071050CF4CCC033
:10D9C00080917E0C882309F447C080907A0C909057
:10D9D0007B0CA0907C0CB0907D0C81149104A10470
:10D9E000B10409F43CC175956795759567958827CD
:10D9F00077FD8095982F0E944AD62B013C01C701E4
:10DA0000B601681979098A099B090E9448D69B01C9
:10DA1000AC01C301B2010E94AFD520E030E04AE77B
:10DA200054E40E947DD84B015C0120E030E040E2EC
:10DA300053E40E94ABD787FF29C120E030E046E9DC
:10DA400052E4C501B4010E94ABD787FD08C12AE0AA
:10DA500030E040E050E007C121E030E040E050E03D
:10DA6000AC2FBB27A7FDB0950E94E3D997FD04C159
:10DA7000AB01BC0175956795579547957595679569
:10DA8000579547958091180A9091190AA0911A0A02
:10DA9000B0911B0A840F951FA61FB71F8093180A09
:10DAA0009093190AA0931A0AB0931B0A10927F0C44
:10DAB000D701C6018856954CAF4FBF4F8093EA09F6
:10DAC0009093EB09A093EC09B093ED0981E080936A
:10DAD0004302809144029091450225E78C3E9207D3
:10DAE00009F472C020914302211178C025E78C3ED1
:10DAF000920791F0805F9C4579F00E94FACF809068
:10DB0000EA099090EB09A090EC09B090ED09861617
:10DB10009706A806B906B8F1809143028111BBC0EF
:10DB200084E6C80ED11CE11CF11CC092130AD092ED
:10DB3000140AE092150AF092160ADF91CF91FF9035
:10DB4000EF90DF90CF90BF90AF909F908F907F909D
:10DB50006F905F904F9008958091220A82FDA8CF28
:10DB6000B8CF8EE996E00E94F0BA8091170A823011
:10DB700009F406CF8091650C811102CF60E088E93D
:10DB80009FE019DBFDCE80914402909145028C5EAE
:10DB9000954771F08CEE95E790934502809344028F
:10DBA0001092180A1092190A10921A0A10921B0A5F
:10DBB00081E080934302B4CF71956195710964301F
:10DBC00071050CF0FDCEC8CF2091120A211143C07F
:10DBD00081E0809343028AE08093120A8091240AB4
:10DBE0008F5F8093240A87E29AE00E94415A1BC00B
:10DBF00061E087E29AE00E94735A4FE36FE787E2A1
:10DC00009AE00E94765A61E087E29AE00E94735A95
:10DC1000E0914402F0914502199587E29AE00E9452
:10DC2000535A882399F084E00E94C75A40E06DE778
:10DC300087E29AE00E943D5A8091240A80FDD8CF65
:10DC400060E087E29AE00E94735AD7CF8091440245
:10DC5000909145024BCF21502093120A43CF21E0EF
:10DC600030E040E050E0C0927A0CD0927B0CE09221
:10DC70007C0CF0927D0CF4CE6D5F7F4F8F4F9F4FE9
:10DC8000F7CE60E08DE89FE096DA7ACE24E630E0C9
:10DC900040E050E0E8CF81508CCF81E00895809142
:10DCA000220A82FB882780F908958F929F92AF9273
:10DCB000BF92CF92DF92EF92FF92FC01C080D180A1
:10DCC000E280F38020E030E040E251E4C701B60199
:10DCD0000E947DD84B015C0120E030E0A9010E9448
:10DCE000ABD718160CF04CC0C501B4010E9417D672
:10DCF0005B0120E030E0A901C701B6010E94ABD76B
:10DD000087FD3CC08BE28093EE09C50168EE73E0AD
:10DD10000E9473D9CB012AE030E0B9010E9473D987
:10DD2000805D8093EF09C50164E670E00E9473D9BD
:10DD3000CB01B9010E9473D9805D8093F009C501C0
:10DD4000B9010E9473D9482FCB01B9010E9473D940
:10DD5000805D8093F1098EE28093F209405D4093EB
:10DD6000F3091092F4098EEE99E0FF90EF90DF90A6
:10DD7000CF90BF90AF909F908F9008958DE2C3CFCA
:10DD8000C501B40190580E9417D65B01B2CF8091B3
:10DD9000180A9091190AA0911A0AB0911B0A0097CB
:10DDA000A105B105F1F480914302811150C0809129
:10DDB000220A82FF15C080914402909145028F5142
:10DDC000964671F08FE196E6909345028093440267
:10DDD0001092180A1092190A10921A0A10921B0A2D
:10DDE0000895BC01882777FD8095982F0E944AD618
:10DDF0002091FA093091FB094091FC095091FD09ED
:10DE00000E947DD89B01AC016091950670919606A9
:10DE100080919706909198060E94CFD460939506C2
:10DE20007093960680939706909398061092180A1E
:10DE30001092190A10921A0A10921B0A60E070E000
:10DE400080E792E40E94AF5E81E08093430285E91F
:10DE500096E02BDFBC0186E792E10E94D45DA7CF5C
:10DE60008F929F92AF92BF92CF92DF92EF92FF92EA
:10DE70000F931F93CF93DF938C01EB017A01809175
:10DE8000180A9091190AA0911A0AB0911B0A892BBD
:10DE90008A2B8B2B51F580914302811194C0809184
:10DEA000220A82FF15C080914402909145028F5151
:10DEB000964671F08FE196E6909345028093440276
:10DEC0001092180A1092190A10921A0A10921B0A3C
:10DED000DF91CF911F910F91FF90EF90DF90CF9046
:10DEE000BF90AF909F908F9008950E94E823CC0F31
:10DEF000DD1FCC0FDD1FCE018757994F6C0160915C
:10DF0000180A7091190A882777FD8095982F0E942A
:10DF10004AD62091FA093091FB094091FC095091B1
:10DF2000FD090E947DD8F601208131814281538113
:10DF30000E94CFD44B015C0120E030E0A9010E9497
:10DF4000A8D5F60187FD37C080829182A282B38274
:10DF5000B701882777FD8095982F0E944AD66B01DC
:10DF60007C01A50194010E94A8D587FF07C0FE018E
:10DF7000E757F94FC082D182E282F3821092180AE9
:10DF80001092190A10921A0A10921B0AFE01EB5CF9
:10DF9000FB4F60817181828193810E94AF5E81E03D
:10DFA00080934302CE018757994F7FDEBC01C801A1
:10DFB0000E94D45D74CF1082118212821382812C50
:10DFC000912C5401C5CFCC0FDD1FCC0FDD1FEACF44
:10DFD00041E551E060E070E081E692E141CF46EE3C
:10DFE00050E061E070E088E692E13ACF48EC50E022
:10DFF00062E070E08FE692E133CFCF92DF92EF9252
:10E00000FF9220E030E040E251E4FC016081718148
:10E01000828193810E947DD86B017C0120E030E0F9
:10E02000A9010E94ABD71816D4F5C701B6010E940A
:10E0300017D6FB01CF0168EE73E00E9473D9CB01C4
:10E040002AE030E0B9010E9473D9805D8093EE0927
:10E05000CF0164E670E00E9473D9CB01B9010E9440
:10E0600073D9805D8093EF09CF01B9010E9473D904
:10E07000482FCB01B9010E9473D9805D8093F009CC
:10E080008EE28093F109405D4093F2091092F3090A
:10E090008EEE99E0FF90EF90DF90CF900895C7014A
:10E0A000B60190580E9417D6FB01C4CF8F929F9261
:10E0B000AF92BF92CF92DF92EF92FF92CF93FC018B
:10E0C000C080D180E280F38020E030E048EC52E470
:10E0D000C701B6010E947DD84B015C0120E030E011
:10E0E000A9010E94ABD718160CF06DC0C501B40190
:10E0F0000E9417D64B015C0120E030E0A901C70166
:10E10000B6010E94ABD787FD66C0C501B40120E10E
:10E1100037E240E050E00E94A8D9CA01B9012AE0E4
:10E1200030E040E050E00E94A8D9605D6093EE09C5
:10E13000C501B40128EE33E040E050E00E94A8D9C8
:10E14000CAE0CC2ED12CE12CF12CCA01B901A701D7
:10E1500096010E94A8D9605D6093EF09C501B401E2
:10E1600024E630E040E050E00E94A8D9CA01B9019D
:10E17000A70196010E94A8D9605D6093F0098EE224
:10E180008093F109C501B401A70196010E94A8D9A5
:10E19000C62FCA01B901A70196010E94A8D9605DE6
:10E1A0006093F209C05DC093F3091092F4098EEEFA
:10E1B00099E0CF91FF90EF90DF90CF90BF90AF901C
:10E1C0009F908F900895C501B40190580E9417D672
:10E1D0004B015C0191CF6DE2A9CF8F929F92AF92DC
:10E1E000BF92FF920F931F93CF93DF9300D01F92A4
:10E1F000CDB7DEB7F090220AF2FAFF24F0F80091D2
:10E20000180A1091190A20911A0A30911B0A37FD39
:10E2100097C0480159014091000A5091010A60914C
:10E22000020A7091030A401751076207730754F4FA
:10E230004093180A5093190A60931A0A70931B0AA4
:10E240004A015B0120914302211157C0FF2009F4CC
:10E2500042C00091080A1091090A6091180A709151
:10E26000190A80911A0A90911B0A8090040A9090D2
:10E27000050AA090060AB090070A680D791D8A1D4C
:10E280009B1D0E944AD620E030E048EC52E40E94F8
:10E29000AFD5F801608371838283938340910C0A28
:10E2A00050910D0A80910E0A90910F0A209144021C
:10E2B000309145028217930771F090934502809345
:10E2C00044021092180A1092190A10921A0A109217
:10E2D0001B0A452B79F48F2D0F900F900F900F9004
:10E2E000DF91CF911F910F91FF90BF90AF909F90C2
:10E2F0008F9008950E94D25EEECF6091040A7091D3
:10E30000050A8091060A9091070A680D791D8A1DF9
:10E310009B1D0E944AD620E030E048EC52E40E9467
:10E32000AFD569837A838B839C83CE010196BEDE51
:10E33000BC0180910A0A90910B0A0E94D45D86CF9D
:10E340001092180A1092190A10921A0A10921B0AB7
:10E3500000E010E09801812C912C54015CCF3DDF4E
:10E36000811101C00895E091FE09F091FF0919940F
:10E370008F929F92AF92BF92CF92DF92EF92FF92D5
:10E38000FC0180809180A280B38020E030E048ECE6
:10E3900052E4C501B4010E947DD86B017C0120E0EC
:10E3A00030E0A9010E94ABD718160CF0BAC0C70123
:10E3B000B6010E9417D66B017C0120E030E0A90174
:10E3C000C501B4010E94A8D587FD7EC0C701B60172
:10E3D00020E137E240E050E00E94A8D97AE0872EA1
:10E3E000912CA12CB12CCA01B901A50194010E9464
:10E3F000A8D9662309F451C0605D6093EE09C70196
:10E40000B60128EE33E040E050E00E94A8D9CA01EE
:10E41000B901A50194010E94A8D9605D6093EF093C
:10E42000C701B60124E630E040E050E00E94A8D9E0
:10E430006AE0862E912CA12CB12CCA01B901A5014C
:10E4400094010E94A8D9605D6093F009C701B601EC
:10E45000A50194010E94A8D961114DC0CA01B9015A
:10E46000A50194010E94A8D9662309F454C0605DF7
:10E470006093F2098EE28093F10980E28093F309C0
:10E480001092F4098EEE99E0FF90EF90DF90CF901C
:10E49000BF90AF909F908F90089580E28093EE0997
:10E4A000C701B60128EE33E040E050E00E94A8D951
:10E4B000CA01B901A50194010E94A8D9611119C02E
:10E4C00060E26093EF09ACCF8DE28093EE09C70163
:10E4D000B60128EE33E040E050E00E94A8D9CA011E
:10E4E000B9012AE030E040E050E00E94A8D966235C
:10E4F00039F3605DE6CF605D6093F309CA01B9014D
:10E50000A50194010E94A8D9605D6093F2098EE292
:10E510008093F109B5CF80E28093F2098093F109ED
:10E52000ACCFC701B60190580E9417D66B017C0191
:10E5300044CFFC012081318137FD31C024363105C3
:10E5400004F580E28093EE092A30310534F1EAE0E7
:10E55000F0E0C901BF010E9473D9CB01BF010E9445
:10E5600073D9805D8093EF09C9016AE070E00E9471
:10E5700073D9805D8093F0091092F1098EEE99E0D5
:10E580000895C90164E670E00E9473D9CB016AE086
:10E5900070E00E9473D9805DD5CF80E2E3CF8DE239
:10E5A0008093EE09319521953109CECF9F92AF929C
:10E5B000BF92CF92DF92EF92FF920F931F93CF9370
:10E5C000DF931F921F92CDB7DEB710927E0C809121
:10E5D000180A9091190AA0911A0AB0911B0A813069
:10E5E00020E89207A105B10508F03FC1782F90906F
:10E5F000210A791518F47093210A972EB090220AF7
:10E60000B2FABB24B0F810E001E0F6E0CF2ED12C36
:10E61000E12CF12C911023C091E0711190E08091D8
:10E6200043028111FCC0BB2011F0911128C1773049
:10E6300008F08BC0472F50E02091210A30E02C5F7A
:10E640003F4F241735070CF07AC0ECEF9E2E970E43
:10E650009092210A0093430210E09920E9F2F1E040
:10E660009F127FC0AA24A394713009F0A12C80913D
:10E6700043028111E0C0BB20D1F2AA20C1F20E9466
:10E68000D25E809144029091450290930F0A80934C
:10E690000E0A8091180A9091190A90930D0A80939E
:10E6A0000C0A82E08093430282E29AE7909345024B
:10E6B000809344028EE091E190930B0A80930A0AC2
:10E6C0008BE292E09093090A8093080A8AE090E036
:10E6D000A0E0B0E08093040A9093050AA093060A94
:10E6E000B093070A8DED93E0A0E0B0E08093000ABC
:10E6F0009093010AA093020AB093030A80912B021F
:10E7000090912C02AA2797FDA095BA2F0A97A109EC
:10E71000B1098093180A9093190AA0931A0AB0932A
:10E720001B0A0F900F90DF91CF911F910F91FF90D7
:10E73000EF90DF90CF90BF90AF909F9008951F5FB4
:10E740009394153008F466CFECCFC092180AD0929B
:10E75000190AE0921A0AF0921B0A46E050E076E0AD
:10E760006BCF22E09212A4C0AA24A394723009F0C5
:10E77000A12C8091430281116BC0BB2009F457CFBB
:10E78000AA2009F454CF0E94D25E80914402909155
:10E79000450290930F0A80930E0A8091180A909177
:10E7A000190A90930D0A80930C0A82E08093430229
:10E7B00082E29AE7909345028093440280E091E1DF
:10E7C00090930B0A80930A0A8BE69FE19093090AC3
:10E7D0008093080A1092040A1092050A1092060A01
:10E7E0001092070A84E091E0A0E0B0E08093000A74
:10E7F0009093010AA093020AB093030A80916B1FC1
:10E8000090916C1FAA2797FDA095BA2F8093180AA4
:10E810009093190AA0931A0AB0931B0A82CF24E09E
:10E820004AE151E1612F892F7A8399830E94835BAA
:10E8300099817A81F8CE8BE292E07A837ADE9C012C
:10E8400044E151E1612F8A2D0E94725D7A8113CFDC
:10E850008BE69FE17A836DDE9C0147E051E1612FF9
:10E860008A2D0E94725D7A8188CF1092180A1092C8
:10E87000190A10921A0A10921B0A70E0B8CE0E9470
:10E88000D25E80914402909145028950994609F4E4
:10E8900048CF89E099E69093450280934402109214
:10E8A000180A1092190A10921A0A10921B0A39CFEC
:10E8B00083E0981279C0AA24A394733009F0A12CA4
:10E8C00080914302811163C0BB2009F4B0CEAA201D
:10E8D00009F4ADCE0E94D25E81E080937E0C10924E
:10E8E0007A0C10927B0C10927C0C10927D0C809113
:10E8F00044029091450290930F0A80930E0A8091F2
:10E90000180A9091190A90930D0A80930C0A82E0DC
:10E910008093430282EF90E190930B0A80930A0A5E
:10E920008BE69FE19093090A8093080A1092040AEB
:10E930001092050A1092060A1092070A84E091E0EC
:10E94000A0E0B0E08093000A9093010AA093020A2D
:10E95000B093030A80916B1F90916C1FAA2797FDBB
:10E96000A095BA2F8093180A9093190AA0931A0AB7
:10E97000B0931B0A83E29AE7909345028093440286
:10E980008CE896E59093FF098093FE09CACE8BE64A
:10E990009FE17A83CEDD9C0149EF50E1612F8A2D02
:10E9A0000E94725D7A8190CFE4E09E1266C0AA2434
:10E9B000A394743009F0A12C809143028111E6C028
:10E9C000BB2009F434CEAA2009F431CE0E94D25ED5
:10E9D00081E080937E0C10927A0C10927B0C109246
:10E9E0007C0C10927D0C8091440290914502909392
:10E9F0000F0A80930E0A8091180A9091190A909339
:10EA00000D0A80930C0A82E08093430282E29AE727
:10EA100090934502809344028EED90E190930B0A0F
:10EA200080930A0A84E994E09093090A8093080A83
:10EA30001092040A1092050A1092060A1092070A10
:10EA40008FEF90E0A0E0B0E08093000A9093010A7D
:10EA5000A093020AB093030A8091940490919504C4
:10EA6000AA2797FDA095BA2F8093180A9093190AA8
:10EA7000A0931A0AB0931B0A54CEF5E09F1262C00D
:10EA8000AA24A394753009F0A12C8091430281112E
:10EA90008AC0BB2009F4CBCDAA2009F4C8CD0E94BE
:10EAA000D25E809144029091450290930F0A809328
:10EAB0000E0A8091180A9091190A90930D0A80937A
:10EAC0000C0A82E08093430282E29AE79093450227
:10EAD0008093440284ED90E190930B0A80930A0A9C
:10EAE00089E292E09093090A8093080A8AE090E014
:10EAF000A0E0B0E08093040A9093050AA093060A70
:10EB0000B093070A8DED93E0A0E0B0E08093000A97
:10EB10009093010AA093020AB093030A80912902FC
:10EB200090912A02AA2797FDA095BA2F0A97A109CA
:10EB3000B1098093180A9093190AA0931A0AB09306
:10EB40001B0AEFCD26E0921272CD91E0763009F0EB
:10EB500090E080914302811133C0BB2009F467CD5E
:10EB6000992309F464CD0E94D25E8BEB90E10F9063
:10EB70000F90DF91CF911F910F91FF90EF90DF9059
:10EB8000CF90BF90AF909F900C94B92484E994E00B
:10EB90007A83CFDC9C0148EE50E1612F8A2D0E94E0
:10EBA000725D7A810DCF89E292E07A83C2DC9C01AA
:10EBB00049ED50E1612F8A2D0E94725D7A8169CF03
:10EBC00020E245EC50E1612F892F7A8399830E94DE
:10EBD000835B99817A81C1CF7F928F929F92AF920E
:10EBE000BF92CF92DF92EF92FF920F931F93CF933A
:10EBF000DF931F921F92CDB7DEB710927E0C61E0BB
:10EC000087E29AE00E94735A0E94BE5A61E087E24E
:10EC10009AE00E94735A46E063E087E29AE00E941D
:10EC20003D5AE091A41BF091A51BE35BFF4F80814F
:10EC3000882309F437C12CE2E22E20E2F22E0DE007
:10EC400022E04EE065E087E29AE00E94B15A8091AE
:10EC5000A41B9091A51B865A9F4F6BDCBC0187E2D9
:10EC60009AE00E9473D486ED9FE00E94DA5C07E090
:10EC700028E04AE26AE287E29AE00E947F5A05E0D1
:10EC800022E04CE262E387E29AE00E947F5A04E0CD
:10EC90002AE041E36AE287E29AE00E94795A4BE275
:10ECA00062E387E29AE00E94765A29E441E366E350
:10ECB00087E29AE00E94795A0E94BE5A8091FC062F
:10ECC000882371F08091E1060E94E4588111ABC263
:10ECD00020E002E042E367E387E29AE00E947F5A85
:10ECE0004FE265E387E29AE00E943D5A80917E04FC
:10ECF00090917F04A0918004B0918104892B8A2B8C
:10ED00008B2B09F4E0C00E94FACFC0907E04D09013
:10ED10007F04E0908004F09081046C197D098E09D5
:10ED20009F0920E63AEE40E050E00E9486D9690152
:10ED30007A018091E1060E94E458811143C224E6E1
:10ED40002C9DC0012D9D900D112460E070E00E946B
:10ED50005FD94B0183E50E94655B9601A9E8B8E89D
:10ED60000E94CAD95C01B694A794B294A294BFE061
:10ED7000AB22AB24BB22AB24C50199270AE010E0EB
:10ED8000B8010E9473D9282FCB01B8010E9473D912
:10ED9000805D8093EE09205D2093EF091092F009C9
:10EDA0008EEE99E00E94EA5B8AE30E94655B8CE349
:10EDB000782E7A9CC0017B9C900D11249601281B13
:10EDC000390BC901B8010E9473D9282FCB01B801B2
:10EDD0000E9473D9805D8093EE09205D2093EF0936
:10EDE0001092F0098EEE99E00E94EA5B4FE26AE52C
:10EDF00087E29AE00E943D5AC4010197843695400B
:10EE000008F071C265E487E29AE00E9474D494012C
:10EE1000A9E8B8E80E94CAD97C01F694E794F29474
:10EE2000E294AFE0EA22EF24FA22EF24C701B8010E
:10EE30000E9473D9282FCB01B8010E9473D9805D3D
:10EE40008093EE09205D2093EF091092F0096EEE99
:10EE500079E087E29AE00E9473D46AE387E29AE05D
:10EE60000E9474D47E9CC0017F9C900D112494015B
:10EE7000281B390BC901B8010E9473D9282FCB0177
:10EE8000B8010E9473D9805D8093EE09205D2093C4
:10EE9000EF091092F0096EEE79E087E29AE00E94A5
:10EEA00073D41FC092E1E92E90E2F92E0DE022E02A
:10EEB0004EE065E087E29AE00E94B15A81ED9FE062
:10EEC0000E94DA5CD4CE83EC9FE00E94DA5C4FE2D1
:10EED0006AE587E29AE00E943D5A8CEB9FE00E942F
:10EEE000DA5C0E94BE5A4BE168E687E29AE00E9433
:10EEF0003D5A8091940490919504019644E6489F70
:10EF00009001499F300D112437FDDBC1832F932FD2
:10EF1000990F990B9A838983892B09F44BC1CE01F0
:10EF2000019607DB0E94EA5B85E20E94655B0E9416
:10EF3000BE5A09E020E84EE160E087E29AE00E94D4
:10EF40007F5A60E087E29AE00E94735A46E262E0EC
:10EF500087E29AE00E943D5A8091780680FD04C0C5
:10EF60008091770680FDA5C188E50E94655B41E23E
:10EF700068E087E29AE00E94765A43E268E087E21E
:10EF80009AE00E94765A46E26AE087E29AE00E949E
:10EF90003D5A8091770680FF08C189E896E02DD818
:10EFA0000E94EA5B46E26BE287E29AE00E943D5AE9
:10EFB0008091780681FD04C08091770681FD77C13C
:10EFC00089E50E94655B41E261E387E29AE00E9485
:10EFD000765A43E261E387E29AE00E94765A46E27B
:10EFE00063E387E29AE00E943D5A8091770681FFB1
:10EFF00072C08DE896E001D80E94EA5B46E263E5C4
:10F0000087E29AE00E943D5A8091780682FD04C012
:10F010008091770682FD49C18AE50E94655B41E2E5
:10F0200069E587E29AE00E94765A43E269E587E261
:10F030009AE00E94765A46E26BE587E29AE00E94E7
:10F040003D5A8091770682FD36C189EA9FE00E9491
:10F05000DA5C61E087E29AE00E94735A84E00E94E1
:10F06000C75A41E363E087E29AE00E943D5A86E096
:10F070000E94655B0E94BE5A41E36CE087E29AE021
:10F080000E943D5A8BE292E054DA0E94EA5B85E2EC
:10F090000E94655B0E94BE5A4FE360E087E29AE0FF
:10F0A0000E943D5A85E592E00E94EA5B8091220A27
:10F0B00082FB882780F99091110A992389F0909119
:10F0C000100A992309F4E8C0811125C01092100A92
:10F0D0001092110A20C080EB9FE00E94DA5C8ECF74
:10F0E0008823C9F080914402909145028950994645
:10F0F00081F089E099E69093450280934402109252
:10F10000180A1092190A10921A0A10921B0A0E94E9
:10F11000D25E0E94E95A80912B0290912C0220919C
:10F12000180A3091190A843691055CF5280F391FA9
:10F13000253631057CF51092180A1092190A1092A2
:10F140001A0A10921B0A2A303105CCF1C901883EF7
:10F1500023E0920714F087EE93E090932C028093C3
:10F160002B020F900F90DF91CF911F910F91FF9085
:10F17000EF90DF90CF90BF90AF909F908F907F9057
:10F1800008958436910509F49FC0280F391F24364D
:10F1900031058CF61092180A1092190A10921A0A68
:10F1A00010921B0A84E690E0D2CF84EB9FE00E948D
:10F1B000DA5CF8CE88EB9FE00E94DA5CB8CE8AE099
:10F1C00090E0CBCF8091FF0690910007A0910107BE
:10F1D000B09102070097A105B10509F4B0CDBC01BB
:10F1E000CD016D597F4F8F4F9F4F24E630E040E0B7
:10F1F00050E00E9486D960910307709104078091C6
:10F200000507909106070E9486D930E044E650E059
:10F21000421B530B4C9DC0014D9D900D5C9D900D6C
:10F220001124B90194CD8091FF0690910007A0911F
:10F230000107B09102070097A105B10509F448CD77
:10F24000BC01CD016D597F4F8F4F9F4F24E630E0B9
:10F2500040E050E00E9486D9609103077091040756
:10F2600080910507909106070E9486D9622F70E071
:10F2700080E090E00E944AD620E030E04EE852E480
:10F280000E947DD820E030E048EC52E40E94AFD5E7
:10F290000E941CD6262F1DCD882309F43CCF0E9446
:10F2A000D25E81E08093100A36CF8FE3B6CE8FE333
:10F2B00088CE8FE35ACE81E996E05AD80E94EA5B65
:10F2C000C8CE21503F4F22CE2B3031058CF010920A
:10F2D000180A1092190A10921A0A10921B0AC901F0
:10F2E000865A9F4F34CF8AEC9FE00E94DA5CF9CDBA
:10F2F000263F4FEF34070CF02ACF1092180A1092D5
:10F30000190A10921A0A10921B0A22593F4F1BCF5A
:10F31000BF92CF92DF92EF92FF920F931F93CF9302
:10F32000DF931F921F92CDB7DEB7B090220AB2FAD8
:10F33000BB24B0F80091180A1091190A20911A0AFA
:10F3400030911B0A37FD6FC0680179014091000AB6
:10F350005091010A6091020A7091030A4017510707
:10F360006207730754F44093180A5093190A609384
:10F370001A0A70931B0A6A017B0180914302811172
:10F380003FC0BB2069F1E091080AF091090A209181
:10F39000040A3091050A8091180A9091190A280FE1
:10F3A000391F3183208340910C0A50910D0A8091BE
:10F3B0000E0A90910F0A2091440230914502821763
:10F3C000930771F090934502809344021092180ABB
:10F3D0001092190A10921A0A10921B0A452B69F40E
:10F3E0008B2D0F900F90DF91CF911F910F91FF9078
:10F3F000EF90DF90CF90BF9008950E94D25EF0CF43
:10F400008091040A9091050A8C0D9D1D9A83898331
:10F41000CE0101968ED8BC0180910A0A90910B0A08
:10F420000E94D45DAECF1092180A1092190A109261
:10F430001A0A10921B0A00E010E09801C12CD12C8E
:10F44000760184CF65CF64DF811101C00895E0911A
:10F45000FE09F091FF0919948F929F92AF92BF928B
:10F46000FF920F931F93CF93DF931F921F92CDB7FD
:10F47000DEB7F090220AF2FAFF24F0F80091180AA1
:10F480001091190A20911A0A30911B0A37FD89C080
:10F49000480159014091000A5091010A6091020A05
:10F4A0007091030A401751076207730754F44093A1
:10F4B000180A5093190A60931A0A70931B0A4A019A
:10F4C0005B012091430221114EC0FF20E1F1009128
:10F4D000080A1091090A6091180A7091190A80911E
:10F4E0001A0A90911B0A8090040A9090050AA09035
:10F4F000060AB090070A680D791D8A1D9B1D0E949F
:10F500004AD6F801608371838283938340910C0A09
:10F5100050910D0A80910E0A90910F0A2091440299
:10F52000309145028217930771F0909345028093C2
:10F5300044021092180A1092190A10921A0A109294
:10F540001B0A452B69F48F2D0F900F90DF91CF91FF
:10F550001F910F91FF90BF90AF909F908F90089553
:10F560000E94D25EF0CF6091040A7091050A8091EA
:10F57000060A9091070A680D791D8A1D9B1D0E943D
:10F580004AD60E9417D67A836983CE0101960E94DB
:10F590009972BC0180910A0A90910B0A0E94D45D75
:10F5A00094CF1092180A1092190A10921A0A109207
:10F5B0001B0A00E010E09801812C912C54016ACFC5
:10F5C0004BCF8F929F92AF92BF92CF92DF92EF92EA
:10F5D000FF92FC01C080D180E280F38020E030E027
:10F5E000A901C701B6010E94ABD718160CF092C052
:10F5F000C701B6010E9417D66B017C01F0E1CF165E
:10F60000F7E2DF06E104F1040CF465C0C701B601BE
:10F6100020E137E240E050E00E94A8D9CA01B901D8
:10F620002AE030E040E050E00E94A8D9605D60939D
:10F63000EE09C701B60128EE33E040E050E00E9439
:10F64000A8D9CA01B9012AE030E040E050E00E94A8
:10F65000A8D9605D6093EF09C701B60124E630E0E8
:10F6600040E050E00E94A8D9CA01B9012AE030E088
:10F6700040E050E00E94A8D9605D6093F0094AE044
:10F68000842E912CA12CB12CC701B601A5019401A7
:10F690000E94A8D9CA01B901A50194010E94A8D964
:10F6A000605D6093F109C701B6012AE030E040E0F7
:10F6B00050E00E94A8D9605D6093F2091092F309AE
:10F6C0008EEE99E0FF90EF90DF90CF90BF90AF90DB
:10F6D0009F908F90089580E28093EE0998EEC9166E
:10F6E00093E0D906E104F1040CF0A3CF8093EF0975
:10F6F000E4E6CE16D104E104F1040CF0ADCF809322
:10F70000F009FAE0CF16D104E104F1040CF0B7CF10
:10F7100060E2C7CFC701B60190580E9417D66B01AF
:10F720007C016CCF8F929F92AF92BF92FF920F930A
:10F730001F93CF93DF9300D01F92CDB7DEB7F09029
:10F74000220AF2FAFF24F0F80091180A1091190A1F
:10F7500020911A0A30911B0A37FD97C048015901C0
:10F760004091000A5091010A6091020A7091030AC7
:10F77000401751076207730754F44093180A5093D7
:10F78000190A60931A0A70931B0A4A015B012091BF
:10F790004302211157C0FF2009F442C00091080A1A
:10F7A0001091090A6091180A7091190A80911A0A39
:10F7B00090911B0A8090040A9090050AA090060A76
:10F7C000B090070A680D791D8A1D9B1D0E944AD6BC
:10F7D0002AE037ED43E25CE30E94AFD5F801608395
:10F7E00071838283938340910C0A50910D0A80911A
:10F7F0000E0A90910F0A209144023091450282171F
:10F80000930771F090934502809344021092180A76
:10F810001092190A10921A0A10921B0A452B79F4B9
:10F820008F2D0F900F900F900F90DF91CF911F9120
:10F830000F91FF90BF90AF909F908F9008950E947E
:10F84000D25EEECF6091040A7091050A8091060A9B
:10F850009091070A680D791D8A1D9B1D0E944AD64A
:10F860002AE037ED43E25CE30E94AFD569837A83F7
:10F870008B839C83CE010196A4DEBC0180910A0A91
:10F8800090910B0A0E94D45D86CF1092180A1092B4
:10F89000190A10921A0A10921B0A00E010E098014F
:10F8A000812C912C54015CCF3DCF8F929F92AF92CF
:10F8B000BF92FF920F931F93CF93DF9300D01F92BD
:10F8C000CDB7DEB7F090220AF2FAFF24F0F80091EB
:10F8D000180A1091190A20911A0A30911B0A37FD53
:10F8E00099C0480159014091000A5091010A609164
:10F8F000020A7091030A401751076207730754F414
:10F900004093180A5093190A60931A0A70931B0ABD
:10F910004A015B0120914302211159C0FF2009F4E3
:10F9200044C00091080A1091090A6091180A709168
:10F93000190A80911A0A90911B0A8090040A9090EB
:10F94000050AA090060AB090070A680D791D8A1D65
:10F950009B1D0E9448D62AE037ED43E25CE30E94FB
:10F96000AFD50E941CD6F801608371838283938394
:10F9700040910C0A50910D0A80910E0A90910F0A45
:10F9800020914402309145028217930771F09093C1
:10F990004502809344021092180A1092190A10929C
:10F9A0001A0A10921B0A452B79F48F2D0F900F9095
:10F9B0000F900F90DF91CF911F910F91FF90BF900B
:10F9C000AF909F908F9008950E94D25EEECF60918D
:10F9D000040A7091050A8091060A9091070A680D41
:10F9E000791D8A1D9B1D0E9448D62AE037ED43E20F
:10F9F0005CE30E94AFD569837A838B839C83CE01BD
:10FA00000196DFDDBC0180910A0A90910B0A0E94E9
:10FA1000D45D84CF1092180A1092190A10921A0A13
:10FA200010921B0A00E010E09801812C912C5401E7
:10FA30005ACF3BCF3ADF811101C00895E091FE0912
:10FA4000F091FF0919948F929F92AF92BF92CF923B
:10FA5000DF92EF92FF92CF93FC01C080D180E280D1
:10FA6000F38020E030E040E251E4C701B6010E949B
:10FA70007DD84B015C0120E030E0A9010E94ABD7AA
:10FA800018160CF070C0C501B4010E9417D64B01C6
:10FA90005C0120E030E0A901C701B6010E94ABD7AC
:10FAA00087FD5FC08BE28093EE09C501B40120E1C0
:10FAB00037E240E050E00E94A8D96AE0C62ED12C7F
:10FAC000E12CF12CCA01B901A70196010E94A8D925
:10FAD000605D6093EF09C501B40128EE33E040E0BA
:10FAE00050E00E94A8D9CA01B901A70196010E945D
:10FAF000A8D9605D6093F009C501B40124E630E047
:10FB000040E050E00E94A8D9CA01B901A7019601BE
:10FB10000E94A8D9605D6093F109C501B401A701F5
:10FB200096010E94A8D9C62FCA01B901A701960162
:10FB30000E94A8D9605D6093F2098EE28093F30978
:10FB4000C05DC093F4091092F5098EEE99E0CF9153
:10FB5000FF90EF90DF90CF90BF90AF909F908F90ED
:10FB600008958DE2A0CFC501B40190580E9417D628
:10FB70004B015C018ECF8F929F92AF92BF92FF920A
:10FB80000F931F93CF93DF9300D01F92CDB7DEB7B3
:10FB9000F090220AF2FAFF24F0F80091180A10916E
:10FBA000190A20911A0A30911B0A37FD97C04801A3
:10FBB00059014091000A5091010A6091020A709126
:10FBC000030A401751076207730754F44093180A59
:10FBD0005093190A60931A0A70931B0A4A015B0139
:10FBE00020914302211157C0FF2009F442C0009127
:10FBF000080A1091090A6091180A7091190A8091F7
:10FC00001A0A90911B0A8090040A9090050AA0900D
:10FC1000060AB090070A680D791D8A1D9B1D0E9477
:10FC20004AD620E030E040E251E40E94AFD5F8012E
:10FC3000608371838283938340910C0A50910D0AF3
:10FC400080910E0A90910F0A209144023091450252
:10FC50008217930771F090934502809344021092AB
:10FC6000180A1092190A10921A0A10921B0A452BB0
:10FC700079F48F2D0F900F900F900F90DF91CF910F
:10FC80001F910F91FF90BF90AF909F908F9008951C
:10FC90000E94D25EEECF6091040A7091050A8091B5
:10FCA000060A9091070A680D791D8A1D9B1D0E9406
:10FCB0004AD620E030E040E251E40E94AFD56983AB
:10FCC0007A838B839C83CE010196BDDEBC0180913B
:10FCD0000A0A90910B0A0E94D45D86CF1092180AEE
:10FCE0001092190A10921A0A10921B0A00E010E0F2
:10FCF0009801812C912C54015CCF3DCF8F929F9223
:10FD0000AF92BF92CF92DF92EF92FF92CF93DF93A9
:10FD1000EC0120E030E0A901688179818A819B8132
:10FD20000E94ABD787FD82C08BE28093EE0920E072
:10FD300030E048EC52E4688179818A819B810E949D
:10FD40007DD86B017C0120E030E0A9010E94ABD797
:10FD500018160CF063C0C701B6010E9417D64B01FC
:10FD60005C01C501B40120E137E240E050E00E94AF
:10FD7000A8D97AE0C72ED12CE12CF12CCA01B90107
:10FD8000A70196010E94A8D9605D6093EF09C501A3
:10FD9000B40128EE33E040E050E00E94A8D9CA0147
:10FDA000B901A70196010E94A8D9605D6093F0098E
:10FDB000C501B40124E630E040E050E00E94A8D93B
:10FDC000CA01B901A70196010E94A8D9605D60939C
:10FDD000F1098EE28093F209C501B401A7019601F1
:10FDE0000E94A8D9C62FCA01B901A70196010E9495
:10FDF000A8D9605D6093F309C05DC093F4091092C7
:10FE0000F5098EEE99E0DF91CF91FF90EF90DF90B2
:10FE1000CF90BF90AF909F908F900895C701B6018B
:10FE200090580E9417D64B015C019BCF8DE27DCF8D
:10FE30008F929F92AF92BF92CF92DF92EF92FF92FA
:10FE40000F931F93CF93DF9300D01F921F92CDB7D4
:10FE5000DEB710927E0C8091180A9091190AA09139
:10FE60001A0AB0911B0A813020E89207A105B1055A
:10FE700008F0DEC0182FB090210A1B1518F410935B
:10FE8000210AB12E0091220A02FB002700F9A12CC1
:10FE900099249394E4E1CE2ED12CE12CF12CB110D5
:10FEA00022C091E0111190E080914302811193C032
:10FEB000002311F09111C6C0153108F048C0212F60
:10FEC00030E08091210A90E00496821793070CF0AD
:10FED00051C0ECEFBE2EB10EB092210A90924302B7
:10FEE000A12CBB20F1F281E0B8124BC0882483948E
:10FEF000113009F0812C80914302811176C00023DA
:10FF0000D9F28820C9F20E94D25E20E030E040E2BF
:10FF100051E46FE17BE182E894E10E945F5984E55E
:10FF20009CE790934502809344020F900F900F90AE
:10FF30000F900F90DF91CF911F910F91FF90EF9055
:10FF4000DF90CF90BF90AF909F908F900895C09218
:10FF5000180AD092190AE0921A0AF0921B0A24E1B8
:10FF600030E014E18091210A90E004968217930713
:10FF70000CF4AFCFA394B39484E08A1508F08FCF2C
:10FF8000D4CF22E0B21277C088248394123009F0D3
:10FF9000812C80914302811133C0002309F48CCF5E
:10FFA000882009F489CF0E94D25EE12C10E8F12E5E
:10FFB00007E714E420E030E040E85FE363E17BE141
:10FFC00080E794E10E948D5680EE9AE79093450277
:10FFD00080934402AACF24E04EE854E16A2D892F91
:10FFE0009D830E94835B9D8163CF8FE19BE1E9DA72
:10FFF0009C0148E854E16A2D882D0E94725D7FCFF4
:020000021000EC
:100000006091131B7091141B8091151B9091161B0E
:100010000E9417D67A836983CE0101960E94997255
:100020009C0149E754E16A2D882D0E94725DB5CF8D
:100030001092180A1092190A10921A0A10921B0AAA
:1000400010E019CF0E94D25E809144029091450247
:100050008159924609F469CF81E992E6909345026D
:10006000809344021092180A1092190A10921A0AE8
:1000700010921B0A5ACF83E0B81232C088248394AE
:10008000133009F0812C8091430281111EC000239E
:1000900009F412CF882009F40FCF0E94D25EE12C20
:1000A00010E8F12E07E714E42DEC3CEC4CEC5DE39A
:1000B0006FE07BE180E694E10E94FC5685E997E8D9
:1000C000909345028093440230CF8FE09BE116DE8F
:1000D0009C0148E654E16A2D882D0E94725DD7CFBD
:1000E00024E0B21227C088248394143009F0812CB4
:1000F00080914302811172C0002309F4DDCE882073
:1001000009F4DACE0E94D25EE12C10ECF12E09E760
:1001100014E420E030E040E85FE367E47BE182E55F
:1001200094E10E948D5680EE9AE790934502809369
:100130004402FBCE85E0B81227C088248394153092
:1001400009F0812C80914302811160C0002309F4E1
:10015000B3CE882009F4B0CE0E94D25EE12C10EC20
:10016000F12E09E714E420E030E040E85FE36BE4BF
:100170007BE184E494E10E948D5680EE9AE79093AF
:10018000450280934402D1CE26E0B2126FC088248B
:100190008394163009F0812C8091430281114EC066
:1001A000002309F489CE882009F486CE0E94D25E0D
:1001B000E12C10ECF12E09E714E420E030E040E8F7
:1001C0005FE36FE47BE186E394E10E948D5680EE6D
:1001D0009AE79093450280934402A7CE6091471B13
:1001E0007091481B8091491B90914A1B0E9417D621
:1001F0007A836983CE0101960E9499729C0149E538
:1002000054E16A2D882D0E94725D76CF60914B1B60
:1002100070914C1B80914D1B90914E1B0E9417D6E4
:100220007A836983CE0101960E9499729C014BE406
:1002300054E16A2D882D0E94725D88CF60914F1B1A
:100240007091501B8091511B9091521B0E9417D6A8
:100250007A836983CE0101960E9499729C014DE3D5
:1002600054E16A2D882D0E94725D9ACF87E0B81202
:100270003EC088248394173009F0812C809143027A
:1002800081111DC0002309F417CE882009F414CE73
:100290000E94D25EE12C10ECF12E09E714E420E07C
:1002A00030E0A90163E27BE18CE294E10E948D568B
:1002B00080EE9AE7909345028093440236CE609197
:1002C000231B7091241B8091251B9091261B0E945B
:1002D00017D67A836983CE0101960E9499729C0198
:1002E00041E354E16A2D882D0E94725DCBCF28E056
:1002F000B2123EC088248394183009F0812C80917A
:10030000430281111DC0002309F4D6CD882009F4D1
:10031000D3CD0E94D25EE12C10ECF12E09E714E45B
:1003200020E030E0A90167E07BE188E194E10E94F0
:100330008D5680EE9AE79093450280934402F5CD66
:100340006091071B7091081B8091091B90910A1BFB
:100350000E9417D67A836983CE0101960E94997212
:100360009C0142E254E16A2D882D0E94725DCBCF40
:1003700089E0B81241C088248394193009F0812C97
:100380008091430281111FC0002309F495CD88207C
:1003900009F492CD0E94D25E24E630E040E050E0C5
:1003A00067E27BE18AE094E10E94EC588AE19DE7F4
:1003B000909345028093440286E097E99093FF0969
:1003C0008093FE09B2CD6091271B7091281B80910C
:1003D000291B90912A1B0E9448D669837A838B83BC
:1003E0009C83CE010196EDD89C0141E154E16A2D38
:1003F000882D0E94725DC8CF2AE0B21233C08824D3
:1004000083941A3009F0812C80914302811111C02C
:10041000002309F451CD882009F44ECD0E94D25E0C
:1004200024E630E040E050E06BE27BE18CEF93E1CA
:10043000BBCF60912B1B70912C1B80912D1B909139
:100440002E1B0E9448D669837A838B839C83CE01BE
:100450000196B7D89C0143E054E16A2D882D0E9493
:10046000725DD6CF8BE0B81233C0882483941B30E2
:1004700009F0812C80914302811111C0002309F4FD
:100480001BCD882009F418CD0E94D25E2AE030E00E
:1004900040E050E06FE27BE18EEE93E185CF60912A
:1004A0002F1B7091301B8091311B9091321B0E9449
:1004B00048D669837A838B839C83CE01019681D849
:1004C0009C0145EF53E16A2D882D0E94725DD6CFC5
:1004D0002CE0B2122DC0882483941C3009F0812CAA
:1004E00080914302811119C0002309F4E5CC8820D2
:1004F00009F4E2CC0E94D25E20E030E048EC52E405
:1005000067E17BE18CED93E10E945F5984E59CE714
:10051000909345028093440208CD87E19BE151D836
:100520009C0145EE53E16A2D882D0E94725DDCCF5F
:100530008DE0B81232C0882483941D3009F0812CDC
:100540008091430281111EC0002309F4B5CC88209C
:1005500009F4B2CC0E94D25EE12C1CE3F12E0CE136
:1005600016E420E030E040EA50E467E37BE186EC0B
:1005700093E10E94FC5685E997E8909345028093A9
:100580004402D3CC87E39BE1B9DB9C0141ED53E10D
:100590006A2D882D0E94725DD7CF2EE0B21232C034
:1005A000882483941E3009F0812C809143028111AC
:1005B0001EC0002309F480CC882009F47DCC0E9461
:1005C000D25EE12C1CE3F12E0CE116E420E030E0D9
:1005D00040EA50E46BE37BE180EB93E10E94FC5640
:1005E00085E997E890934502809344029ECC8BE383
:1005F0009BE184DB9C014BEB53E16A2D882D0E942B
:10060000725DD7CF8FE0B81229C0882483941F3041
:1006100009F0812C80914302811115C0002309F457
:100620004BCC882009F448CC0E94D25E6FE37BE17A
:100630008AE993E10E94D0598DE79EE790934502A5
:100640008093440272CC8FE39BE1FDD99C0145EA83
:1006500053E16A2D882D0E94725DE0CF20E1B21235
:100660003FC088248394103109F0812C809143028B
:1006700081111EC0002309F41FCC882009F41CCC72
:100680000E94D25EE12C10E8F12E07E714E420E08E
:1006900030E040E85FE36BE07BE186E893E10E94B5
:1006A0008D5680EE9AE790934502809344023DCCAC
:1006B00060910B1B70910C1B80910D1B90910E1B78
:1006C0000E9417D67A836983CE0101960E9499729F
:1006D0009C0140E953E16A2D882D0E94725DCACFCA
:1006E00081E1B8123FC088248394113109F0812C34
:1006F0008091430281111EC0002309F4DDCB8820C4
:1007000009F4DACB0E94D25EE12C10ECF12E09E75D
:1007100014E420E030E040E85FE363E57BE186E756
:1007200093E10E948D5680EE9AE790934502809364
:100730004402FBCB6091531B7091541B8091551B5D
:100740009091561B0E9417D67A836983CE01019639
:100750000E9499729C014EE753E16A2D882D0E94F8
:10076000725DCACF22E1B2123CC088248394123158
:1007700009F0812C80914302811119C0002309F4F2
:100780009BCB882009F498CB0E94D25E24E630E00F
:1007900040E050E063E37BE186E693E10E94EC58A1
:1007A00089E19DE79093450280934402BECB60911E
:1007B000331B7091341B8091351B9091361B0E9426
:1007C00048D669837A838B839C83CE0101960E94ED
:1007D000E17A9C014EE653E16A2D882D0E94725DFC
:1007E000CDCF83E1B8122EC088248394133109F051
:1007F000812C80914302811119C0002309F45CCB44
:10080000882009F459CB0E94D25E20E030E048EC09
:1008100052E46BE17BE18EE493E10E945F5984E551
:100820009CE790934502809344027FCB8BE19BE150
:100830000E94E17A9C014AE553E16A2D882D0E94CD
:10084000725DDBCF24E1B21237CB8824839414315C
:1008500009F0812C80914302811115C0002309F415
:100860002BCB882009F428CB0E94D25E63E47BE185
:1008700086E393E10E94D0598DE79EE7909345026D
:100880008093440252CB83E49BE1DDD89C0142E497
:1008900053E16A2D882D0E94725DE0CF0F931F9364
:1008A000CF93DF93CDB7DEB76C970FB6F894DEBF6A
:1008B0000FBECDBF9B01AC018091770682FD0CC0BD
:1008C00084EE9FE0298F3A8F4B8F5C8F0E94B92472
:1008D0005C8D4B8D3A8D298D2093F6093093F70965
:1008E0004093F8095093F90960E070E085E992E4DB
:1008F0000E94CED46D8B7E8B8F8B988FCE014596C8
:10090000FDD99F938F9388ED9FE09F938F938E01E6
:100910000F5F1F4F1F930F930E9466DEC8010E9456
:10092000B9240F900F900F900F900F900F906C962E
:100930000FB6F894DEBF0FBECDBFDF91CF911F91F0
:100940000F9108956091F6097091F7098091F80967
:100950009091F909A3CF9F92AF92BF92CF92DF926D
:10096000EF92FF920F931F93CF93DF931F921F92EB
:10097000CDB7DEB710927E0C8091180A9091190ABB
:10098000A0911A0AB0911B0A813020E89207A105B4
:10099000B10508F0B6C0782F9090210A791518F4A7
:1009A0007093210A972E0091220A02FB002700F97A
:1009B00010E0BB24B394A8E0CA2ED12CE12CF12C7A
:1009C000911021C091E0711190E08091430281115A
:1009D00074C0002311F091119EC07930E8F5472FC3
:1009E00050E02091210A30E02C5F3F4F241735075B
:1009F00004F5FCEF9F2E970E9092210AB0924302CD
:100A000010E09920F9F2F1E09F1232C091E07130CC
:100A100009F090E08091430281115BC00023E9F26C
:100A20009923D9F20E94D25E60E070E080E89FE3F3
:100A300036C01F5F9394153008F4C2CF0F900F900B
:100A4000DF91CF911F910F91FF90EF90DF90CF90AA
:100A5000BF90AF909F900895C092180AD092190A43
:100A6000E0921A0AF0921B0A48E050E078E0B9CF11
:100A700022E0921269C091E0723009F090E080911A
:100A80004302811132C0002309F4A7CF992309F44E
:100A9000A4CF0E94D25E60E070E080E090E40F900E
:100AA0000F90DF91CF911F910F91FF90EF90DF900A
:100AB000CF90BF90AF909F90F1CE24E049E250E1FB
:100AC000612F892F7A8399830E94835B99817A8130
:100AD00080CF20E245E250E1612F892F7A8399830C
:100AE0000E94835B99817A8199CF20E241E250E1B3
:100AF000612F892F7A8399830E94835B99817A8100
:100B0000C2CF1092180A1092190A10921A0A109263
:100B10001B0A70E041CF0E94D25E80914402909106
:100B20004502805C974609F489CF80EC97E6909364
:100B30004502809344021092180A1092190A1092EA
:100B40001A0A10921B0A7ACF83E0981221C091E012
:100B5000733009F090E08091430281110DC00023B1
:100B600009F43BCF992309F438CF0E94D25E60E0AC
:100B700070E080E490E493CF20E245E150E1612F02
:100B8000892F7A8399830E94835B99817A81E7CF49
:100B9000E4E09E1215C091E0743009F090E080917D
:100BA000430281113DC0002309F417CF992309F4B2
:100BB00014CF0E94D25E60E070E080E890E46FCFD6
:100BC000F5E09F1215C091E0753009F090E080913A
:100BD0004302811131C0002309F4FFCE992309F4A7
:100BE000FCCE0E94D25E60E070E080EA90E457CFD5
:100BF00026E0921239C091E0763009F090E08091C1
:100C00004302811125C0002309F4E7CE992309F49A
:100C1000E4CE0E94D25E60E070E080EC90E43FCFD2
:100C200020E241E150E1612F892F7A8399830E946C
:100C3000835B99817A81B7CF20E24DE050E1612F4B
:100C4000892F7A8399830E94835B99817A81C3CFAC
:100C500020E241E050E1612F892F7A8399830E943D
:100C6000835B99817A81CFCF87E0981221C091E090
:100C7000773009F090E08091430281110DC000238C
:100C800009F4ABCE992309F4A8CE0E94D25E60E0AD
:100C900070E080EE90E403CF20E24DEF5FE0612F43
:100CA000892F7A8399830E94835B99817A81E7CF28
:100CB000E8E09E1292CEAA24A394783009F0A12CE9
:100CC00080914302811160C0002309F486CEAA20DE
:100CD00009F483CE0E94D25E809144029091450235
:100CE00090930F0A80930E0A8091180A9091190A26
:100CF00090930D0A80930C0A82E0809343028FEE5A
:100D00009FE090930B0A80930A0A86EF99E09093F4
:100D1000090A8093080A1092040A1092050A109298
:100D2000060A1092070A8AE19DE1A0E0B0E08093F4
:100D3000000A9093010AA093020AB093030A20E0EC
:100D400030E048EC52E46091F6097091F709809127
:100D5000F8099091F9090E947DD80E941CD66093F1
:100D6000180A7093190A80931A0A90931B0A8FEA43
:100D700091E7909345028093440282EA94E890932D
:100D8000FF098093FE095ACE86EF99E07A830E948C
:100D900056709C0146EF5FE0612F8A2D0E94725DC4
:100DA0007A8192CF8F929F92AF92BF92FF920F93D0
:100DB0001F93CF93DF9300D01F92CDB7DEB7F09093
:100DC000220AF2FAFF24F0F80091180A1091190A89
:100DD00020911A0A30911B0A37FD98C04801590129
:100DE0004091000A5091010A6091020A7091030A31
:100DF000401751076207730754F44093180A509341
:100E0000190A60931A0A70931B0A4A015B01209128
:100E10004302211157C0FF2009F442C00091080A83
:100E20001091090A6091180A7091190A80911A0AA2
:100E300090911B0A8090040A9090050AA090060ADF
:100E4000B090070A680D791D8A1D9B1D0E944AD625
:100E500020E030E048EC52E40E94AFD5F801608316
:100E600071838283938340910C0A50910D0A809183
:100E70000E0A90910F0A2091440230914502821788
:100E8000930771F090934502809344021092180AE0
:100E90001092190A10921A0A10921B0A452B79F423
:100EA0008F2D0F900F900F900F90DF91CF911F918A
:100EB0000F91FF90BF90AF909F908F9008950E94E8
:100EC000D25EEECF6091040A7091050A8091060A05
:100ED0009091070A680D791D8A1D9B1D0E944AD6B4
:100EE00020E030E048EC52E40E94AFD569837A8379
:100EF0008B839C83CE0101960E947E7EBC018091F3
:100F00000A0A90910B0A0E94D45D85CF1092180AAC
:100F10001092190A10921A0A10921B0A00E010E0AF
:100F20009801812C912C54015BCF3CCF60E087E28B
:100F30009AE00C94585B2F923F924F925F926F927F
:100F40007F928F929F92AF92BF92CF92DF92EF9259
:100F5000FF920F931F93CF93DF93CDB7DEB76897C0
:100F60000FB6F894DEBF0FBECDBF1C012A013B01B6
:100F700048015901DC01D8966D917D918D919C912C
:100F8000DB970E9448D66B017C01A30192010E946D
:100F90007DD80E9495D50E941CD669877A878B8759
:100FA0009C87A5019401C701B6010E947DD80E94CB
:100FB00095D50E941CD66D877E878F87988B298553
:100FC0003A854B855C85283731054105510540F44C
:100FD00088E790E0A0E0B0E089879A87AB87BC877C
:100FE0002D853E854F8558892837310541055105A6
:100FF00040F488E790E0A0E0B0E08D879E87AF875F
:10100000B88B91012C5B3F4FD9018D919D910D9033
:10101000BC91A02D8D839E83AF83B887BC01CD0189
:101020000E944AD669837A838B839C8369857A85FB
:101030008B859C850E9448D6698B7A8B8B8B9C8B89
:1010400020E030E0A90169817A818B819C810E9436
:10105000A8D5882339F1A7019601C701B6010E94DE
:101060007DD84B015C0129893A894B895C89CA0189
:10107000B9010E947DD89B01AC01C501B4010E9459
:10108000CED44B015C0129813A814B815C81CA013C
:10109000B9010E94CFD49B01AC01C501B4010E94EB
:1010A000AFD503C060E070E0CB010E9495D50E94EF
:1010B00017D62B013C016D817E818F81988590959B
:1010C0008095709561957F4F8F4F9F4F0E944AD6B4
:1010D0004B015C016D857E858F8598890E9448D67D
:1010E0006D837E838F83988720E030E0A901C5015E
:1010F000B4010E94A8D5882349F12D813E814F81FA
:101100005885CA01B9010E947DD86D8B7E8B8F8B6B
:10111000988FA7019601C701B6010E947DD89B0157
:10112000AC016D897E898F89988D0E94CED46B0128
:101130007C01A5019401C501B4010E94CFD49B019B
:10114000AC01C701B6010E94AFD503C060E070E0FA
:10115000CB010E9485D6F10180889188A288B3884E
:1011600075016401C418D508E608F7080E9417D66F
:10117000C61AD70AE80AF90AF7FE6BC020E030E089
:10118000A90169817A818B819C810E94A8D58823DD
:1011900009F447C029813A814B815C81CA01B901B8
:1011A0000E94CFD46B017C01C501B4010E9448D6D6
:1011B0009B01AC01C701B6010E947DD86B017C0187
:1011C00029893A894B895C89CA01B9010E947DD875
:1011D0009B01AC01C701B6010E94CED46B017C011A
:1011E0002D813E814F815885CA01B9010E947DD869
:1011F0009B01AC01C701B6010E94CFD46B017C01F9
:1012000020E030E040E850E469817A818B819C8164
:101210000E947DD89B01AC01C701B6010E94AFD5E9
:1012200003C060E070E0CB010E9495D50E9417D604
:101230002B013C0197FF03C0412C512C3201481473
:1012400059046A047B0410F024013501C12CD12C0F
:1012500076018FB7F894F101EC51FF4F9081911115
:1012600025C0D10154964D925D926D927C92579714
:10127000C40CD51CE61CF71CF101C08ED18EE28E89
:10128000F38E29853A854B855C85DC962D933D93BD
:101290004D935C93DF97A05CBF4F2D853E854F85B6
:1012A00058892D933D934D935C9313978FBF689608
:1012B0000FB6F894DEBF0FBECDBFDF91CF911F9167
:1012C0000F91FF90EF90DF90CF90BF90AF909F90E5
:1012D0008F907F906F905F904F903F902F900895E8
:1012E0004F925F926F927F92AF92BF92CF92DF92B6
:1012F000EF92FF920F931F93CF93DF93EB017A014D
:10130000209709F458C04115510509F454C0AAA406
:10131000BBA40CA51DA59501A8016EA17FA188A560
:1013200099A50E94A8D5882309F445C08FA98111E9
:101330003AC0F70146A057A060A471A4A30192018E
:10134000B501C8010E94ABD718166CF5A301920134
:10135000C301B2010E947DD86B017C018AA99BA9BF
:10136000ACA9BDA9BC01CD0190589B01AC010E9464
:10137000CFD42EA53FA548A959A90E947DD89B018D
:10138000AC01C701B6010E94CED40E94EAD86B011D
:101390007C019B01AC01B501C8010E94A8D587FD65
:1013A00002C056018701A501B8014EA35FA368A73B
:1013B00079A781E08EABDF91CF911F910F91FF90C4
:1013C000EF90DF90CF90BF90AF907F906F905F9045
:1013D0004F900895DF92EF92FF920F931F93CF9358
:1013E000DF938091A50C8FB7F894E090A40C8FBF89
:1013F0008091A50C90E08E1991098F709927049720
:10140000E4F01091A50C13501F7040E050E000E094
:10141000F12C85EED82E1E1581F011501F70D19E33
:10142000E0011124CA55D34F602F7F2DCE0158DF24
:10143000402F5F2D0C2FFD2EEECFDF91CF911F910E
:101440000F91FF90EF90DF9008954F925F926F920F
:101450007F92AF92BF92CF92DF92EF92FF920F9363
:101460001F93CF93DF938C01EB01009709F453C0D6
:10147000FC0187A981114FC046A057A060A471A4A8
:10148000AEA0BFA0C8A4D9A49501A601C301B20112
:101490000E94A8D587FF3FC0A3019201C301B201FA
:1014A0000E947DD82B013C01F80182A993A9A4A92F
:1014B000B5A9BC01CD0190589B01AC010E94CFD4CD
:1014C000F80126A537A540A951A90E947DD89B0106
:1014D000AC01C301B2010E94CED40E94EAD87B01C4
:1014E0008C019B01AC01B501C6010E94A8D587FF04
:1014F00002C0750186019701A801B501C6010E94CD
:10150000A8D5882341F0A701B8014EA35FA368A71F
:1015100079A781E08EABDF91CF911F910F91FF9062
:10152000EF90DF90CF90BF90AF907F906F905F90E3
:101530004F900895EF92FF920F931F93CF93DF93F5
:101540001091A40CF12C00E080E090E025EEE22E5A
:101550002091A50C121781F0E19EE0011124CA55DB
:10156000D34FAE016F2D702F70DF1F5F1F708F2D57
:10157000902FFC2E0D2FECCF40E050E06F2D702F00
:10158000DF91CF911F910F91FF90EF905ECF4F921F
:101590005F926F927F928F929F92AF92BF92CF9203
:1015A000DF92EF92FF920F931F93CF93DF93909070
:1015B000A40CC0E0D0E035EE832E892D992787FD5D
:1015C00090952091A50C30E082179307B1F1889E89
:1015D0005001899EB00C1124C5018A55934F5C01BE
:1015E000209729F18EA9811104C0F50186A98823CD
:1015F000F1F0CAA0DBA0ECA0FDA0A7019601F501C7
:1016000066A177A180A591A50E94AFD52B013C01D1
:10161000A70196016EA17FA188A599A50E94AFD5CB
:10162000AB01BC0193018201CE0185DC1EAA93941B
:10163000F92DFF709F2EE501C0CF2097E9F0CAA0D9
:10164000DBA0ECA0FDA0A70196016DEC7CEC8CE486
:101650009DE30E94AFD54B015C01A70196016EA1ED
:101660007FA188A599A50E94AFD5AB01BC019501CA
:101670008401CE0160DC1EAADF91CF911F910F91F2
:10168000FF90EF90DF90CF90BF90AF909F908F90A2
:101690007F906F905F904F9008959CDE4BDF77CFE7
:1016A0001092A40C1092A50C80E1E4E9FCE0DF01AB
:1016B0001D928A95E9F71092840C1092850C109275
:1016C000860C1092870C1092880C1092890C109244
:1016D0008A0C10928B0C10928C0C10928D0C109224
:1016E0008E0C10928F0C1092900C1092910C109204
:1016F000920C1092930C1092800C1092810C10920C
:10170000820C1092830C0895609194049091A50C22
:101710008091A40C981781F08091A40C95EE899F7C
:10172000F0011124E251F34F60819091A50C8917CB
:1017300019F08F5F8F70F9CF70E089E00C94CDD0F5
:101740002F923F924F925F926F927F928F929F92D1
:10175000AF92BF92CF92DF92EF92FF920F931F93BF
:10176000CF93DF93CDB7DEB7C957D1090FB6F89441
:10177000DEBF0FBECDBF2C014B013A011901EFAA0C
:101780002A96FFAE2A970BAF1FAFABAA2091A50CEC
:101790002F5F2F7062962FAF6297E22EFF24E7FC37
:1017A000F0948091A40C90E08E159F0521F480E0C8
:1017B0000E944F40F6CF2091371B3091381B40914B
:1017C000391B50913A1BD2016D917D918D919C9165
:1017D0000E947DD80E944DD8A6966CAF7DAF8EAF8B
:1017E0009FAFA69720913B1B30913C1B40913D1B26
:1017F00050913E1BF40160817181828193810E942E
:101800007DD80E944DD8AA966CAF7DAF8EAF9FAFAA
:10181000AA9720913F1B3091401B4091411B509152
:10182000421BD3016D917D918D919C910E947DD839
:101830000E944DD8AE966CAF7DAF8EAF9FAFAE9786
:101840000C2D10E0F8013396EE0FFF1FEE0FFF1F77
:10185000FAAFE9AFE95CF44E2081318142815381D6
:10186000D1016D917D918D919C910E947DD80E94B6
:101870004DD8E2966CAF7DAF8EAF9FAFE29780916F
:10188000940C9091950CA091960CB091970CA69603
:101890004CAC5DAC6EAC7FACA697481A590A6A0A8C
:1018A0007B0A8091980C9091990CA0919A0CB09120
:1018B0009B0CAA968CAC9DACAEACBFACAA97881A18
:1018C000990AAA0ABB0A80919C0C90919D0CA09148
:1018D0009E0CB0919F0CAE96CCACDDACEEACFFACE8
:1018E000AE97C81AD90AEA0AFB0A8091A00C909117
:1018F000A10CA091A20CB091A30CE2962CAD3DAD31
:101900004EAD5FADE297281B390B4A0B5B0B2FA343
:1019100038A749A75AA78091A50C35EE839F1001DF
:101920001124A1014A55534F1A01FA01EC51FF4FFE
:1019300010824BA25CA26DA27EA277FE0BC066272E
:101940007727CB0164197509860997096BA37CA3D6
:101950008DA39EA38BA19CA1ADA1BEA1F10180830B
:101960009183A283B3838BA69CA6ADA6BEA6B7FE29
:101970000BC022273327A901281939094A095B0915
:101980002BA73CA74DA75EA74BA55CA56DA57EA583
:10199000D10114964D935D936D937C931797CFA6C9
:1019A000D8AAE9AAFAAAF7FE0BC022273327A90171
:1019B0002C193D094E095F092FA738AB49AB5AAB2B
:1019C0004FA558A969A97AA9D10118964D935D939D
:1019D0006D937C931B976FA178A589A59AA597FF16
:1019E00007C090958095709561957F4F8F4F9F4F61
:1019F0000E944AD6F801EE0FFF1FEE0FFF1F25963B
:101A0000FFAFEEAF2597E15EFD4F2081318142812E
:101A100053810E947DD80E9417D69B01AC01F8012A
:101A2000EE0FFF1FE75DFD4FA081B1810E94E3D95A
:101A300024E630E040E050E00E94A8D929962CAF7F
:101A40003DAF4EAF5FAF2997D1011C962D933D93CB
:101A50004D935C931F972FA538A949A95AA96BA547
:101A60007CA58DA59EA5261737074807590724F49E
:101A70006FA778AB89AB9AAB8FA598A9A9A9BAA98A
:101A800029962CAD3DAD4EAD5FAD299782179307DA
:101A9000A407B50714F4DA01C9013BA13BA74CA187
:101AA0004FA73DA12EA14BA15CA16DA17EA148171E
:101AB00059076A077B0724F48BA79FA73A2F2B2F80
:101AC000EBA5D1015096EC935097FFA55196FC934E
:101AD000519752963C93529753962C93F101E85BA1
:101AE000FF4F8091940490919504AA2797FDA095AB
:101AF000BA2F80839183A283B383D301C201882745
:101B0000B7FD83959927AA27BB27282FB7FC22600A
:101B1000F7FC24604FA158A569A57AA577FD286038
:101B2000D10190962C939097EBA99196EC932BA1D1
:101B30003CA14DA15EA1232B242B252B09F05F98FE
:101B4000F10184819581A681B781892B8A2B8B2B0A
:101B500009F08A98F10180859185A285B385892B4A
:101B60008A2B8B2B41F09FB7F894809108018E7FD0
:101B7000809308019FBFF10184859585A685B7856F
:101B8000892B8A2B8B2B09F01298F101848595857E
:101B9000A685B785892B8A2B8B2B29F1F091231BE6
:101BA000FBA32091241B2BA73091251B3FA740911D
:101BB000261B4BAB2F2F3BA54FA55BA96FA92A96E0
:101BC0007FAD2A978BAD9FAD0E94A8D587FD1CC025
:101BD0005FA95BA32A966FAD2A976BA77BAD7FA702
:101BE0008FAD8BAB11C09091071B9BA3A091081BDD
:101BF000ABA7B091091BBFA7E0910A1BEBAB292F44
:101C00003A2F4B2F5E2FDACFC301B2010E944AD682
